:020000040800F2
:10000000586101206D020008A5C0000825A700085E
:1000100085BE00089534000861F700080000000064
:1000200000000000000000000000000091CD00086A
:10003000A15000080000000011C6000891E000086F
:10004000870200088702000887020008870200086C
:100050008702000887020008F153000887020008A1
:100060008702000887020008FD5300088702000885
:10007000594E00088702000887020008870200081E
:10008000870200088702000887020008870200082C
:1000900099340008A93400088702000809540008B0
:1000A000870200088702000887020008870200080C
:1000B00087020008870200088702000887020008FC
:1000C00087020008870200088702000887020008EC
:1000D0008702000819F700088702000829F70008BE
:1000E00087020008870200088702000887020008CC
:1000F00087020008870200088702000887020008BC
:1001000087020008870200088702000887020008AB
:10011000870200088702000887020008870200089B
:1001200087020008694E0008794E0008894E0008D1
:10013000870200088702000887020008870200087B
:10014000B9340008C9340008870200088702000893
:10015000994E0008A94E00088702000845F70008DC
:10016000870200088702000887020008870200084B
:1001700087020008870200088702000800000000CC
:10018000870200088702000800F002F800F05EF81D
:100190000AA090E8000C82448344AAF10107DA45E2
:1001A00001D100F053F8AFF2090EBAE80F0013F0D6
:1001B000010F18BFFB1A43F001031847BC7D010073
:1001C000DC7D01000A444FF0000C10F8013B13F0F5
:1001D000070408BF10F8014B1D1108BF10F8015BA0
:1001E000641E05D010F8016B641E01F8016BF9D193
:1001F00013F0080F1EBF10F8014BAD1C0C1B09D1EA
:100200006D1E58BF01F801CBFAD505E014F8016B5B
:1002100001F8016B6D1EF9D59142D6D370470000ED
:100220000023002400250026103A28BF78C1FBD8FF
:10023000520728BF30C148BF0B6070471FB517F089
:10024000E2FB00F0C0F81FBD10B510BD00F080F952
:100250001146FFF7F3FF0FF071FD00F09EF903B4B4
:10026000FFF7F2FF03BC00F0A1F900000948804746
:1002700009480047FEE7FEE7FEE7FEE7FEE7FEE788
:10028000FEE7FEE7FEE7FEE704480549054A064BA0
:100290007047000065E1000889010008583101201D
:1002A00058610120584101205841012053EA020CB5
:1002B00000F069802DE9F04B4FF00006002B1FBFC6
:1002C000B3FA83F503FA05F424FA05F65E4012BF8B
:1002D0001643B2FA82F502FA05F4C5F120051EBFF5
:1002E00022FA05FC44EA0C04203556EA044C4FEA95
:1002F000144418BF641C4FF000084FF000099042EE
:1003000071EB030C39D3002919BFB1FA81F701FA57
:1003100007F6B0FA80F700FA07F6C7F120071EBF0C
:1003200020FA07FC46EA0C062037B6FBF4FCA7EBE4
:100330000507103F07F01F0BCBF120062CFA06F63D
:100340000CFA0BFB44BFB3460026202FA4BF5E4629
:100350004FF0000B5BEA060C08BF4FF0010B19EBE6
:100360000B0948EB0608ABFB027C06FB02CC0BFB3F
:1003700003CCC01B71EB0C01C1E70B4602464146A2
:100380004846BDE8F08B13B5084318BF4FF0FF3067
:100390000146AFF30080BDE81C4070470B4910B523
:1003A000A1F17C020A4CC2E93712372106E000EBCA
:1003B000104342F82130074B00FB03400B1EA1F114
:1003C0000101F4DC10BD0120E8E70000FC0300207F
:1003D000E119D666CD0D0100032A40F2308010F0FD
:1003E000030C00F0158011F8013BBCF1020F6244D0
:1003F00098BF11F801CB00F8013B38BF11F8013B61
:10040000A2F1040298BF00F801CB38BF00F8013B0D
:1004100011F0030300F02580083AC0F0088051F87D
:10042000043B083A51F804CBA0E80810F5E7121D88
:100430005CBF51F8043B40F8043BAFF30080D207A7
:1004400024BF11F8013B11F801CB48BF11F8012B73
:1004500024BF00F8013B00F801CB48BF00F8012B96
:10046000704710B5203AC0F00B80B1E81850A0E8F2
:100470001850B1E81850A0E81850203ABFF4F5AF72
:100480005FEA027C24BFB1E81850A0E8185044BFCE
:1004900018C918C0BDE810405FEA827C24BF51F83B
:1004A000043B40F8043B08BF7047D20728BF31F82F
:1004B000023B48BF11F8012B28BF20F8023B48BF80
:1004C00000F8012B704702F0FF0343EA032242EADF
:1004D000024200F002B84FF0000200B51346944605
:1004E0009646203922BFA0E80C50A0E80C50B1F18C
:1004F0002001BFF4F7AF090728BFA0E80C5048BFA0
:100500000CC05DF804EB890028BF40F8042B08BF3D
:10051000704748BF20F8022B11F0804F18BF00F839
:10052000012B704770477047704710B500F008F80E
:10053000006810BD10B5044600F002F8046010BD5C
:10054000004870476404002000487047640400209D
:100550007546FFF7F9FFAE4605006946534620F0A1
:100560000700854618B020B5FFF78EFEBDE8204095
:100570004FF000064FF000074FF000084FF0000B5F
:10058000AC46ACE8C009ACE8C009ACE8C009ACE8CE
:10059000C00921F007018D46704710B50446AFF33E
:1005A00000802046BDE81040FFF759BE01491820E1
:1005B000ABBEFEE7260002007047000080B58AB09F
:1005C00008900791089820B9FFE7FF208DF82700D1
:1005D0009BE0079820B9FFE7FF208DF8270094E003
:1005E000079890ED000A90ED013A90ED021A90ED17
:1005F000032A20EE030A21EE021A30EE010A30EE41
:10060000000A8DED060A079890ED010A90ED021A96
:1006100020EE000A21EE011A30EE010A30EE001A37
:10062000B7EE000A8DED010A30EE410A8DED050AA4
:100630009DED060ADDED050A14F03AF99DED011A6B
:10064000089880ED010A079890ED000A90ED013AB4
:1006500090ED024A90ED032A20EE040A22EE032ACE
:1006600030EE420A30EE000A8DED040A9DED040AD8
:10067000B0EEC00AB4EE410AF1EE10FA0ADBFFE771
:10068000DDED040A9FED230A0FF0A0FA089880ED33
:10069000020A07E09DED040A13F008FE089880EDB9
:1006A000020AFFE7079890ED000A90ED011A90ED1D
:1006B000022A90ED033A20EE030A21EE021A30EEF0
:1006C000010A30EE000A8DED030A079890ED020A48
:1006D00090ED031A20EE000A21EE011A30EE010A15
:1006E00030EE001AB7EE000A30EE410A8DED020A34
:1006F0009DED030ADDED020A14F0DAF8089880EDAA
:10070000000A00208DF82700FFE79DF927000AB0B6
:1007100080BD00BFDB0FC93F80B58CB00A90099146
:100720008DED080A0A9820B9FFE7FF208DF82F0009
:1007300029E19DED081AB7EE000A80EE010A0A9839
:1007400080ED040A0A994FF07E5008600A99002053
:1007500048600A9988600A99C8600998002800F0E2
:100760000E81FFE7099801680091406817F080F852
:100770000246009801920A46019942EC101B8DED49
:10078000020B17F075F89DED020B41EC110B13F005
:100790008FFF8DED040B9DF8170080F080008DF821
:1007A00017000498059916F03DF90790099890ED07
:1007B000000AB5EE400AF1EE10FA2BD1FFE70998D6
:1007C00090ED010AB5EE400AF1EE10FA22D1FFE7F2
:1007D000099890ED020AB5EE400AF1EE10FA19D12F
:1007E000FFE70A9940F2C560C3F64D7008600A99A8
:1007F00044F62D20C3F60D4048600A994AF256404F
:10080000CBF6393088600A9944F2AD70C3F619709E
:10081000C860B3E09DED070A9FED5D1AB4EE410A92
:10082000F1EE10FA08DBFFE79DED070AB5EE400A8E
:10083000F1EE10FA19DDFFE70A9945F66E10C3F6DE
:100840007F7008600A9945F20C30C3F6B01048601A
:100850000A9948F6AB00CBF6BB3088600A9949F29A
:100860008550C3F69750C86087E09DED070A9FED5D
:10087000491AB4EE410AF1EE10FA0ADBFFE79DEDEA
:10088000070A9FED431AB4EE410AF1EE10FA19DDA2
:10089000FFE70A9940F2C560C3F64D7008600A99F7
:1008A00044F62D20C3F60D4048600A994AF256409E
:1008B000CBF6393088600A9944F2AD70C3F61970EE
:1008C000C86059E09DED070A9FED331AB4EE410A66
:1008D000F1EE10FA0ADBFFE79DED070A9FED2D1AF6
:1008E000B4EE410AF1EE10FA19DDFFE70A9940F281
:1008F000C560C3F64D7008600A9944F62D20C3F612
:100900000D4048600A994AF25640CBF6393088606B
:100910000A9944F2AD70C3F61970C8602BE09DEDE2
:10092000070A9FED1D1AB4EE410AF1EE10FA08DB3A
:10093000FFE79DED070AB5EE400AF1EE10FA19DD6A
:10094000FFE70A9940F2C560C3F64D7008600A9946
:1009500044F62D20C3F60D4048600A994AF25640ED
:10096000CBF6393088600A9944F2AD70C3F619703D
:10097000C860FFE7FFE7FFE7FFE7FFE7FFE70020CB
:100980008DF82F00FFE79DF92F000CB080BD00BF50
:10099000DB0FC93FDB0F49400000B44281B000903B
:1009A0000099002088604860086001B0704700002E
:1009B00080B52DED048BB2B030902F912E922D93F7
:1009C000309828B9FFE7FF208DF8C70000F0F7BD89
:1009D0002F9828B9FFE7FF208DF8C70000F0EFBD82
:1009E0002E9828B9FFE7FF208DF8C70000F0E7BD7B
:1009F00040F20401C2F200014EF69E70C3F6275089
:100A000008602D9848B9FFE730982F992E9A00F08A
:100A1000DDFD8DF8C70000F0D2BD2D98006809906B
:100A20002D98406808902D98806807909DED090AE0
:100A3000B5EE400AF1EE10FA19D1FFE79DED080A74
:100A4000B5EE400AF1EE10FA11D1FFE79DED070A6D
:100A5000B5EE400AF1EE10FA09D1FFE730982F9970
:100A60002E9A00F0B3FD8DF8C70000F0A8BD2F98B6
:100A7000006806902F98406805902F988068049031
:100A80002E98006803902E98406802902E988068F7
:100A9000019030989DED033A90ED010A90ED022A05
:100AA00090ED031A20EE430A9DED023A22EE032A4E
:100AB00030EE420A9DED012A21EE021A30EE410A83
:100AC000B6EE001A20EE010A8DED270A30989DED52
:100AD000034A90ED000A90ED023A90ED032A20EED1
:100AE000040A9DED014A23EE043A30EE030A9DED1F
:100AF000023A22EE032A30EE420A20EE010A8DED80
:100B0000260A30989DED024A90ED000A90ED013AD8
:100B100090ED032A20EE040A9DED014A23EE043AEB
:100B200030EE430A9DED033A22EE032A30EE020A2C
:100B300020EE010A8DED250A30989DED014A90EDD9
:100B4000000A90ED013A90ED022A20EE040A9DED94
:100B5000024A23EE043A30EE030A9DED033A22EEF8
:100B6000032A30EE420A20EE010A8DED240A9DEDA3
:100B7000060AB5EE400AF1EE10FA11D1FFE79DED3D
:100B8000050AB5EE400AF1EE10FA09D1FFE79DED36
:100B9000040AB5EE400AF1EE10FA00F09984FFE77E
:100BA0009DED060A20EE000A9DED051A21EE011AC0
:100BB00030EE010A9DED041A21EE011A30EE010A11
:100BC00009F0B2FD8DED2C0A9DED2C1A9DED060A63
:100BD00020EE010A8DED060A9DED2C1A9DED050A09
:100BE00020EE010A8DED050A9DED2C1A9DED040AFB
:100BF00020EE010A8DED040A9DED090A20EE000A9F
:100C00009DED081A21EE011A30EE010A9DED071A3A
:100C100021EE011A30EE010A09F086FD8DED2C0A55
:100C20009DED2C1A9DED090A20EE010A8DED090AB1
:100C30009DED2C1A9DED080A20EE010A8DED080AA3
:100C40009DED2C1A9DED070A20EE010A8DED070A95
:100C5000309890ED000A30EE000A9DED091A20EE62
:100C6000010A8DED210A309890ED000A30EE000A5D
:100C70009DED081A20EE010A8DED200A309890EDC6
:100C8000000A30EE000A9DED071A20EE010A8DEDF4
:100C90001F0A309890ED010A30EE000A9DED091A06
:100CA00020EE010A8DED1E0A309890ED000A30EE1C
:100CB000000A8DED190A309890ED010A30EE000A15
:100CC0008DED180A309890ED020A30EE000A8DED95
:100CD000170A309890ED030A30EE000A8DED160ADF
:100CE000309890ED000A90ED021A30EE000A20EEE6
:100CF000010A8DED150A309890ED020A90ED031A65
:100D000030EE000A20EE010A8DED140A309890EDC5
:100D1000000A20EE000A8DED130A309890ED000ACB
:100D200090ED011A20EE010A8DED120A309890ED37
:100D3000000A90ED021A20EE010A8DED110A30989A
:100D400090ED000A90ED031A20EE010A8DED100AD5
:100D5000309890ED010A20EE000A8DED0F0A3098D0
:100D600090ED010A90ED021A20EE010A8DED0E0AB7
:100D7000309890ED010A90ED031A20EE010A8DEDF6
:100D80000D0A309890ED020A20EE000A8DED0C0A53
:100D9000309890ED020A90ED031A20EE010A8DEDD5
:100DA0000B0A309890ED030A20EE000A8DED0A0A36
:100DB0009DED091A9DED130A21EE000A9DED202AF2
:100DC000309890ED025A90ED033A22EE032A30EE6D
:100DD000420A9DED1F2A22EE052A30EE020A9DED01
:100DE0000F2A21EE022A30EE020A9DED182A9DED0F
:100DF000084A22EE044A24EE054A30EE040A9DED2C
:100E0000074A22EE042A22EE032A30EE020A9DED62
:100E10000C2A21EE022A30EE420A9DED0A2A21EE2A
:100E2000021A30EE410A8DED230A9DED210A309819
:100E300090ED015A90ED024A90ED033A20EE030A3C
:100E40009DED081A9DED132A21EE022A30EE020ACA
:100E50009DED1F2A22EE052A30EE420A9DED1E2A44
:100E600022EE042A30EE020A9DED0F2A21EE022A1C
:100E700030EE420A9DED0C2A21EE022A30EE020AE3
:100E80009DED172A9DED074A22EE042A22EE032A41
:100E900030EE020A9DED0A2A21EE021A30EE410AD6
:100EA0008DED220A9DED230A20EE000A9DED221A07
:100EB00021EE011A30EE010A09F036FCB7EE006AA5
:100EC00086EE000A8DED1D0A9DED210A309890ED09
:100ED000012A90ED021A90ED033A20EE011A9DEDE1
:100EE000200A20EE020A30EE412A9DED071A9DED00
:100EF000130A21EE000A30EE022A9DED1E0A20EEB2
:100F0000030A30EE020A9DED0F2A21EE022A30EE8E
:100F1000420A9DED172A9DED084A22EE042A22EE90
:100F2000032A30EE020A9DED0C2A21EE022A30EE51
:100F3000420A9DED0A2A21EE021A30EE010A8DEDD9
:100F40001C0A9DED1D0A30EE000A8DED1B0A9DED79
:100F50001C0A30EE000A8DED1A0A9DED170ADDED30
:100F60000D0A30EEA02A9DED151A31EE422A9DEDB4
:100F7000061A31EE021A20EE010A9DED181ADDED77
:100F8000123A33EEA32A9DED143A32EE032A9DED78
:100F9000053A32EE432A21EE021A70EE014A9DED27
:100FA0001C3A309890ED011A90ED020AD0ED032A18
:100FB00063EE001A9DED1D2A9DED0C7AB6EE004AF7
:100FC0008DED004A77EE445A9DED0A5A35EE255ACA
:100FD00062EE055A9DED115A75EE606A63EE266A5F
:100FE00075EEA66ADDED095A75EEA65A61EEA51AF0
:100FF00071EEA41A62EE222A23EE011A31EE621A71
:10100000DDED0E2ADDED104A72EEE42A62EE222AB0
:10101000DDED0B4A73EEA43A63EE233A72EEA32A97
:10102000DDED083A72EEE32A21EE221A31EE211AA2
:1010300022EE000A35EE205A22EE052A9DED0F5AC7
:1010400034EE455A35EE475A23EE053A32EE032A7E
:101050009DED073A32EE432A20EE020A30EE010AF5
:101060008DED2B0A9DED160ADDED0D2A32EEA21A4A
:101070009DED152A31EE421A9DED062A31EE421AF7
:1010800020EE010A9DED191ADDED126A36EEA62A50
:101090009DED143A32EE032A9DED053A32EE432AD5
:1010A00021EE021A30EE011A3098D0ED005AD0ED40
:1010B000014AD0ED023A90ED032AB1EE000A24EE87
:1010C000803A9DED0F7A37EE075A75EE461ADDED40
:1010D0000C0A30EEA05A75EE211A9DED045A35EE39
:1010E000215A23EE053A31EE031A9DED1C5A65EEA6
:1010F000027A9DED1D3A74EE601A9DED0A8A71EE3A
:10110000C81A23EE218ADDED111A32EEE19A25EE9E
:10111000099A38EE098A9DED099A38EE498A67EEF8
:10112000887A31EE271A63EE233A65EE255A73EE7C
:10113000A53ADDED0E5ADDED107A75EEE75A63EE55
:10114000255ADDED0B7A76EEA76A65EE266A75EE16
:10115000A65ADDED086A75EEE65A63EEA53A31EE61
:10116000231A23EE022ADDED1A3A63EEA43A32EE98
:10117000632A71EEA21A23EE213A34EE477A37EE53
:10118000607A25EE075A33EE053A9DED075A33EEA5
:10119000453A22EE032A31EE021A8DED2A1A9DED10
:1011A000191ADDED0D0A30EEA03A9DED152A32EE4A
:1011B000433A9DED062A32EE032A21EE021A9DEDF6
:1011C000162ADDED124A34EEA43A9DED145A33EEA0
:1011D000053A9DED055A33EE453A22EE032A31EEEB
:1011E000022A309890ED001AD0ED011AD0ED022AB3
:1011F000D0ED033A22EE800A9DED0F5A35EE053A06
:1012000033EE467A9DED0C6A36EE063A33EE077AF7
:101210009DED043A33EE073A20EE030A70EE025ACF
:101220009DED1B0A20EE620A9DED1C3A23EE012A79
:1012300030EE420A9DED1D2A34EE467ADDED0A6A53
:1012400037EE667A62EE076A9DED117A70EEC77A24
:1012500063EE277A76EEA76ADDED097A76EEE76A25
:1012600020EE260A30EE250A62EE211A63EE233ABA
:1012700071EEA31ADDED0E3ADDED105A73EEE53A8C
:1012800062EE233ADDED0B5A74EEA54A63EE244A72
:1012900073EEA43ADDED084A73EEE43A61EEA31A68
:1012A00030EE210A22EE011ADDED1A1A61EEA21AC1
:1012B00031EE611A37EE207A22EE072A34EE455AD3
:1012C00035EE465A23EE053A32EE032A9DED073AF3
:1012D00032EE432A21EE021A30EE010A8DED290A80
:1012E0009DED180A9DED0D7A37EE071A9DED152A32
:1012F00031EE421A9DED062A31EE421A20EE010A25
:101300009DED171ADDED122A32EEA22A9DED143A58
:1013100032EE032A9DED053A32EE432A21EE021AFF
:1013200070EE013A9DED1B1A3098D0ED001A90ED49
:10133000010AD0ED020A90ED032A21EE022A9DED6A
:101340001C3A23EE001A31EE421A9DED1D2A9DED46
:101350000C5A34EE456ADDED0A4A36EE646A62EEF6
:10136000064A9DED116A77EE465A63EE255A74EEF1
:10137000A54ADDED095A74EEE54A21EE241A31EE54
:10138000231A62EE211A63EE200A70EEE10ADDED07
:101390000E1ADDED103A71EEE31A62EE211ADDED60
:1013A0000B3A72EEA32A63EE222A71EEA21ADDED49
:1013B000082A71EEE21A60EEA10A31EE201A22EE3E
:1013C000000A36EE076A22EE062A9DED0F6A34EE19
:1013D000464A34EE454A23EE043A32EE032A9DEDA6
:1013E000073A32EE432A20EE020A30EE010A8DED72
:1013F000280A9DED2B0A20EE000A9DED2A1A21EE07
:10140000011A30EE010A9DED291A21EE011A30EE83
:10141000010A9DED281A21EE011A30EE010A09F0A9
:1014200083F98DED2C0A9DED2C1A9DED2B0A20EEF3
:10143000010A8DED2B0A9DED2C1A9DED2A0A20EE56
:10144000010A8DED2A0A9DED2C1A9DED290A20EE48
:10145000010A8DED290A9DED2C1A9DED280A20EE3A
:10146000010A8DED280A40F20400C2F2000090ED5E
:10147000000A9DED2B1A20EE011A9DED270A30EE91
:10148000410A8DED270A90ED000A9DED2A1A20EE03
:10149000011A9DED260A30EE410A8DED260A90EDE7
:1014A000000A9DED291A20EE011A9DED250A30EE65
:1014B000410A8DED250A90ED000A9DED281A20EED7
:1014C000011A9DED240A30EE410A8DED240AFFE752
:1014D0009DED271A309890ED000A90ED042A21EE38
:1014E000021A30EE010A80ED000A9DED261A3098AE
:1014F00090ED010A90ED042A21EE021A30EE010A65
:1015000080ED010A9DED251A309890ED020A90EDCC
:10151000042A21EE021A30EE010A80ED020A9DED46
:10152000241A309890ED030A90ED042A21EE021A55
:1015300030EE010A80ED030A309890ED000A90ED3C
:10154000013A90ED022A90ED031A20EE000A23EEF4
:10155000033A30EE030A22EE022A30EE020A21EEAE
:10156000011A30EE010A09F0DFF88DED2C0A9DED2D
:101570002C1A309890ED000A20EE010A80ED000A46
:101580009DED2C1A309890ED010A20EE010A80EDB5
:10159000010A9DED2C1A309890ED020A20EE010A06
:1015A00080ED020A9DED2C1A309890ED030A20EE92
:1015B000010A80ED030A00208DF8C700FFE79DF9BE
:1015C000C70032B0BDEC048B80BD000080B5A0B078
:1015D0001E901D911C921E9820B9FFE7FF208DF8E8
:1015E0007F00D3E21D9820B9FFE7FF208DF87F0030
:1015F000CCE21C9820B9FFE7FF208DF87F00C5E200
:1016000040F20401C2F2000142F60230C3F6075074
:1016100008601D9800681B901D9840681A901D98DE
:10162000806819901C98006818901C984068179062
:101630001C98806816901E989DED183A90ED010A4E
:1016400090ED022A90ED031A20EE430A9DED173A21
:1016500022EE032A30EE420A9DED162A21EE021AEE
:1016600030EE410AB6EE001A20EE010A8DED100AA6
:101670001E989DED184A90ED000A90ED023A90ED0B
:10168000032A20EE040A9DED164A23EE043A30EEBA
:10169000030A9DED173A22EE032A30EE420A20EEAD
:1016A000010A8DED0F0A1E989DED174A90ED000A74
:1016B00090ED013A90ED032A20EE040A9DED164AC2
:1016C00023EE043A30EE430A9DED183A22EE032A47
:1016D00030EE020A20EE010A8DED0E0A1E989DEDF5
:1016E000164A90ED000A90ED013A90ED022A20EEA4
:1016F000040A9DED174A23EE043A30EE030A9DEDED
:10170000183A22EE032A30EE420A20EE010A8DED4D
:101710000D0A9DED1B0AB5EE400AF1EE10FA11D14B
:10172000FFE79DED1A0AB5EE400AF1EE10FA09D175
:10173000FFE79DED190AB5EE400AF1EE10FA00F050
:10174000AE81FFE79DED1B0A20EE000A9DED1A1AFF
:1017500021EE011A30EE010A9DED191A21EE011A4F
:1017600030EE010A08F0E0FF8DED150A9DED151A27
:101770009DED1B0A20EE010A8DED1B0A9DED151A49
:101780009DED1A0A20EE010A8DED1A0A9DED151A3B
:101790009DED190A20EE010A8DED190A1E9890EDB3
:1017A000000A30EE000A8DED0C0A1E9890ED010A39
:1017B00030EE000A8DED0B0A1E9890ED020A30EE15
:1017C000000A8DED0A0A1E9890ED030A30EE000A19
:1017D0008DED090A1E9890ED000AB1EE003A20EE58
:1017E000030A8DED080A1E9890ED010A20EE030A07
:1017F0008DED070A1E9890ED020A20EE030A8DED8A
:10180000060A1E9890ED010AB2EE001A20EE010AB7
:101810008DED050A1E9890ED020A20EE010A8DED6D
:10182000040A1E9890ED000A20EE000A8DED030ACE
:101830001E9890ED010A20EE000A8DED020A1E9816
:1018400090ED020A20EE000A8DED010A1E9890ED3F
:10185000030A20EE000A8DED000A9DED081A9DEDA9
:10186000010A21EE000A9DED0A2A9DED1B4A22EE97
:10187000042A30EE020A9DED022A21EE021A30EE11
:10188000010A9DED0B1A9DED1A2A21EE021A30EE87
:10189000410A8DED140A9DED071A9DED000A21EE17
:1018A000000A9DED092A9DED1B4A22EE042A30EE26
:1018B000420A9DED032A22EE032A1E9890ED014A6A
:1018C00022EE042A30EE020A9DED0C2A9DED1A4A02
:1018D00022EE042A30EE420A30EE410A9DED052A3E
:1018E0009DED024A22EE044A30EE040A9DED014AC3
:1018F00022EE042A30EE020A9DED192A21EE021A88
:1019000030EE010A8DED130A9DED030A20EE030A65
:101910001E9890ED021A20EE010A9DED0C1A9DED25
:101920001B2A21EE021A30EE010A9DED061A9DEDEA
:10193000002A21EE022A30EE020A9DED092A9DEDD1
:101940001A4A22EE042A30EE420A30EE410A9DED98
:10195000042A9DED024A22EE044A30EE040A9DED6F
:10196000014A22EE042A30EE020A9DED192A21EEE8
:10197000021A30EE010A8DED120A9DED020A20EEE8
:10198000030A1E9890ED032A20EE020A9DED0B1A21
:101990009DED1B4A21EE041A30EE410A9DED011A1D
:1019A00021EE031A21EE021A30EE010A9DED0A1A09
:1019B0009DED1A2A21EE021A30EE410A8DED110A30
:1019C0009DED140A20EE000A9DED131A21EE011A76
:1019D00030EE010A9DED121A21EE011A30EE010AD5
:1019E0009DED111A21EE011A30EE010A08F09CFE5D
:1019F0008DED150A9DED151A9DED140A20EE010AD4
:101A00008DED140A9DED151A9DED130A20EE010AC5
:101A10008DED130A9DED151A9DED120A20EE010AB7
:101A20008DED120A9DED151A9DED110A20EE010AA9
:101A30008DED110A40F20400C2F2000090ED000AA0
:101A40009DED141A20EE011A9DED100A30EE410AA8
:101A50008DED100A90ED000A9DED131A20EE011A8B
:101A60009DED0F0A30EE410A8DED0F0A90ED000A50
:101A70009DED121A20EE011A9DED0E0A30EE410A7C
:101A80008DED0E0A90ED000A9DED111A20EE011A5F
:101A90009DED0D0A30EE410A8DED0D0AFFE79DED3B
:101AA000101A1E9890ED000A90ED042A21EE021AF9
:101AB00030EE010A80ED000A9DED0F1A1E9890EDA0
:101AC000010A90ED042A21EE021A30EE010A80ED9F
:101AD000010A9DED0E1A1E9890ED020A90ED042A5F
:101AE00021EE021A30EE010A80ED020A9DED0D1A78
:101AF0001E9890ED030A90ED042A21EE021A30EEB2
:101B0000010A80ED030A1E9890ED000A90ED013A5B
:101B100090ED022A90ED031A20EE000A23EE033A1C
:101B200030EE030A22EE022A30EE020A21EE011AFA
:101B300030EE010A08F0F8FD8DED150A9DED151A3D
:101B40001E9890ED000A20EE010A80ED000A9DED3E
:101B5000151A1E9890ED010A20EE010A80ED010A87
:101B60009DED151A1E9890ED020A20EE010A80EDF7
:101B7000020A9DED151A1E9890ED030A20EE010A47
:101B800080ED030A00208DF87F00FFE79DF97F00BC
:101B900020B080BD84B08DED030ACDED020A9DED2D
:101BA000030A9DED021AB1EE411AB4EE410AF1EEBC
:101BB00010FA07DAFFE79DED020AB1EE400A8DED5B
:101BC000010A18E09DED030A9DED021AB4EE410AE8
:101BD000F1EE10FA05DDFFE79DED020A8DED000A3A
:101BE00004E09DED030A8DED000AFFE79DED000A7C
:101BF0008DED010AFFE79DED010A04B0704700007A
:101C000080B542F25810C2F20000006808210EF0C0
:101C10009BFC80BD80B582B040F22862C2F2000217
:101C2000002001901221132300F02CFA019802B039
:101C300080BD000080B5022001214FF0FF320EF080
:101C4000D5FC80BD81B000909FED010A01B07047C6
:101C50000000C84380B542F25810C2F2000000688C
:101C600010210EF071FC80BD80B540F22860C2F2F8
:101C70000000C21D01200221062300F003FA00200B
:101C800080BD000080B5042001214FF0FF320EF02E
:101C9000ADFC80BD80B58AB008900791089820B946
:101CA000FFE7FE208DF82700B4E0079820B9FFE792
:101CB000FE208DF82700ADE041F24140C2F2000065
:101CC0000078C00720B1FFE7FD208DF82700A1E0D4
:101CD0000EF01AFD42F25811C2F20001086020B95C
:101CE000FFE7FE208DF8270094E007980899C86266
:101CF000002006907E21B622049200F059FA049A40
:101D00000120142100F054FA1E20059001F09CFAE5
:101D10000599069800F0F2F90699084600F0EEF9E8
:101D20001E2804D0FFE7FC208DF8270072E0012078
:101D3000002100F0E3F90F2804D0FFE7FC208DF824
:101D4000270067E00320019001F014F804200290BE
:101D500001F010F842F22902C0F6000200200390C0
:101D60000121009101F00EFA019841F60141C0F6FF
:101D7000000101F079F8029841F65541C0F60001E2
:101D800001F072F803984021AA2200F011FA009A9B
:101D90000398412100F00CFA03985321082200F027
:101DA00007FA029A0398582100F002FA029A03985F
:101DB0007D2100F0FDF9322001F046FA009A0F2152
:101DC000104600F0F5F90098019A102100F0F0F9A2
:101DD0000098039A162100F0EBF9009A182110469A
:101DE00000F0E6F900981521802200F0E1F90A20C0
:101DF00001F02AFA0099019841F24142C2F2000230
:101E0000117000F0E1FF029800F0DEFF03988DF8FA
:101E10002700FFE79DF927000AB080BD84B002903B
:101E2000029820B9FFE7FE208DF80F006AE040F22B
:101E30002861C2F20001B1F80100ADF80600B1F866
:101E40000300ADF80400B1F80500ADF80200BDF9DB
:101E5000060000EE100AB8EEC00A029880ED040AEF
:101E6000BDF9040000EE100AB8EEC00A029880ED39
:101E7000050ABDF9020000EE100AB8EEC00A029889
:101E800080ED060A029890ED040A9FED201A80EE7C
:101E9000010A80ED040A029890ED050A80EE010A1D
:101EA00080ED050A029890ED060A80EE010A80EDA9
:101EB000060A487C897CC00040EA5110ADF8000059
:101EC000BDF90000B0F5806F07DBFFE7BDF800004B
:101ED000A0F50060ADF80000FFE7BDF9000000EEDE
:101EE000100AB8EEC00AB4EE001A20EE010AB3EEF2
:101EF000071A30EE010A029880ED0A0A00208DF8D8
:101F00000F00FFE79DF90F0004B0704700A0AA453D
:101F100084B00290029820B9FFE7FE208DF80F00F0
:101F20007AE040F22860C2F20000B0F80710ADF885
:101F30000610B0F80910ADF80410B0F80B00ADF8B9
:101F40000200BDF9060000EE100AB8EEC00A0298C1
:101F500080ED070ABDF9040000EE100AB8EEC00AD1
:101F6000029880ED080ABDF9020000EE100AB8EEF2
:101F7000C00A029880ED090A029890ED070A9FEDC9
:101F8000281A80EE010A80ED070A029890ED080AEF
:101F900080EE010A80ED080A029890ED090A80EEB1
:101FA000010A80ED090A029890ED070A9FED1D1ABB
:101FB00020EE010A80ED070A029890ED080A20EE53
:101FC000010A80ED080A029890ED090A20EE010A44
:101FD00080ED090A0298C16A91ED001A90ED070A96
:101FE00030EE410A80ED070A0298C16A91ED011AAC
:101FF00090ED080A30EE410A80ED080A0298C16AA5
:1020000091ED021A90ED090A30EE410A80ED090ABD
:10201000FE208DF80F00FFE79DF90F0004B0704718
:102020006F12034235FA8E3C80B5012000F0F6FEB7
:1020300068B9FFE70121084600F05EFF42F2581040
:10204000C2F20000006802210EF07EFAFFE70220D3
:1020500000F0E4FE68B9FFE70220012100F04CFF28
:1020600042F25810C2F20000006804210EF06CFA2F
:10207000FFE780BD80B5182001214FF0FF320EF040
:10208000B5FA80BD80B586B08DF817008DF81610B2
:1020900004928DF80F30049808B9FFE72BE09DF803
:1020A00017000146029120B1FFE70298012805D0F0
:1020B00009E00120002100F01FFF04E002200021C0
:1020C00000F01AFFFFE79DF8160040F0800040F294
:1020D0003B61C2F2000108700122009200230193CB
:1020E000184601F071F8009B019804999DF80F20A3
:1020F00001F008F8FFE706B080BD000080B586B0AB
:102100008DF816008DF81510012001F09DF89DF84E
:1021100016000146049120B1FFE70498012805D07C
:1021200009E00120002100F0E7FE04E00220002188
:1021300000F0E2FEFFE79DF8150040F0800040F25D
:102140003B61C2F200010191087001220023029359
:10215000184601F039F80199029B0222184600F056
:10216000D1FF9DF816000146039120B1FFE70398C7
:1021700001280CD017E00121084600F0BDFE40F216
:102180003B60C2F2000040788DF817000BE002209F
:10219000012100F0B1FE40F23B60C2F20000007885
:1021A0008DF81700FFE79DF8170006B080BD00000E
:1021B00080B584B08DF80F008DF80E108DF80D20CD
:1021C0009DF80E0000F07F0040F23B61C2F200017A
:1021D00008709DF80D004870012001F035F89DF859
:1021E0000F000146029120B1FFE70298012805D0B7
:1021F00009E00120002100F07FFE04E00220002120
:1022000000F07AFEFFE740F23B61C2F200010222D9
:102210000023184600F0D8FF9DF80F0001460191F9
:1022200020B1FFE70198012805D009E00121084607
:1022300000F062FE04E00220012100F05DFEFFE7F5
:1022400004B080BD80B586B08DF8160004918DF87D
:102250000F209DF80F0020B9FFE70A208DF80F002E
:10226000FFE741F6C810C2F20000006864210EF0DA
:1022700047F820B1FFE7FB208DF8170070E041F62A
:10228000C410C2F2000000680290FFE70298E0B1BB
:10229000FFE7029800789DF81610884211D1FFE7F9
:1022A00002984068049988420BD1FFE741F6C810B4
:1022B000C2F2000000680EF007F9FF208DF8170049
:1022C0004EE0029800690290E0E7142000F03CFE26
:1022D0000190019858B9FFE741F6C810C2F200001A
:1022E00000680EF0F1F8FE208DF8170038E09DF838
:1022F0000F001C2100220DF001FF01998860019858
:10230000806870B9FFE7019800F02CFD41F6C81015
:10231000C2F2000000680EF0D7F8FF208DF8170019
:102320001EE09DF816000199087004980199486014
:102330009DF80F000199087341F6C411C2F2000123
:102340000868019A10610198086041F6C810C2F24D
:10235000000000680EF0B8F800208DF81700FFE7C5
:102360009DF9170006B080BD82B001908DF8031072
:10237000019802B07047000084B08DF80B00019105
:1023800041F6C410C2F2000000680090FFE7009818
:10239000A8B1FFE7009800789DF80B1088420AD199
:1023A000FFE7009840680199884204D1FFE7009850
:1023B0008068039006E0009800690090E7E700203D
:1023C0000390FFE7039804B07047000082B00090CC
:1023D0000098C068022809D1FFE7009881680220B0
:1023E000042908BF03208DF8070008E000988068E2
:1023F0000438B0FA80F040098DF80700FFE79DF837
:10240000070002B07047000083B08DF807009DF808
:102410000700022803DBFFE70020029018E09DF888
:1024200007000146009120B1FFE70098012806D07F
:102430000BE040F6EC70C2F20000029008E041F2BE
:102440001400C2F20000029002E000200290FFE7B8
:10245000029803B07047000080B586B08DF8160072
:1024600004910392029341F24040C2F200000078CE
:10247000C00720B9FFE7FD208DF8170037E003986B
:1024800020B9FFE7FE208DF8170030E041F6C810B4
:10249000C2F20000006864210DF032FF20B1FFE7B6
:1024A000FB208DF8170022E09DF816000499FFF735
:1024B00063FF019041F6C810C2F2000000680EF000
:1024C00003F8019820B9FFE7FC208DF817000EE013
:1024D00001980399029B00220DF0B0FD0090009836
:1024E000002818BF4FF0FF308DF81700FFE79DF967
:1024F000170006B080BD000080B596B041F24040A4
:10250000C2F200000078C00720B1FFE7FD208DF87F
:102510005700A7E040F2C440C2F200006821FDF776
:10252000DAFF00201490FFE71498012809DCFFE788
:102530009DF8500000F01CFBFFE714980130149048
:10254000F2E741F2F431C2F2000142F26930C0F622
:102550000000086000200DF023FF014641F6C8107E
:10256000C2F200000160006820B9FFE7FF208DF88B
:10257000570077E041F24041C2F20001079101208B
:10258000089008700AA803902821FDF7A4FF03997A
:10259000089A002009900F900A900B9010901192C9
:1025A0000C900D9012920E22029213920E9040F611
:1025B000EC70C2F20000019003F0D6FB019804F029
:1025C000BFFA099842F27972C0F60002062100F0C3
:1025D0006FF8099942F6F922C0F600020592084602
:1025E00000F066F8059A0899099800F061F8059AD4
:1025F00009980221049100F05BF80198032103F08F
:10260000DDFA029A039908980F920E9041F2140095
:10261000C2F20000069003F0A7FB069804F090FABF
:10262000089842F65D02C0F60002082100F040F86A
:10263000059A0999089800F03BF8059A0899084608
:1026400000F036F80499059A089800F031F80698D9
:10265000112103F0B3FA079A0899099811708DF8BF
:102660005700FFE79DF9570016B080BD80B584B0D4
:1026700002908DF8071041F2F430C2F200000068B9
:1026800058B1FFE741F2F430C2F20000026802984C
:102690009DF807109047039006E002989DF80710F8
:1026A000FFF762FE0390FFE7039804B080BD0000CF
:1026B00082B08DF806008DF80510009241F240407E
:1026C000C2F200000078C00720B9FFE7FD208DF8B6
:1026D00007002AE0009820B9FFE7FE208DF80700E8
:1026E00023E09DF80600022804DBFFE7FF208DF8B9
:1026F00007001AE09DF805000D2804DBFFE7FF2026
:102700008DF8070011E000989DF8061040F2C443D0
:10271000C2F20003342211FB02319DF8052041F87A
:10272000220000208DF80700FFE79DF9070002B0A6
:102730007047000080B584B08DF80E0002918DF8CE
:10274000072041F24040C2F200000078C00720B9E3
:10275000FFE7FD208DF80F0009E09DF80E000299BB
:102760009DF80720FFF76EFD8DF80F00FFE79DF93C
:102770000F0004B080BD000080B598B000200E901E
:10278000FFE70E98012867DCFFE79DF83800FFF7A8
:102790003BFE0D900D9808B9FFE759E0FFE70D9853
:1027A000002103F0D9FB002851D0FFE70D9800214C
:1027B00011AA0FAB03F0FAFB002847D1FFE71398EB
:1027C00018B9FFE71198019002E012980190FFE715
:1027D00001980C9011A8FFF7F9FD8DF82F000C98C7
:1027E0009DF82F10FFF742FF0A909DF838000A99D4
:1027F000FFF7C2FD0990099838B3FFE70020089061
:102800000790069005900490039002909DF82F0089
:102810008DF808000C9803900A98049015988DF88C
:102820001400149838B9FFE702A80D30159A0FA9C3
:10283000FDF7D2FDFFE705F09FF80890099802A97F
:1028400000231A460DF0DAFCFFE7FFE7A7E7FFE7F2
:102850000E9801300E9094E718B080BD80B598B006
:1028600000200E90FFE70E98012867DCFFE79DF837
:102870003800FFF7C9FD0D900D9808B9FFE759E042
:10288000FFE70D98012103F067FB002851D0FFE717
:102890000D98012111AA0FAB03F088FB002847D146
:1028A000FFE7139818B9FFE71198019002E012981A
:1028B0000190FFE701980C9011A8FFF787FD8DF8B4
:1028C0002F000C989DF82F10FFF7D0FE0A909DF86E
:1028D00038000A99FFF750FD0990099838B3FFE7CF
:1028E00000200890079006900590049003900290B5
:1028F0009DF82F008DF808000C9803900A9804901A
:1029000015988DF81400149838B9FFE702A80D3017
:10291000159A0FA9FDF760FDFFE705F02DF8089067
:10292000099802A900231A460DF068FCFFE7FFE7AB
:10293000A7E7FFE70E9801300E9094E718B080BD2E
:1029400080B592B0844614988DF846C08DF8451035
:1029500010920F938DF83B0041F24040C2F200000C
:102960000078C00720B9FFE7FD208DF847009EE002
:102970009DF84600022804DBFFE7FF208DF84700A2
:1029800095E00F9870B9FFE79DF84500022809D03F
:10299000FFE79DF84500032804D0FFE7FE208DF8EF
:1029A000470084E09DF83B00092804DBFFE7FF2097
:1029B0008DF847007BE09DF84600FFF725FD0D9060
:1029C0000D9820B9FFE7FE208DF847006FE000204A
:1029D00001900C900B900A90099008900790069037
:1029E00005909DF845000146029103281FD80299E1
:1029F000DFE801F002080F161098059000200790FC
:102A0000089018E010980690042007900020089085
:102A100011E01098059000200790022008900AE02D
:102A200010980690042007900220089003E0FF20F1
:102A30008DF847003BE09DF83B00099000208DF8A1
:102A400028000F9868B1FFE79DF83B00012808DBDC
:102A5000FFE705A818300F999DF83B20FDF7BCFC57
:102A6000FFE70D9803F0ACFB90B1FFE70D9805A9C7
:102A700001F1180204AB03F0CBF88DF80F009DF8BC
:102A80000F0020B9FFE700208DF847000FE0FFE7B7
:102A90009DF8460005A900F00FF920B1FFE70020DE
:102AA0008DF8470003E0FF208DF84700FFE79DF910
:102AB000470012B080BD000080B584B08DF80E00D4
:102AC0000291029820B9FFE7FE208DF80F000EE07A
:102AD0009DF80E0002990A684B1D0979EC46CCF866
:102AE00000100021FFF72CFF8DF80F00FFE79DF984
:102AF0000F0004B080BD000080B58CB000200B90AA
:102B0000FFE70B98012831DCFFE70B988DF82B00CD
:102B10009DF82B00FFF778FC0990099808B9FFE7AA
:102B200020E0FFE79DF82B0000F044F8C8B9FFE76C
:102B3000099803F045FB08B9FFE712E09DF82B0068
:102B400001A900F063F808B9FFE70AE0099801A9B4
:102B500001F118026B4603F05BF808B1FFE700E0F3
:102B6000E0E7FFE70B9801300B90CAE70CB080BD9F
:102B700081B08DF803009DF80300022801DBFFE718
:102B800015E09DF8030000EBC01042F26011C2F2A4
:102B9000000101EBC0020020C2F800049DF80320F0
:102BA00002EBC21201EBC201C1F80404FFE701B05D
:102BB0007047000081B08DF802009DF802000228E5
:102BC00004DBFFE701208DF803001AE09DF8020006
:102BD00000EBC01042F26011C2F2000101EBC00034
:102BE000D0F800049DF8022002EBC21201EBC201F2
:102BF000D1F80414401AB0FA80F040098DF80300AF
:102C0000FFE79DF8030001B070470000B0B584B045
:102C10008DF80E0002919DF80E00012803DCFFE7FD
:102C2000029820B9FFE700208DF80F0040E09DF8E2
:102C30000E0000EBC01142F26010C2F2000000EB87
:102C4000C10001900198D0F800040199D1F8041452
:102C5000884204D1FFE700208DF80F0028E0029998
:102C600000910198D0F8043400EB43125B01C05886
:102C70005368D2F808C0D2F80CE0146955694D6168
:102C80000C61C1F80CE0C1F808C04B6008609069A5
:102C9000D269CA6188610198D0F80404013000F05B
:102CA0001F000199C1F8040401208DF80F00FFE70F
:102CB0009DF80F0004B0B0BDF0B585B08DF81200DE
:102CC00003919DF81200012803DCFFE7039820B967
:102CD000FFE700208DF8130040E09DF8120000EBA4
:102CE000C01142F26010C2F2000000EBC10002907D
:102CF0000298D0F80004013000F01F000190019804
:102D00000299D1F80414884204D1FFE700208DF81D
:102D1000130023E0029ED6F8000406EB40114701A1
:102D2000039A0092D2F810E05469156850689368CD
:102D3000D2F80CC0F5514C61C1F810E0C1F80CC0DC
:102D40008B6048609069D269CA6188610198029974
:102D5000C1F8000401208DF81300FFE79DF813006F
:102D600005B0F0BD80B582B0019001980FF044F835
:102D700002B080BD80B582B08DF806009DF80600D7
:102D80000146009140B1FFE70098032808D0FFE713
:102D90000098042808D00BE0062004F081FE0BE028
:102DA0000A2004F07DFE07E0172004F079FE03E01E
:102DB000FF208DF8070003E000208DF80700FFE7F3
:102DC0009DF9070002B080BD80B582B08DF8060085
:102DD0009DF806000146009140B1FFE700980328E6
:102DE00008D0FFE70098042808D00BE0062004F084
:102DF00061FE0BE00A2004F05DFE07E0172004F0FE
:102E000059FE03E0FF208DF8070003E000208DF855
:102E10000700FFE79DF9070002B080BD80B582B0D2
:102E20008DF806009DF80600082804DBFFE7002067
:102E30008DF8070013E09DF8062047F6B051C0F664
:102E4000010101EBC200406831F8321004F064FD6A
:102E50000138B0FA80F040098DF80700FFE79DF8CF
:102E6000070002B080BD000083B08DF80A00019118
:102E7000019820B9FFE7FE208DF80B0038E09DF89F
:102E80000A00082804DBFFE7FF208DF80B002FE085
:102E90009DF80A1047F6B050C0F6010030F8310036
:102EA000ADF8020000208DF80100FFE79DF8010059
:102EB0000F2819DCFFE7BDF802009DF80110C8409B
:102EC000C00750B1FFE701989DF8012040F22C5156
:102ED000C2F2000141F8220006E0FFE79DF8010080
:102EE00001308DF80100E1E700208DF80B00FFE7CD
:102EF0009DF90B0003B0704780B582B08DF80600D5
:102F00008DF805109DF80600082804DBFFE7FF2078
:102F10008DF8070014E09DF8062047F6B051C0F682
:102F2000010101EBC200406831F832109DF8052024
:102F300002F0010204F008FD00208DF80700FFE711
:102F40009DF9070002B080BD80B582B00190019864
:102F50000EF0AAFC02B080BD86B08DF816008DED93
:102F6000040A9DF81600012804DBFFE7FF208DF816
:102F700017008CE09DED040AB7EE001AB4EE410A8A
:102F8000F1EE10FA04DDFFE74FF07E500490FFE70A
:102F90009DED040AB5EE400AF1EE10FA03DAFFE700
:102FA00000200490FFE79DF8161047F6F050C0F699
:102FB000010050F831100968C96A03919DED040AB7
:102FC0000399013101EE101AB8EE411A20EE010A00
:102FD000BCEEC00A8DED020A9DF8161000EBC10090
:102FE000808860B9FFE702989DF8162047F6F051F7
:102FF000C0F6010151F832100968486343E09DF8BA
:10300000161047F6F050C0F6010000EBC1008088B2
:1030100004280DD1FFE702989DF8162047F6F051DD
:10302000C0F6010151F8321009688863019028E068
:103030009DF8161047F6F050C0F6010000EBC100F5
:10304000808808280DD1FFE702989DF8162047F6E2
:10305000F051C0F6010151F832100968C8630090C0
:103060000CE002989DF8162047F6F051C0F60101D9
:1030700051F83210096808640090FFE70098019049
:10308000FFE70198FFE700208DF81700FFE79DF9A3
:10309000170006B07047000080B582B08DF80600BA
:1030A0009DF80600012804DBFFE7FF208DF80700EC
:1030B00010E09DF8062047F6F050C0F6010000EB46
:1030C000C20150F83200898806F032FD00208DF8E8
:1030D0000700FFE79DF9070002B080BD82B08DF8C0
:1030E00003009DF8030030B9FFE741F27C20C2F2F3
:1030F0000000019002E000200190FFE7019802B07B
:103100007047000080B584B08DF80E000291ADF8D4
:1031100006208DF805309DF80E00012804DBFFE73E
:10312000FF208DF80F0029E09DF80E00FFF7D6FF75
:103130000090009820B9FFE7FF208DF80F001DE0F8
:103140009DF80500C00760B1FFE700980299BDF83F
:10315000062005F0A7FC002818BF01208DF80F00FD
:103160000CE000980299BDF80620142305F072FBCC
:10317000002818BF01208DF80F00FFE79DF90F0010
:1031800004B080BD82B08DF806008DF80510009265
:10319000009820B9FFE7FE208DF8070010E00098A6
:1031A0009DF8062040F27451C2F2000101EB421179
:1031B0009DF8052041F8220000208DF80700FFE768
:1031C0009DF9070002B0704780B584B08DF80E00FD
:1031D0000291ADF806208DF805309DF80E0001280B
:1031E00004DBFFE7FF208DF80F0029E09DF80E00BB
:1031F000FFF774FF0090009820B9FFE7FF208DF8DB
:103200000F001DE09DF80500C00760B1FFE70098C2
:103210000299BDF8062006F093F9002818BF012096
:103220008DF80F000CE000980299BDF806201423D9
:1032300005F058FD002818BF01208DF80F00FFE7AA
:103240009DF90F0004B080BD80B586B004900CF0ED
:103250003FFE01464FF47A70B0FBF1F00390049802
:103260000399B0FBF1F002900CF0F4FD0146481C0C
:10327000019198B1FFE70198022820D3FFE7019858
:1032800002280FD0FFE701980338022806D3FFE792
:1032900001986FF00041884215D1FFE7FF208DF8BB
:1032A000170014E0029818B1FFE70298009002E0BE
:1032B00001200090FFE700980CF086FD03E00498E1
:1032C00004F0DCF8FFE700208DF81700FFE79DF918
:1032D000170006B080BD000080B58AB00CF0F8FD84
:1032E000079010F083FB079A4FF47A710191B1FBBC
:1032F000F2F1484306904EF21800CEF20000029020
:103300000068059010F072FB019A01460298079B35
:10331000B2FBF3F2514304910068039006980499BC
:10332000884215D1FFE704984FF47A72504305990B
:1033300051434EF21402CEF2000212680132B1FB88
:10334000F2F1401A00F57A7000210991089014E01A
:1033500004984FF47A725043039951434EF2140289
:10336000CEF2000212680132B1FBF2F1401A00F510
:103370007A70002109910890FFE7089809990AB02E
:1033800080BD000083B08DF807009DF8070001465E
:10339000009120B1FFE70098012806D00BE041F230
:1033A0006430C2F20000029008E041F2AC30C2F298
:1033B0000000029002E000200290FFE7029803B0B4
:1033C0007047000080B582B00190019800680068E5
:1033D000C00600282AD5FFE7FFE7002000900198EB
:1033E00000680068009001980068406800900098AC
:1033F000FFE701980BF038FF00EBC00140F2985056
:10340000C2F2000000EB8100006A70B1FFE7019892
:103410000BF02AFF00EBC00140F29850C2F200000E
:1034200000EB8100006A8047FFE7FFE702B080BD44
:1034300082B08DF806008DF805100092009820B932
:10344000FFE7FE208DF8070020E09DF80600012828
:1034500005DCFFE79DF80500092804DBFFE7FF20F6
:103460008DF8070012E000989DF8061001EBC102EC
:1034700040F29851C2F2000101EB82019DF8052053
:1034800041F8220000208DF80700FFE79DF90700B2
:1034900002B07047FFE7FEE780B540F6EC70C2F27D
:1034A000000002F0C5FE80BD80B540F6EC70C2F2AF
:1034B000000002F0BDFE80BD80B541F21400C2F2F2
:1034C000000002F0B5FE80BD80B541F21400C2F2EA
:1034D000000002F0ADFE80BD82B00090009820B9DF
:1034E000FFE703208DF807001DE00098006846F212
:1034F0000041C4F20001884204D1FFE700208DF8AA
:10350000070010E00098006846F60001C4F20001D0
:10351000884204D1FFE701208DF8070003E0032073
:103520008DF80700FFE79DF8070002B07047000024
:1035300089B0089007910692059307980078E0B942
:10354000FFE70798807C01460491032814D804996A
:10355000DFE801F00E02060A0899012008710BE06D
:1035600008990220087107E008990220087103E019
:10357000089902200871FFE777E007980078022891
:1035800040F07280FFE7079890F82300014603910E
:10359000032814D80399DFE801F00E020A060899FF
:1035A000022008710BE008990420087107E00899CF
:1035B0000520087103E0089902200871FFE70798C9
:1035C00090F8270001460291032814D80299DFE8F9
:1035D00001F00E020A060699002008700BE0069919
:1035E0000120087007E006990220087003E00699A0
:1035F00000200870FFE7079890F825000146019128
:10360000032814D80199DFE801F00E020A06059993
:10361000002008700BE005990120087007E005996B
:103620000320087003E0059900200870FFE7079861
:1036300090F8260001460091032814D80099DFE88D
:1036400001F00E020A060599002088700BE005992A
:103650000020887007E005990120887003E0059933
:1036600000208870FFE7FFE7FFE7002009B0704700
:1036700082B001900091019900200860019A022116
:1036800011710099087002B07047000080B584B0D5
:10369000039002910192029800780146009148B18E
:1036A000FFE70098013802281BD3FFE700980328A2
:1036B00028D02CE00298807C20B1FFE70298407C63
:1036C00040B9FFE70398019900F024F8039900201E
:1036D000086005E002980399019A00F025F8FFE7D9
:1036E00015E0029890F8260028B9FFE703980199A1
:1036F00000F010F805E002980399019A00F014F820
:10370000FFE704E00398019900F004F8FFE704B034
:1037100080BD000082B001900091019900200871E5
:103720000099087002B0704783B002900191009236
:1037300002980078D0B9FFE70298D0F80900019903
:1037400088600298D0F80D000199C8600298D0F8FE
:103750000100019908610298D0F809000099C86039
:103760000298D0F80D0000998860FFE70298007871
:10377000022828D1FFE70298D0F81B000199886041
:103780000298D0F81F000199C8600298D0F8130081
:10379000019908610298D0F8130001998861029894
:1037A000D0F817000199C8610298D0F81B0080F08A
:1037B00000400099C8600298D0F81F0080F00040D7
:1037C00000998860FFE703B0704700000000000028
:1037D00080B588B08DED070ACDED060A05909DED08
:1037E000050AB8EE400A10EE100A14F041F841EC58
:1037F000100B9FED2B1B53EC112B51EC100B13F006
:1038000095FC41EC100B51EC100B13F00BF900EE92
:10381000100A12F0C9F99FED261A20EE010A10EEE7
:10382000100A14F025F841EC100B51EC100B9FED31
:103830001E0B52EC103BD20F62F3DF7141EC100B08
:103840008DED020B079814F013F89DED021B41EC6F
:10385000100B51EC110B53EC102B13F015F941EC3C
:10386000100B51EC100B13F0DDF804909DED040AE1
:103870009FED101AB4EE410AF1EE10FA05DDFFE7F4
:103880009DED060A8DED010A04E09DED040A8DED23
:10389000010AFFE79DED010A08B080BD00BF00BF2F
:1038A000FCA9F1D24D62503F000000000000000072
:1038B000CDCC4C3ECDCC4C3F80B58CB00A9009911C
:1038C00008920A9818B1FFE7099820B9FFE7FE208F
:1038D0008DF82F004BE108990A980268891A00EECA
:1038E000101AB8EE400A9FEDA41A80EE010A80ED8E
:1038F000010A08980A9908600A9809990979089AAA
:1039000000F042F920B1FFE7FD208DF82F002EE1F5
:103910000A98007A0146029105286BD80299DFE8DF
:1039200001F0030B03034E2E0A990020C8600A9988
:1039300008610A99486161E0099890ED020A90EDEA
:10394000051A20EE010A0A9880ED030A099890ED05
:10395000030A90ED051A20EE010A0A9880ED040A88
:10396000099890ED040A90ED051A20EE010A0A98D4
:1039700080ED050A099840690A9988613EE0099836
:10398000C0690A99C860099880690A9908610A980B
:1039900000F2146090ED000A8DED010A08989FED89
:1039A000780ADFED780AFFF713FFB0EE401A9DEDBD
:1039B000010A20EE010A0A9880ED050A1EE0099826
:1039C000C0690A99C860099880690A9908610A99CA
:1039D00001F57470D1ED011AD1ED3F0AB0EE000A85
:1039E0009FED661A08F096FBB1EE400A0A9880ED4A
:1039F000050A03E0FD208DF82F00B8E00A9901F2D6
:103A0000844091ED030A06F0F3FE0A9880ED030A64
:103A10000A9901F2A44091ED040A06F0E9FE0A9821
:103A200080ED040A0A9901F2C44091ED050A06F0FE
:103A3000DFFE0A9880ED050A0A98099900F044F91A
:103A400000200790FFE70798032800F38C80FFE72A
:103A50000A98079900EB8101C86CC8650A99079A12
:103A6000C2EB021001EB800000F5807001EB8202D6
:103A700092ED170AD2ED330AD1ED011A9FED3F1AEC
:103A80008DED001A08F046FB9DED001A079803AB78
:103A900003EB800080ED000A0A99079AC2EB02103E
:103AA00001EB800000F5F87003EB820393ED000A50
:103AB00001EB8202D2ED2F0AD1ED011A08F02AFBA8
:103AC0000A98079900EB810080ED1F0A0A99079A6E
:103AD00001EB421000F2645001EB820191ED1F0AEC
:103AE00006F086FE9DED001A0A98079900EB81000A
:103AF00000F2046080ED000A0A98079900EB81014A
:103B0000C86AC8660A99079AC2EB021001EB8000E6
:103B100000F5387001EB820292ED1B0AD2ED270A04
:103B2000D1ED011A08F0F6FA0A98079900EB810026
:103B300080ED230A0A99079A01EB421000F2E44053
:103B400001EB820191ED230A06F052FE0A980799D3
:103B500000EB810000F2F45080ED000AFFE70798C7
:103B6000013007906FE700208DF82F00FFE79DF9E7
:103B70002F000CB080BD00BF00007A4400000000A0
:103B80009A99193FCDCC4C3F80B586B004908DF802
:103B90000F100292049820B9FFE7FE208DF817005D
:103BA0004FE09DF80F000499097A884204D1FFE79D
:103BB00000208DF8170044E09DF80F0005280ED175
:103BC000FFE70498007A052809D0FFE70298FCF780
:103BD000E5FB04994FF07E50C1F81406FFE7002082
:103BE0000190FFE70198032823DCFFE7049801997F
:103BF000C1EB011100EB810000F5387008F0CEFC3C
:103C000004980199C1EB011100EB810000F5F870F7
:103C100008F0C4FC04980199C1EB011100EB81008C
:103C200000F5807008F0BAFCFFE7019801300190C0
:103C3000D8E79DF80F000499087200208DF817004E
:103C4000FFE79DF9170006B080BD000080B582B087
:103C5000019000200090FFE70098032823DCFFE795
:103C60000199D1F86004009A00EBC200803001EBAA
:103C7000820101F2F45191ED000A07F01BFD019958
:103C8000D1F86004009A00EBC200A03001EB820181
:103C900001F2046191ED000A07F00CFDFFE70098C6
:103CA00001300090D8E70198D0F86004803007F028
:103CB000C7FA0198D0F86004A03007F0C1FA02B04A
:103CC00080BD00000000000080B5ADF53E7DBD90D8
:103CD000BC91BD98007A01287ED1FFE7BD98C068ED
:103CE00013F0C6FD41EC100B9FED551B50EC111B62
:103CF000C20F51EC100B62F3DF7141EC100B51EC71
:103D0000100B9FED510B53EC102B13F0F1FD00281D
:103D100062D1FFE7BD98006913F0AAFD41EC100BDA
:103D20009FED471B50EC111BC20F51EC100B62F3BF
:103D3000DF7141EC100B51EC100B9FED430B53EC7A
:103D4000102B13F0D5FD002846D1FFE7BD98406940
:103D500013F08EFD41EC100B9FED391B50EC111B45
:103D6000C20F51EC100B62F3DF7141EC100B51EC00
:103D7000100B9FED350B53EC102B13F0B9FD58BB16
:103D8000FFE7BD9890F80C0428B9FFE7BD99012022
:103D900081F80C04FFE700208DF8EF02FFE79DF8A3
:103DA000EF02032816DCFFE7BD989DF8EF1200EB49
:103DB0008101D1F8E405C863BD989DF8EF1200EBCE
:103DC00081010020C861FFE79DF8EF0201308DF806
:103DD000EF02E4E700F0CCBDBD99002081F80C04AF
:103DE0008DF8EE02FFE79DF8EE0203280FDCFFE7F7
:103DF000BD989DF8EE1200EB8101C86BC1F8E40597
:103E0000FFE79DF8EE0201308DF8EE02EBE7BD987A
:103E1000007A0146B491002800F08D85FFE7B49840
:103E2000012819D0FFE7B49802380228C0F0838532
:103E3000FFE7B4980438012800F299850CE000BF30
:103E400000000000000000009A9999999999B93FE3
:103E5000000000000000F03FBD980090C06813F023
:103E600007FD0246009801920A46019942EC101B98
:103E70008DED040B406913F0FBFC41EC100B8DED54
:103E8000020B1FED0D0B8DEDAA0B10F0A5FA11F032
:103E900027FE9DED021B51EC110B53EC102B13F080
:103EA00045F99DED040B41EC110B53EC112B51EC3A
:103EB000100B12F0E9FD41EC100B8DED0C0BBD99D0
:103EC000C8684969069113F0D3FC02460698079228
:103ED0000A46079942EC101B8DED0A0B13F0C8FC43
:103EE0009DEDAA0B41EC110B8DED081B10F074FA3F
:103EF00011F0F6FD9DED081B51EC110B53EC102B4E
:103F000013F014F99DED0A0B41EC110B53EC112B3E
:103F100051EC100B12F0B8FD9DED0C1B41EC100B99
:103F200051EC110B53EC102B13F000F941EC100B7A
:103F30008DED1C0BBD99086949690E9113F098FC31
:103F400002460E980F920A460F9942EC101B8DED17
:103F5000120B13F08DFC9DEDAA0B41EC110B8DEDB6
:103F6000101B10F039FA10F0FBFD9DED101B51EC09
:103F7000110B53EC102B13F0D9F89DED120B41EC03
:103F8000110B53EC112B51EC100B12F07DFD41EC99
:103F9000100B8DED1A0BBD9908694969149113F046
:103FA00067FC0246149815920A46159942EC101BBC
:103FB0008DED180B13F05CFC9DEDAA0B41EC110B81
:103FC0008DED161B10F008FA10F0CAFD9DED161BC2
:103FD00051EC110B53EC102B13F0A8F89DED180BBE
:103FE00041EC110B53EC112B51EC100B12F04CFD6A
:103FF0009DED1A1B41EC100B51EC110B53EC102BE7
:1040000013F094F89DED1C1B41EC100B51EC110BBF
:1040100053EC102B12F038FD41EC100B11F08CFE1C
:1040200051EC100B12F0FEFCBD99C861BD99C86837
:1040300049691E9113F01CFC02461E981F920A4605
:104040001F9942EC101B8DED220B13F011FC9DED1E
:10405000AA0B41EC110B8DED201B10F0BDF911F0F6
:104060003FFD9DED201B51EC110B53EC102B13F079
:104070005DF89DED220B41EC110B53EC112B51EC33
:10408000100B12F001FD41EC100B8DED2A0BBD99C8
:10409000C8684969249113F0EBFB024624982592E5
:1040A0000A46259942EC101B8DED280B13F0E0FB1E
:1040B0009DEDAA0B41EC110B8DED261B10F08CF938
:1040C00011F00EFD9DED261B51EC110B53EC102B46
:1040D00013F02CF89DED280B41EC110B53EC112B38
:1040E00051EC100B12F0D0FC9DED2A1B41EC100B93
:1040F00051EC110B53EC102B13F018F841EC100B92
:104100008DED3A0BBD99086949692C9113F0B0FB0C
:1041100002462C982D920A462D9942EC101B8DEDEB
:10412000300B13F0A5FB9DEDAA0B41EC110B8DEDAF
:104130002E1B10F051F910F013FD9DED2E1B51ECCC
:10414000110B53EC102B12F0F1FF9DED300B41ECF5
:10415000110B53EC112B51EC100B13F09BFA41ECAB
:10416000100B8DED380BBD9908694969329113F038
:104170007FFB0246329833920A46339942EC101B79
:104180008DED360B13F074FB9DEDAA0B41EC110B7A
:104190008DED341B10F020F910F0E2FC9DED341B86
:1041A00051EC110B53EC102B12F0C0FF9DED360BB0
:1041B00041EC110B53EC112B51EC100B13F06AFA7C
:1041C0009DED381B41EC100B51EC110B53EC102BF7
:1041D00012F0ACFF9DED3A1B41EC100B51EC110BB2
:1041E00053EC102B12F050FC41EC100B11F0A4FD1D
:1041F00051EC100B12F016FCBD990862BD99C8680D
:1042000049693C9113F034FB02463C983D920A46C2
:104210003D9942EC101B8DED400B13F029FB9DEDF9
:10422000AA0B41EC110B8DED3E1B10F0D5F811F0EF
:1042300057FC9DED3E1B51EC110B53EC102B12F073
:1042400075FF9DED400B41EC110B53EC112B51EC24
:10425000100B13F01FFA41EC100B8DED480BBD99BC
:10426000C8684969429113F003FB024642984392A1
:104270000A46439942EC101B8DED460B13F0F8FAF9
:104280009DEDAA0B41EC110B8DED441B10F0A4F831
:1042900011F026FC9DED441B51EC110B53EC102B3F
:1042A00012F044FF9DED460B41EC110B53EC112B2A
:1042B00051EC100B13F0EEF99DED481B41EC100B87
:1042C00051EC110B53EC102B12F030FF41EC100BA2
:1042D0008DED580BBD99086949694A9113F0C8FAE8
:1042E00002464A984B920A464B9942EC101B8DEDC0
:1042F0004E0B13F0BDFA9DEDAA0B41EC110B8DEDA9
:104300004C1B10F069F810F02BFC9DED4C1B51EC90
:10431000110B53EC102B12F009FF9DED4E0B41ECED
:10432000110B53EC112B51EC100B13F0B3F941ECC2
:10433000100B8DED560BBD9908694969509113F02A
:1043400097FA0246509851920A46519942EC101B36
:104350008DED540B13F08CFA9DEDAA0B41EC110B73
:104360008DED521B10F038F810F0FAFB9DED521B4A
:1043700051EC110B53EC102B12F0D8FE9DED540BA9
:1043800041EC110B53EC112B51EC100B13F082F993
:104390009DED561B41EC100B51EC110B53EC102B07
:1043A00012F0C4FE9DED581B41EC100B51EC110BAB
:1043B00053EC102B12F068FB41EC100B11F0BCFC1D
:1043C00051EC100B12F02EFBBD994862BD99C868E4
:1043D00049695A9113F04CFA02465A985B920A4680
:1043E0005B9942EC101B8DED5E0B13F041FA9DEDD5
:1043F000AA0B41EC110B8DED5C1B0FF0EDFF11F0E2
:104400006FFB9DED5C1B51EC110B53EC102B12F06C
:104410008DFE9DED5E0B41EC110B53EC112B51EC1D
:10442000100B13F037F941EC100B8DED660BBD99B5
:10443000C8684969609113F01BFA0246609861925E
:104440000A46619942EC101B8DED640B13F010FAD3
:104450009DEDAA0B41EC110B8DED621B0FF0BCFF23
:1044600011F03EFB9DED621B51EC110B53EC102B38
:1044700012F05CFE9DED640B41EC110B53EC112B23
:1044800051EC100B13F006F99DED661B41EC100B7F
:1044900051EC110B53EC102B12F048FE41EC100BB9
:1044A0008DED760BBD9908694969689113F0E0F9C3
:1044B0000246689869920A46699942EC101B8DED94
:1044C0006C0B13F0D5F99DEDAA0B41EC110B8DEDA2
:1044D0006A1B0FF081FF10F043FB9DED6A1B51EC4E
:1044E000110B53EC102B12F021FE9DED6C0B41ECE7
:1044F000110B53EC112B51EC100B12F0C5FA41ECDF
:10450000100B8DED740BBD99086949696E9113F01C
:10451000AFF902466E986F920A466F9942EC101BF3
:104520008DED720B13F0A4F99DEDAA0B41EC110B6C
:104530008DED701B0FF050FF10F012FB9DED701B06
:1045400051EC110B53EC102B12F0F0FD9DED720BA2
:1045500041EC110B53EC112B51EC100B12F094FAAF
:104560009DED741B41EC100B51EC110B53EC102B17
:1045700012F0DCFD9DED761B41EC100B51EC110BA4
:1045800053EC102B12F080FA41EC100B11F0D4FB1D
:1045900051EC100B12F046FABD998862BD9908697A
:1045A0004969789113F064F90246789879920A463D
:1045B000799942EC101B8DED7C0B13F059F99DEDB0
:1045C000AA0B41EC110B8DED7A1B0FF005FF10F0DB
:1045D000C7FA9DED7A1B51EC110B53EC102B12F026
:1045E000A5FD9DED7C0B41EC110B53EC112B51EC17
:1045F000100B12F049FA41EC100B8DED840BBD99B4
:10460000C86849697E9113F033F902467E987F921B
:104610000A467F9942EC101B8DED820B13F028F9AE
:104620009DEDAA0B41EC110B8DED801B0FF0D4FE1C
:1046300011F056FA9DED801B51EC110B53EC102B31
:1046400012F074FD9DED820B41EC110B53EC112B1C
:1046500051EC100B12F018FA9DED840B41EC110B8C
:1046600010F026F851EC100B9FEDED0B53EC102BD6
:10467000B393B29212F05AFD41EC100B51EC100BB7
:1046800012F0D0F9BD99C863BD990869496986914E
:1046900013F0EEF80246869887920A46879942EC14
:1046A000101B8DED8A0B13F0E3F89DEDAA0B41EC86
:1046B000110B8DED881B0FF08FFE10F051FA9DED60
:1046C000881B51EC110B53EC102B12F02FFD9DEDBC
:1046D0008A0B41EC110B53EC112B51EC100B12F027
:1046E000D9FF41EC100B8DED920BBD99C86849695B
:1046F0008C9113F0BDF802468C988D920A468D99E4
:1047000042EC101B8DED900B13F0B2F89DEDAA0B4F
:1047100041EC110B8DED8E1B0FF05EFE11F0E0F9F8
:104720009DED8E1B51EC110B53EC102B12F0FEFC87
:104730009DED900B41EC110B53EC112B51EC100B38
:1047400012F0A2F99DED920B41EC110B0FF0B0FFAE
:10475000B29AB39B51EC100B12F0E8FC41EC100B39
:1047600051EC100B12F05EF9BD990864BD9908690F
:104770004969949113F07CF80246949895920A4600
:10478000959942EC101B8DED980B13F071F89DED8F
:10479000AA0B41EC110B8DED961B0FF01DFE10F0D6
:1047A000DFF99DED961B51EC110B53EC102B12F021
:1047B000BDFC9DED980B41EC110B53EC112B51EC12
:1047C000100B12F067FF41EC100B8DEDA00BBD99A3
:1047D000C86849699A9113F04BF802469A989B92DF
:1047E0000A469B9942EC101B8DED9E0B13F040F88E
:1047F0009DEDAA0B41EC110B8DED9C1B0FF0ECFD18
:1048000011F06EF99DED9C1B51EC110B53EC102B2C
:1048100012F08CFC9DED9E0B41EC110B53EC112B17
:1048200051EC100B12F036FF9DEDA00B41EC110B7B
:104830000FF03EFFB29AB39B51EC100B12F076FCD6
:1048400041EC100B51EC100B12F0ECF8BD994864E0
:10485000BD9908694969A29113F00AF80246A29825
:10486000A3920A46A39942EC101B8DEDA60B12F001
:10487000FFFF9DEDAA0B41EC110B8DEDA41B0FF07A
:10488000ABFD10F06DF99DEDA41B51EC110B53EC39
:10489000102B12F04BFC9DEDA60B41EC110B53ECD1
:1048A000112B51EC100B12F0EFF841EC100B8DEDC9
:1048B000B00BBD99C8684969A89112F0D9FF0246AA
:1048C000A898A9920A46A99942EC101B8DEDAE0B4F
:1048D00012F0CEFF9DEDAA0B41EC110B8DEDAC1B40
:1048E0000FF07AFD11F0FCF89DEDAC1B51EC110BB3
:1048F00053EC102B12F01AFC9DEDAE0B41EC110B9A
:1049000053EC112B51EC100B12F0C4FE9DEDB00BCB
:1049100041EC110B0FF0CCFEB29AB39B51EC100B93
:1049200012F004FC41EC100B51EC100B12F07AF871
:10493000BD9988641BE00020BA90FFE7BA9803286D
:104940000BDCFFE7BD98BA9900EB81010020C8613C
:10495000FFE7BA980130BA90F0E7BD990020C8632C
:10496000BD990864BD994864BD998864FFE7FFE775
:1049700000208DF8E702FFE79DF8E702032822DC1C
:10498000FFE7BD989DF8E71200EB810090ED0F0A5C
:10499000B5EE400AF1EE10FA0EDAFFE7BD989DF889
:1049A000E71200EB810090ED0F0A9FED871A30EEC1
:1049B000010A80ED0F0AFFE7FFE79DF8E7020130EB
:1049C0008DF8E702D8E700208DF8E602FFE79DF8B2
:1049D000E602032800F3EC80FFE7BD989DF8E6129D
:1049E00000EB810090ED0F0A90ED331A30EE410A92
:1049F000B5A800EB810080ED000AFFE79DF8E61204
:104A0000B5A800EB810090ED000A9FED6B1AB4EEA3
:104A1000410AF1EE10FA15DD06E000BF00BF00BF4D
:104A200000000000DCA54C409DF8E612B5A800EBA4
:104A3000810090ED000A9FED651A30EE010A80EDCD
:104A4000000ADBE7FFE79DF8E612B5A800EB81005E
:104A500090ED000A9FED591AB4EE410AF1EE10FAFA
:104A60000EDAFFE79DF8E612B5A800EB810090EDA5
:104A7000000A9FED551A30EE010A80ED000AE2E7C8
:104A80009DF8E612B5A800EB810090ED000A9FEDBD
:104A90004C1AB4EE410AF1EE10FA2BDDFFE79DF857
:104AA000E612B5A800EB810090ED000A9FED421AD6
:104AB000B4EE410AF1EE10FA1CDCFFE7BD989DF858
:104AC000E61200EB8101C869C862BD989DF8E62234
:104AD00000EB820090ED330AB5A901EB820191ED64
:104AE000001A30EE010A9FED351A30EE010A80ED12
:104AF000130A56E09DF8E612B5A800EB810090ED90
:104B0000000A9FED301AB4EE410AF1EE10FA2BDAEA
:104B1000FFE79DF8E612B5A800EB810090ED000AD2
:104B20009FED261AB4EE410AF1EE10FA1CDBFFE706
:104B3000BD989DF8E61200EB8101C869C862BD9876
:104B40009DF8E62200EB820090ED330AB5A901EB57
:104B5000820191ED001A30EE010A9FED171A30EE36
:104B6000010A80ED130A1BE0BD989DF8E61200EBE8
:104B7000810090ED070AB1EE400A80ED0B0ABD9866
:104B80009DF8E62200EB820090ED330AB5A901EB17
:104B9000820191ED001A30EE010A80ED130AFFE761
:104BA000FFE7FFE79DF8E60201308DF8E6020EE729
:104BB0000DF53E7D80BD00BF00003443000034C3CE
:104BC0000000B4420000B4C20000B4430000B4C30B
:104BD00080B584B00290029820B9FFE7FE208DF8DE
:104BE0000F0091E006F076FE00200190FFE70198AB
:104BF000032800F38580FFE70298D0F8600401994C
:104C000000EBC100A03006F055FC183006F0A8FA01
:104C10009FED411A80EE010A9FED401A20EE010A35
:104C20000298019900EB810080ED330A0298D0F8D8
:104C30006004019900EBC100A03006F03BFC183085
:104C400006F0A0FA9FED361A80EE010A029801994B
:104C500000EB810080ED2F0A0298D0F860040199E2
:104C600000EBC100803006F025FC183006F08AFA0F
:104C70009FED2C1A80EE010A0298019900EB810049
:104C800080ED270A0298019900EB810090ED330A2C
:104C900000F58A6090ED001A30EE410A10EE100A1D
:104CA00012F0E6FD41EC100B9FED191B10F064F8BB
:104CB00051EC100B11F0B6FE0299019A01EB820142
:104CC000C1F8CC000298019900EB810090ED330A05
:104CD000B5EE400AF1EE10FA0DDAFFE702980199FD
:104CE00000EB810090ED330A9FED0F1A30EE010AC0
:104CF00080ED330AFFE7FFE701980130019076E786
:104D000000208DF80F00FFE79DF90F0004B080BD73
:104D10000000000000807640DB0F49400000344373
:104D20000000A04300401C460000B44384B0039040
:104D30008DED020ACDED010A039890ED000A9DED7C
:104D4000021A30EE010A8DED000A9DED010AB5EE62
:104D5000400AF1EE10FA26DDFFE79DED000A9DED19
:104D6000011AB4EE410AF1EE10FA09DBFFE79DEDFE
:104D7000011A9DED000A30EE410A8DED000A11E0A6
:104D80009DED000AB5EE400AF1EE10FA09DAFFE7F0
:104D90009DED011A9DED000A30EE010A8DED000A2D
:104DA000FFE7FFE7FFE700980399086004B070474A
:104DB00085B08DED040ACDED030A8DED021A9DED4F
:104DC000040A9DED031A30EE410A8DED010A9DEDB6
:104DD000020AB5EE400AF1EE10FA32DDFFE79DED72
:104DE000020AB0EE001A80EE010A8DED000A9DED78
:104DF000010A9DED001AB4EE410AF1EE10FA09DD48
:104E0000FFE79DED021A9DED010A30EE410A8DED9E
:104E1000010A15E09DED010A9DED001AB1EE411A5F
:104E2000B4EE410AF1EE10FA09DAFFE79DED021A3D
:104E30009DED010A30EE010A8DED010AFFE7FFE763
:104E4000FFE79DED010A05B07047000040F2140035
:104E5000C2F200007047000080B541F25C10C2F25F
:104E6000000002F061F880BD80B541F2BC10C2F2D2
:104E7000000002F059F880BD80B541F23C00C2F25A
:104E8000000002F051F880BD80B541F29C00C2F2F2
:104E9000000002F049F880BD80B541F2FC00C2F28A
:104EA000000002F041F880BD80B541F21C20C2F242
:104EB000000002F039F880BD82B0019001980078BE
:104EC00010384AF6AB21CAF6AA21A0FB011000094E
:104ED0000090009947F6A850C0F60100405C019987
:104EE000C8650098042807D3FFE7019908680422E1
:104EF00062F30900886506E00199086840F2FF3214
:104F000090438865FFE70198806D02B0704700000C
:104F100086B0059000208DF813000598806A0390F4
:104F20000598806910BBFFE70398029003281BD8FF
:104F30000299DFE801F0020D0218059890F82F00A1
:104F4000C00720B1FFE701208DF81300FFE70CE058
:104F50000598C06AB0F1C07F04D1FFE701208DF849
:104F60001300FFE701E000E0FFE745E005988069F6
:104F7000B0F5005F25D1FFE70398019003281ED804
:104F80000199DFE801F00206021101208DF81300FB
:104F900016E0059890F82F00C00720B1FFE7012028
:104FA0008DF81300FFE70BE00598C06AB0F1C07FF1
:104FB00004D1FFE701208DF81300FFE700E0FFE7D1
:104FC00019E003980090032804D3FFE70098032812
:104FD00004D00EE001208DF813000BE0059890F846
:104FE0002F00C00720B1FFE701208DF81300FFE775
:104FF00000E0FFE7FFE7FFE79DF8130006B070470A
:1050000084B00390029101920093039801680868AC
:1050100020F480200860009803990968486003988C
:105020008068402809D1FFE70198039909688860E2
:10503000029803990968C86008E002980399096812
:105040008860019803990968C860FFE704B0704759
:1050500083B001900091019820B9FFE7FE208DF800
:105060000B0018E0009820B9FFE7FE208DF80B0038
:1050700011E000990320087000990020A1F81100A8
:10508000C1F80D00C1F80900C1F80500C1F8010020
:105090008DF80B00FFE79DF90B0003B0704700008F
:1050A0007047000085B003900291039820B9FFE794
:1050B000FE208DF8130020E0029820B9FFE7FE20C3
:1050C0008DF8130019E002990320087002990091ED
:1050D00000200190C1F82F00C1F82B00C1F8270073
:1050E000C1F82300C1F81F00C1F81B00C1F8170068
:1050F000C1F813008DF81300FFE79DF9130005B008
:10510000704700000000000080B586B0059040F2B6
:105110005461C2F20001009148788A7840EA022086
:105120006FF3DF2000EE100AB8EEC00A059880ED9C
:10513000000A8878CA78C00840EA42106FF3DF207E
:1051400000EE100AB8EEC00A059880ED030AC87890
:105150000B794A79800940EA830040EA82206FF3A4
:10516000DF2000EE100AB8EEC00A059880ED010AB3
:1051700048798A79400840EAC2106FF3DF2000EED8
:10518000100AB8EEC00A059880ED020A8879CA793B
:10519000000940EA02106FF3DF20059A9083C87976
:1051A0000B7A4A7AC00940EA430040EA42206FF392
:1051B000DF20059A1082487A8A7A800840EA8210B5
:1051C0006FF3DF20059A5083887ACA7A400940EA53
:1051D000C200059A1083087B4A7B40EA02206FF3E5
:1051E000DF20059AD082487B8A7BC00840EA4210C3
:1051F0006FF3DF20059A9082887BCB7B0A7C800945
:1052000040EA830040EA82206FF3DF20059A508253
:10521000087C497C400840EAC1106FF3DF20059903
:10522000C883059890ED010ADFED6F0ACDED010A04
:105230009FED6E1A8DED021AFFEE001ACDED031AE6
:10524000B7EE002A8DED042A0AF09AFDDDED010A81
:105250009DED021ADDED031A9DED042A059880EDFF
:10526000010A059890ED000A0AF08AFDDDED010AB9
:105270009DED021ADDED031A9DED042A059880EDDF
:10528000000A059890ED020A0AF07AFDDDED010AA8
:105290009DED021ADDED031A9DED042A059880EDBF
:1052A000020A059890ED030A0AF06AFD059880ED60
:1052B000030A0598006812F0DBFA41EC100B9FED31
:1052C000461B53EC112B51EC100B12F018FBA0B93C
:1052D000FFE70598006812F0CBFA41EC100B9FED48
:1052E000401B53EC112B51EC100B12F0FAFA20B9C1
:1052F000FFE7059900200860FFE70598406812F075
:10530000B7FA41EC100B9FED341B53EC112B51EC11
:10531000100B12F0F4FAA0B9FFE70598406812F0FC
:10532000A7FA41EC100B9FED2E1B53EC112B51EC07
:10533000100B12F0D6FA20B9FFE70599002048605B
:10534000FFE70598806812F093FA41EC100B9FED8F
:10535000221B53EC112B51EC100B12F0D0FAA0B918
:10536000FFE70598806812F083FA41EC100B9FED7F
:105370001C1B53EC112B51EC100B12F0B2FA20B99C
:10538000FFE7059900208860FFE70598C06812F0E4
:105390006FFA41EC100B9FED101B53EC112B51ECED
:1053A000100B12F0ACFAA0B9FFE70598C06812F034
:1053B0005FFA41EC100B9FED0A1B53EC112B51ECE3
:1053C000100B12F08EFA20B9FFE705990020C86093
:1053D000FFE7012006B080BD7B14AE47E17A84BFB1
:1053E0007B14AE47E17A843F0080B04300E0D344B1
:1053F00080B5012002F098F880BD000080B5102033
:1054000002F092F880BD000080B5202002F08CF8F8
:1054100080BD000072B6FFE7FEE7000080B598B0DF
:1054200016901591169818B1FFE7159820B9FFE767
:10543000FF208DF85F00E2E1FDF74EFF169A08921B
:1054400013685268C01A914112F067FA0146089831
:1054500000EE101A9FEDE11A80EE010A80ED020ABB
:10546000FDF73AFF0A4616994A60086016981599A2
:10547000097800F09FFA159890ED030AB0EE081A2B
:1054800020EE010A169890ED021A20EE010A8DED29
:10549000140A1698C06890ED3B0AB5EE400AF1EE8A
:1054A00010FA72DDFFE7169890ED871A90ED920AD8
:1054B00030EE410A8DED130A9DED130A9FEDD21ACD
:1054C000B4EE410AF1EE10FA09DDFFE79DED130A93
:1054D0009FEDCE1A30EE010A8DED130AFFE79DED28
:1054E000130A9FEDCB1AB4EE410AF1EE10FA09DA75
:1054F000FFE79DED130A9FEDC71A30EE010A8DED0F
:10550000130AFFE7169890ED051A90ED630A9DEDDA
:10551000132A31EE021A9DED142A71EE020A9FED54
:10552000BD1A8DED071AFFF743FC9DED071A8DEDAF
:10553000120A169890ED052A90ED640A9DED133A33
:1055400032EE032A9DED143A72EE030AFFF730FCA7
:105550008DED110A9DED140A9DED121AB4EE410A6B
:10556000F1EE10FA03DDFFE712981490FFE79DEDCE
:10557000140A9DED111AB4EE410AF1EE10FA03DAA5
:10558000FFE711981490FFE7FFE7169814309DEDA0
:10559000140ADFEDA00AFFF7C9FB1698C06890ED6A
:1055A000380A90ED3B1AB6EE002A21EE021A30EED0
:1055B000010A8DED100A109816990862159890ED61
:1055C000020AB0EE081A20EE010A169890ED021AAF
:1055D00020EE010A8DED0F0A1698C06890ED3D0A85
:1055E000B5EE400AF1EE10FA72DDFFE7169890ED85
:1055F000891A90ED8E0A30EE410A8DED0E0A9DED6E
:105600000E0A9FED811AB4EE410AF1EE10FA09DD9F
:10561000FFE79DED0E0A9FED7D1A30EE010A8DED3C
:105620000E0AFFE79DED0E0A9FED791AB4EE410ACE
:10563000F1EE10FA09DAFFE79DED0E0A9FED751AFB
:1056400030EE010A8DED0E0AFFE7169890ED061A6E
:1056500090ED670A9DED0E2A31EE021A9DED0F2A9C
:1056600071EE020A9FED6B1A8DED061AFFF7A0FB93
:105670009DED061A8DED0D0A169890ED062A90ED17
:10568000680A9DED0E3A32EE032A9DED0F3A72EE56
:10569000030AFFF78DFB8DED0C0A9DED0F0A9DEDC2
:1056A0000D1AB4EE410AF1EE10FA03DDFFE70D9892
:1056B0000F90FFE79DED0F0A9DED0C1AB4EE410A25
:1056C000F1EE10FA03DAFFE70C980F90FFE7FFE71F
:1056D000169818309DED0F0ADFED4E0AFFF726FBF6
:1056E0001698007C0146059140B1FFE70598012816
:1056F0000FD0FFE70598022872D07CE016990020B1
:10570000C1F808021699C1F80C021699C1F80402F2
:1057100071E0169901F12400D1ED021A91ED050A0C
:10572000D1ED870A9FED3C1A8DED011A06F0F2FCCF
:105730009DED011A8DED090A169901F160009DEDAC
:10574000090AD1ED021AD1ED860A06F0E3FC16989B
:1057500080ED810A169901F19C00D1ED021A91EDBC
:10576000080AD1ED920A91ED931A06F0D3FC9DED53
:10577000011A8DED0B0A0B981699C1F808021699BB
:1057800001F58A70D1ED021A91ED060AD1ED890A70
:1057900006F0C0FC8DED0A0A0A9812F069F841EC97
:1057A000100B8DED020B1698D0F8380212F060F84D
:1057B00041EC100B0BF090F89DED021B51EC110B1E
:1057C00053EC102B11F060F941EC100B51EC100B65
:1057D00011F028F91699C1F80C020CE00024744964
:1057E00016990020C1F808021699C1F80C02169902
:1057F000C1F80402FFE700208DF85F00FFE79DF984
:105800005F0018B080BD00BFDB0F4940DB0FC9C08F
:10581000DB0F49C0DB0FC9400000000080B586B037
:10582000049003918DED020A049818B1FFE70398E4
:1058300020B9FFE7FF208DF8170082E00398049954
:10584000C8600498002101910174049A02F12400B7
:105850009DED020AD268383206F0D4FD049901F1B8
:1058600060009DED020AC96801F118020121009152
:1058700006F0C8FD049901F19C009DED020AC9687B
:1058800001F17802022106F0BDFD0199049A02F5AA
:105890008A709DED020AD268B83206F0B3FD009915
:1058A000049A02F5A8709DED020AD268983206F0BB
:1058B000A9FD049901F5D2709DED020AC968D1EDE8
:1058C000360A04F0F1FF0498C16891ED380A91EDB1
:1058D0003B1A30EE010A80ED630A0499C868D0F8DB
:1058E000E000C1F890010498C16891ED3A0A91ED89
:1058F0003D1A30EE010A80ED670A0499C868D0F8B5
:10590000E800C1F8A001FCF7F7FD0498C068083072
:1059100005F068FA0498C068103005F063FA04983E
:10592000C06805F02BFE0498C068083005F0F0F858
:105930000498C068103005F0EBF801988DF8170056
:10594000FFE79DF9170006B080BD000080B58CB060
:105950000B900B99C86891ED810A05F0ABFE002011
:105960000A9009900890079006900B99D1F80812B8
:105970000691059004900390029001900B98D0F846
:105980000C0201904CF6CD40C3F64C6005900B988C
:10599000C06805F055FC0B98C068083006A905F0F2
:1059A00051F90B98C068103001A905F04BF90CB003
:1059B00080BD000080B584B002908DF80710029879
:1059C00020B9FFE7FF208DF80F005AE09DF807008F
:1059D0000299097C884204D1FFE700208DF80F006E
:1059E0004FE002989C3006F0D9FD0298D83006F0BE
:1059F000D5FD029800F58A7006F0D0FD029800F5FA
:105A0000A87006F0CBFD0298243006F0C7FD02987E
:105A1000603006F0C3FD029800F5E2709FED1B0AAE
:105A20008DED000A04F0DEFF9DED000A029800F5FE
:105A3000F27004F0D7FF9DED000A029800F5D270D5
:105A400004F0D0FF0298C068083005F061F80298B1
:105A5000C068103005F05CF8029800F50770FAF79E
:105A60009DFF0299D1F8240288610299D1F81C02A5
:105A700048619DF807000299087400208DF80F0016
:105A8000FFE79DF90F0004B080BD00BF00000000DB
:105A900080B584B00290029820B9FFE7FE208DF80F
:105AA0000F0057E005F016FF0298C06805F090FE61
:105AB0000298C06805F0FEFC183005F051FB029812
:105AC00080ED920A0298C06805F0F4FC183005F0E9
:105AD00059FB029880ED930A0298C068083005F0DF
:105AE000B9FA0298C068083005F068F8019001988A
:105AF00078B1FFE70198083005F032FB029880ED9D
:105B00008A0A0198083005F03DFB029880ED8B0A67
:105B1000FFE70298C068103005F09CFA0298C06850
:105B2000103005F04BF80090009878B1FFE700982E
:105B3000083005F015FB029880ED8E0A00980830B9
:105B400005F020FB029880ED8F0AFFE700208DF81A
:105B50000F00FFE79DF90F0004B080BD83B00190F6
:105B60000091019820B9FFE7FF208DF80B0021E09C
:105B70000199009B18685A689B68C1F81832C1F8EF
:105B80001422C1F810020199009BD8681A695B6958
:105B9000C1F82432C1F82022C1F81C02009890ED0F
:105BA000050AB1EE400A019880ED880A00208DF8C0
:105BB0000B00FFE79DF90B0003B0704784B0029023
:105BC0000191029890F820008DF803009DF80300E1
:105BD000012805D0FFE79DF8030002280AD1FFE75E
:105BE000019A0298016848691043486100208DF8C5
:105BF0000F0008E00299486A40F4802048620120C2
:105C00008DF80F00FFE79DF80F0004B0704700000B
:105C100088B00690059104920393069890F82000AE
:105C20008DF80700069800688068009005988068E5
:105C300008B9FFE700E0FFE79DF80700012806D05C
:105C4000FFE79DF80700022840F08080FFE79DF8FD
:105C50000300400700280CD4FFE79DF8030000076D
:105C6000002806D4FFE79DF80300C006002864D58D
:105C7000FFE70098C0F3016002900299012088407C
:105C8000039908600598806868B9FFE7059801687E
:105C9000C06840EA415006990968029A01EB021176
:105CA000C1F880010EE005994A688868C96840EA31
:105CB000C200084306990968029A01EB0211C1F873
:105CC0008001FFE70598006906990968029A01EBCF
:105CD0000211C1F884010598007D01280CD1FFE76D
:105CE00006980068029900EB0111D1F8840140F494
:105CF0008070C1F88401FFE704984068069909683C
:105D0000029A01EB0211C1F88C010498006806990F
:105D10000968029A01EB0211C1F88801069800682F
:105D2000029900EB0111D1F8800140F00100C1F8A7
:105D3000800100208DF81F0011E00699486A40F4A8
:105D40000010486201208DF81F0008E00699486A9B
:105D500040F48020486201208DF81F00FFE79DF885
:105D60001F0008B07047000086B0049003910498AB
:105D700090F820008DF803009DF80300012806D05C
:105D8000FFE79DF80300022840F0B080FFE746F2ED
:105D90000040C4F2000001900199D1F8000240F0E7
:105DA0000100C1F800020199D1F8000220F47C50F2
:105DB000C1F800020398426A0199D1F8000240EA52
:105DC0000220C1F800020398406900F01F01012081
:105DD00088400290029A0199D1F81C029043C1F8C0
:105DE0001C020398C069F0B9FFE7029A0199D1F843
:105DF0000C029043C1F80C02039A9088D168526952
:105E000040EA0140019901EBC201C1F84002039A46
:105E100010889168526940EA0140019901EBC20182
:105E2000C1F84402FFE70398C06901281ED1FFE7CB
:105E3000029A0199D1F80C021043C1F80C02039A9E
:105E400090881168526940EA0140019901EBC20152
:105E5000C1F84002039A90899168526940EA014072
:105E6000019901EBC201C1F84402FFE70398806980
:105E700040B9FFE7029A0199D1F804029043C1F8B2
:105E8000040207E0029A0199D1F804021043C1F814
:105E90000402FFE70398006940B9FFE7029A0199FD
:105EA000D1F814029043C1F8140207E0029A019954
:105EB000D1F814021043C1F81402FFE70398006AF6
:105EC000012808D1FFE7029A0199D1F81C0210437A
:105ED000C1F81C02FFE70199D1F8000220F001008F
:105EE000C1F8000200208DF8170008E00499486A04
:105EF00040F48020486201208DF81700FFE79DF8EC
:105F0000170006B07047000080B582B0019001987C
:105F1000FDF7E2FA8DF803009DF80300032819D07D
:105F2000FFE79DF8030040F2C442C2F200023421B0
:105F300010FB0120006B60B1FFE79DF8030040F209
:105F4000C442C2F20002342110FB0120006B8047E2
:105F5000FFE7FFE702B080BD84B00390029100200C
:105F60000190039890F820008DF803009DF803003D
:105F7000012805D0FFE79DF80300022812D1FFE7B2
:105F8000029838B9FFE703980068C06800F0030082
:105F9000019006E003980068006900F0030001909A
:105FA000FFE7FFE7019804B07047000086B0049057
:105FB000039102920193049890F820008DF8030059
:105FC0009DF80300012806D0FFE79DF80300022892
:105FD00040F0E880FFE7039880B9FFE70498006885
:105FE000C068800748B9FFE70499486A40F4001088
:105FF000486201208DF81700DDE00FE0049800688A
:106000000069800748B9FFE70499486A40F4001026
:10601000486201208DF81700CDE0FFE70498006882
:10602000039900EB0110D0F8B00100F004000299D0
:1060300088600298806858B9FFE70498006803995F
:1060400000EB0110D0F8B001400D029908600AE0A1
:1060500004980068039900EB0110D0F8B001C00863
:1060600002994860FFE704980068039900EB01106B
:10607000D0F8B00100F002000299C86004980068EE
:10608000039900EB0110D0F8B40100F00F000828CC
:1060900004D3FFE70299082008610BE00498006828
:1060A000039900EB0110D0F8B40100F00F00029941
:1060B0000861FFE704980068039900EB0110D0F82D
:1060C000B40180B2000A02998861049800680399BB
:1060D00000EB0110D0F8B401000C0299486104985B
:1060E0000068039900EB0110D0F8B801019908701D
:1060F00004980068039900EB0110D0F8B801000A79
:106100000199487004980068039900EB0110D0F8D9
:10611000B801000C0199887004980068039900EB9D
:106120000110D0F8B801000E0199C87004980068F9
:10613000039900EB0110D0F8BC0101990871049893
:106140000068039900EB0110D0F8BC01000A019926
:10615000487104980068039900EB0110D0F8BC0165
:10616000000C0199887104980068039900EB0110F4
:10617000D0F8BC01000E0199C871039838B9FFE747
:1061800004980168C86840F02000C86006E00498E0
:106190000168086940F020000861FFE700208DF8E1
:1061A000170008E00499486A40F480204862012002
:1061B0008DF81700FFE79DF8170006B07047000044
:1061C00083B0029000200190029890F820008DF892
:1061D00003009DF80300012805D0FFE79DF80300A8
:1061E000022822D1FFE70298006880684001002859
:1061F00004D5FFE7019801300190FFE7029800689D
:1062000080680001002804D5FFE701980130019063
:10621000FFE7029800688068C000002804D5FFE707
:10622000019801300190FFE7FFE7019803B0704744
:1062300080B58AB0099000200890099800684069EC
:10624000079009980068406806900998006880687F
:10625000059009980068C068049009980068006972
:10626000039009980068806902909DF81C00C0079F
:10627000002800F09480FFE79DF81400C00758B391
:10628000FFE709980168012088609DF814008007E5
:10629000002804D5FFE7099800F0C0FC1BE09DF83A
:1062A00014004007002805D5FFE7089840F4006077
:1062B00008900FE09DF814000007002805D5FFE7BF
:1062C000089840F48050089003E0099800F07EFCA4
:1062D000FFE7FFE7FFE7FFE79DF81500C00760B3A2
:1062E000FFE7099801684FF4807088609DF81500F9
:1062F0008007002804D5FFE7099800F0DDFC1BE0CB
:106300009DF815004007002805D5FFE7089840F4E0
:10631000005008900FE09DF815000007002805D5F3
:10632000FFE7089840F48040089003E0099800F0E7
:106330009BFCFFE7FFE7FFE7FFE79DF81600C007BC
:1063400060B3FFE7099801684FF4803088609DF8DA
:1063500016008007002804D5FFE7099800F0FCFC30
:106360001BE09DF816004007002805D5FFE70898B8
:1063700040F4004008900FE09DF816000007002848
:1063800005D5FFE7089840F48030089003E00998AD
:1063900000F0BAFCFFE7FFE7FFE7FFE7FFE79DF844
:1063A0001C000007002810D5FFE79DF81000C0066C
:1063B000002809D5FFE7089840F400700890099874
:1063C00001681020C860FFE7FFE79DF81C00400748
:1063D00000280FD5FFE79DF810000007002808D51A
:1063E000FFE7099801680820C860099800F0E0FA02
:1063F000FFE7FFE79DF81C00800700280BD5FFE7AB
:1064000009980068C068800720B1FFE7099800F08C
:10641000F7FAFFE7FFE79DF81C004006002810D5BB
:10642000FFE79DF80C00C006002809D5FFE7089893
:1064300040F4806008900998016810200861FFE727
:10644000FFE79DF81C00800600280FD5FFE79DF8A8
:106450000C000007002808D5FFE70998016808200C
:106460000861099800F0F4FAFFE7FFE79DF81C00C7
:10647000C00600280BD5FFE709980068006980076F
:1064800020B1FFE7099800F00BFBFFE7FFE79DF85D
:106490001E00800700280FD5FFE79DF81800C006F2
:1064A000002808D5FFE7099801681020486009987E
:1064B00000F01EFBFFE7FFE79DF81E00C00778B164
:1064C000FFE79DF818000007002808D5FFE70998A6
:1064D000016808204860099800F066FCFFE7FFE7C4
:1064E0009DF81D000006002840F18D80FFE79DF813
:1064F00018004007002840F18180FFE79DF81D004B
:10650000C00750B1FFE79DF80800C00728B1FFE7BA
:10651000089840F001000890FFE79DF81D008007F3
:1065200000280BD5FFE79DF808008007002805D557
:10653000FFE7089840F002000890FFE79DF81D0073
:10654000400700280BD5FFE79DF80800400700280A
:1065500005D5FFE7089840F004000890FFE79DF894
:106560001D000007002848D5FFE79DF8080010F03F
:10657000700F42D0FFE7029800F0700001460191D1
:10658000102814D0FFE70198202815D0FFE70198C4
:10659000302816D0FFE70198402817D0FFE7019870
:1065A000502818D0FFE70198602819D01DE00898FE
:1065B00040F00800089019E0089840F0100008909A
:1065C00014E0089840F0200008900FE0089840F090
:1065D000400008900AE0089840F08000089005E02C
:1065E000089840F48070089000E0FFE7099801687F
:1065F000886920F070008861FFE7FFE7099801686B
:1066000004204860FFE7089848B1FFE7089A099915
:10661000486A104348620998FFF776FCFFE70AB022
:1066200080BD000080B584B00290029820B9FFE7D9
:1066300001208DF80F00E0E0029890F8200020B9CA
:10664000FFE7029800F0DEF8FFE7029801680868AB
:1066500040F00100086001F08FF90190FFE7029817
:1066600000684068C007A8B9FFE701F085F9019903
:10667000401A0B280DD3FFE70299486A40F4003016
:1066800048620299052081F8200001208DF80F0052
:10669000B3E0E4E702980168086820F002000860AF
:1066A00001F06AF90190FFE70298006840688007EE
:1066B000002815D5FFE701F05FF90199401A0B2872
:1066C0000DD3FFE70299486A40F40030486202990E
:1066D000052081F8200001208DF80F008DE0E3E710
:1066E0000298007E012807D1FFE702980168086838
:1066F00040F08000086006E002980168086820F019
:1067000080000860FFE70298407E012807D1FFE77C
:1067100002980168086840F04000086006E00298AE
:106720000168086820F040000860FFE70298807E5A
:10673000012807D1FFE702980168086840F02000AF
:10674000086006E002980168086820F020000860F0
:10675000FFE70298C07E012807D1FFE70298016891
:10676000086820F01000086006E0029801680868D8
:1067700040F010000860FFE70298007F012807D171
:10678000FFE702980168086840F00800086006E02A
:1067900002980168086820F008000860FFE7029886
:1067A000407F012807D1FFE702980168086840F0A0
:1067B0000400086006E002980168086820F0040000
:1067C0000860FFE7029B19685A689868D3F80CC004
:1067D00040EA0C00D3F810C040EA0C005B69184393
:1067E000013A1043C861029900204862029A0121CF
:1067F00082F820108DF80F00FFE79DF80F0004B01D
:1068000080BD000080B594B01390002012901190CC
:1068100010900F900E901398006846F20041C4F259
:106820000001884253D1FFE740F26C50C2F20000F1
:106830000168013101600068012812D1FFE7FFE71C
:1068400000200D9043F64000C4F20200016841F0C0
:1068500000710160006800F000700D900D98FFE776
:10686000FFE7FFE700200C9043F63000C4F202007F
:10687000016841F008010160006800F008000C9018
:106880000C98FFE703200E9002210F910021079141
:10689000109111900920129040F60040C4F20200BD
:1068A0000EA900F05DFE079A1420059005210691BF
:1068B00001F00AF9059801F0FDF80699079A1520EC
:1068C000089001F001F9089801F0F4F86EE01398CF
:1068D000006846F60001C4F20001884265D1FFE776
:1068E000FFE700200B9043F64000C4F2020001686D
:1068F00041F080610160006800F080600B900B98AF
:10690000FFE740F26C50C2F2000001680131016003
:106910000068012812D1FFE7FFE700200A9043F644
:106920004000C4F20200016841F00071016000689B
:1069300000F000700A900A98FFE7FFE7FFE70020E9
:10694000099043F63000C4F20200016841F00201F0
:106950000160006800F0020009900998FFE76020DC
:106960000E9002200F9000200390109003201190B1
:106970000920129040F20040C4F202000EA900F07B
:10698000EFFD039A402001900521029101F09CF84F
:10699000019801F08FF80299039A4120049001F0C8
:1069A00093F8049801F086F8FFE7FFE714B080BD84
:1069B00080B582B001900198FCF78EFD8DF8030040
:1069C0009DF80300032819D0FFE79DF8030040F26B
:1069D000C442C2F20002342110FB0120C06960B140
:1069E000FFE79DF8030040F2C442C2F200023421E6
:1069F00010FB0120C0698047FFE7FFE702B080BDC0
:106A000080B582B001900198FCF766FD8DF8030017
:106A10009DF80300032819D0FFE79DF8030040F21A
:106A2000C442C2F20002342110FB0120806960B12F
:106A3000FFE79DF8030040F2C442C2F20002342195
:106A400010FB012080698047FFE7FFE702B080BDAF
:106A500080B582B001900198FCF73EFD8DF80300EF
:106A60009DF80300032819D0FFE79DF8030040F2CA
:106A7000C442C2F20002342110FB0120406A60B11E
:106A8000FFE79DF8030040F2C442C2F20002342145
:106A900010FB0120406A8047FFE7FFE702B080BD9E
:106AA00080B582B001900198FCF716FD8DF80300C7
:106AB0009DF80300032819D0FFE79DF8030040F27A
:106AC000C442C2F20002342110FB0120006A60B10E
:106AD000FFE79DF8030040F2C442C2F200023421F5
:106AE00010FB0120006A8047FFE7FFE702B080BD8E
:106AF00080B582B001900198FCF7EEFC8DF80300A0
:106B00009DF80300032819D0FFE79DF8030040F229
:106B1000C442C2F20002342110FB0120806A60B13D
:106B2000FFE79DF8030040F2C442C2F200023421A4
:106B300010FB0120806A8047FFE7FFE702B080BDBD
:106B400080B584B00290029890F8200001282FD1DF
:106B5000FFE70299022081F8200002980168086886
:106B600020F00100086000F007FF0190FFE70298A5
:106B700000684068C007A8B1FFE700F0FDFE01997A
:106B8000401A0B280DD3FFE70299486A40F4003001
:106B900048620299052081F8200001208DF80F003D
:106BA0000FE0E4E70299002048628DF80F0008E04A
:106BB0000299486A40F40020486201208DF80F00D5
:106BC000FFE79DF80F0004B080BD000080B582B0E3
:106BD00001900198FCF780FC8DF803009DF80300FC
:106BE000032819D0FFE79DF8030040F2C442C2F227
:106BF0000002342110FB0120C06860B1FFE79DF85E
:106C0000030040F2C442C2F20002342110FB012012
:106C1000C0688047FFE7FFE702B080BD80B582B063
:106C200001900198FCF758FC8DF803009DF80300D3
:106C3000032817D0FFE79DF803003421414340F2B9
:106C4000C440C2F20000405858B1FFE79DF803006D
:106C50003421414340F2C440C2F200004058804712
:106C6000FFE7FFE702B080BD80B582B001900198D8
:106C7000FCF732FC8DF803009DF80300032819D0BF
:106C8000FFE79DF8030040F2C442C2F20002342143
:106C900010FB0120006960B1FFE79DF8030040F29E
:106CA000C442C2F20002342110FB01200069804777
:106CB000FFE7FFE702B080BD80B582B00190019888
:106CC000FCF70AFC8DF803009DF80300032819D097
:106CD000FFE79DF8030040F2C442C2F200023421F3
:106CE00010FB0120406860B1FFE79DF8030040F20F
:106CF000C442C2F20002342110FB012040688047E8
:106D0000FFE7FFE702B080BD80B582B00190019837
:106D1000FCF7E2FB8DF803009DF80300032819D06F
:106D2000FFE79DF8030040F2C442C2F200023421A2
:106D300010FB0120406960B1FFE79DF8030040F2BD
:106D4000C442C2F20002342110FB01204069804796
:106D5000FFE7FFE702B080BD80B582B001900198E7
:106D6000FCF7BAFB8DF803009DF80300032819D047
:106D7000FFE79DF8030040F2C442C2F20002342152
:106D800010FB0120806860B1FFE79DF8030040F22E
:106D9000C442C2F20002342110FB01208068804707
:106DA000FFE7FFE702B080BD80B582B00190019897
:106DB000FCF792FB8DF803009DF80300032819D01F
:106DC000FFE79DF8030040F2C442C2F20002342102
:106DD00010FB0120C06A60B1FFE79DF8030040F29C
:106DE000C442C2F20002342110FB0120C06A804775
:106DF000FFE7FFE702B080BD80B584B00290029843
:106E0000806D019000F0B8FD0090029890F8350078
:106E100002280DD0FFE7029980204865FFE702991C
:106E2000002081F83400FFE701208DF80F0055E0C5
:106E300002980168086820F016000860029801684E
:106E4000486920F0800048610298006C20B9FFE793
:106E50000298806C38B1FFE702980168086820F05A
:106E600008000860FFE702980168086820F0010048
:106E70000860FFE7029800680068C007C8B1FFE734
:106E800000F07AFD0099401A062811D3FFE7029915
:106E9000202048650299032081F83500FFE7029918
:106EA000002081F83400FFE703208DF80F0015E083
:106EB000E0E70298C16D3F208840019988600299FF
:106EC000012081F83500FFE70299002081F83400A5
:106ED000FFE7FFE700208DF80F00FFE79DF80F00A8
:106EE00004B080BD82B00090009890F83500022870
:106EF00007D0FFE700998020486501208DF8070042
:106F00000EE00099052081F83500009801680868B6
:106F100020F001000860FFE700208DF80700FFE780
:106F20009DF8070002B0704780B586B0059000203C
:106F3000039040F20000C2F20000006848F2B51170
:106F4000C1F64E31A0FB0110800A02900598806DB9
:106F5000019001980068049004980599C96DC84093
:106F6000000700281AD5FFE7059800680068400769
:106F7000002812D5FFE705980168086820F0040092
:106F800008600598C16D08208840019988600599BE
:106F9000486D40F001004865FFE7FFE70498059958
:106FA000C96DC840C007A0B1FFE7059800684069F7
:106FB000000600280CD5FFE70598C16D0120884028
:106FC000019988600599486D40F002004865FFE727
:106FD000FFE704980599C96DC8404007002814D5FB
:106FE000FFE7059800680068800700280CD5FFE7D8
:106FF0000598C16D04208840019988600599486D05
:1070000040F004004865FFE7FFE704980599C96D63
:10701000C840C006002847D5FFE70598006800680B
:10702000000700283FD5FFE70598C16D1020884074
:1070300001998860059800680068400300281AD507
:10704000FFE70598006800680003002809D4FFE7FF
:107050000598006C20B1FFE70598016C8847FFE7B1
:1070600008E00598806C20B1FFE70598816C88479F
:10707000FFE7FFE716E0059800680068C0050028F4
:1070800007D4FFE705980168086820F00800086049
:10709000FFE70598006C20B1FFE70598016C884771
:1070A000FFE7FFE7FFE7FFE704980599C96DC840D0
:1070B0008006002840F18D80FFE705980068006891
:1070C000C006002840F18480FFE70598C16D2020AC
:1070D000884001998860059890F83500052834D1DA
:1070E000FFE705980168086820F016000860059819
:1070F0000168486920F0800048610598006C20B95B
:10710000FFE70598806C38B1FFE7059801680868CB
:1071100020F008000860FFE70598C16D3F20884017
:10712000019988600599012081F83500FFE70599EC
:10713000002081F83400FFE70598006D20B1FFE7DB
:107140000598016D8847FFE77BE0059800680068B7
:10715000400300281AD5FFE705980068006800037F
:10716000002809D4FFE70598406C20B1FFE7059897
:10717000416C8847FFE708E00598C06B20B1FFE746
:107180000598C16B8847FFE7FFE720E00598006896
:107190000068C005002811D4FFE705980168086859
:1071A00020F0100008600599012081F83500FFE704
:1071B0000599002081F83400FFE7FFE70598C06BD0
:1071C00020B1FFE70598C16B8847FFE7FFE7FFE7BE
:1071D000FFE70598406DA0B3FFE70598406DC00735
:1071E00030B3FFE70599052081F83500059801685F
:1071F000086820F001000860FFE703980130039061
:107200000299884201D9FFE707E0FFE70598006887
:107210000068C0070028F0D1FFE70599012081F838
:107220003500FFE70599002081F83400FFE7FFE70C
:107230000598C06C20B1FFE70598C16C8847FFE74F
:10724000FFE706B080BD000080B586B00490002046
:10725000039000F091FB0290049820B9FFE7012011
:107260008DF81700A3E00498406A08B1FFE7FFE734
:107270000499022081F83500FFE70499002081F885
:107280003400FFE704980168086820F001000860F6
:10729000FFE7049800680068C00790B1FFE700F0BE
:1072A0006BFB0299401A06280AD3FFE704992020B5
:1072B00048650499032081F835008DF8170076E0C1
:1072C000E7E70498006800680390039848F23F01DC
:1072D000CFF2100108400390049900914868D1F85A
:1072E00008C0CB680A6940EA0C00184310434A6999
:1072F00010438A691043CA691043096A014303981D
:10730000084303900498406A042808D1FFE70499D1
:10731000C86A096B0143039808430390FFE7039889
:10732000049909680860049800684069039003980C
:1073300020F0070003900498416A039808430390E3
:107340000498406A04281AD1FFE70498816A0398D8
:10735000084303900498C06A80B1FFE70498FDF7E2
:10736000D7FD50B1FFE704994020486504990120FA
:1073700081F835008DF8170019E0FFE7FFE7039863
:107380000499096848610498FDF796FD01900498F6
:10739000C16D3F20884001998860049900204865AC
:1073A000049A012182F835108DF81700FFE79DF847
:1073B000170006B080BD000080B588B0069005912A
:1073C0000492039300208DF80B000698806D0190C5
:1073D000FFE7069890F83400012804D1FFE7022067
:1073E0008DF81F0045E00699012081F83400FFE781
:1073F000FFE7069890F8350001282BD1FFE70699A2
:10740000022081F835000699002048650698059904
:10741000049A039BFDF7F4FD0698C16D3F20884058
:107420000199886006980168086840F016000860B5
:107430000698006C38B1FFE706980168086840F0CC
:1074400008000860FFE706980168086840F001003E
:10745000086009E0FFE70699002081F83400FFE7A3
:1074600002208DF80B00FFE79DF80B008DF81F0040
:10747000FFE79DF81F0008B080BD000080B584B014
:10748000039000F079FA029003980190019801307E
:1074900048B1FFE740F27030C2F200000178019875
:1074A00008440190FFE7FFE700F066FA0299401AEE
:1074B0000199884201D2FFE7F6E704B080BD0000E1
:1074C00080B582B0ADF8060000208DF80500FFE71A
:1074D0009DF805000F2824DCFFE7BDF806009DF8A5
:1074E0000510C840C007A8B1FFE79DF8051040F29D
:1074F0002C50C2F2000050F8210050B1FFE79DF877
:10750000051040F22C50C2F2000050F821008047D4
:10751000FFE7FFE7FFE79DF8050001308DF8050064
:10752000D6E702B080BD000080B582B0ADF806009D
:1075300043F61440C4F201000068BDF8061008428A
:107540000CD0FFE7BDF8060043F61441C4F2010178
:107550000860BDF80600FFF7B3FFFFE702B080BD8B
:107560008EB00D900C9100200A90099008900B901D
:10757000FFE70B980F2800F2CC81FFE70B99012061
:1075800088400A900C9800680A9908400990099868
:107590000A99884240F0B881FFE70C98406800F0F3
:1075A0000300012807D0FFE70C98406800F00300B3
:1075B00002282FD1FFE70D98806808900B984100B2
:1075C000032000FA01F10898884308900C98C068DD
:1075D0000B99490000FA01F10898084308900898AF
:1075E0000D9988600D98406808900B99012000FA69
:1075F00001F10898884308900C984068C0F3001087
:107600000B9900FA01F108980843089008980D9921
:107610004860FFE70C98406800F00300032818D08A
:10762000FFE70D98C06808900B984100032000FA0E
:1076300001F10898884308900C9880680B994900DC
:1076400000FA01F108980843089008980D99C8605D
:10765000FFE70C98406800F00300022826D1FFE7FE
:107660000D980B996FF0030202EA51010844006A79
:1076700008900B9800F0070081000F2000FA01F13C
:107680000898884308900C9800690B9901F007014D
:10769000890000FA01F108980843089008980D99AC
:1076A0000B9B02EA530211440862FFE70D98006841
:1076B00008900B984100032000FA01F108988843D4
:1076C00008900C98406800F003000B99490000FAFC
:1076D00001F108980843089008980D9908600C98E3
:1076E00080798007002800F00E81FFE7FFE7002087
:1076F000079043F64400C4F20200016841F480415F
:107700000160006800F4804007900798FFE70B983D
:1077100020F0030043F60801C4F20101405808902C
:107720000B9800F0030081000F2000FA01F1089887
:10773000884308900D980021C4F20201884203D1C9
:10774000FFE7002006905EE00D9840F20041C4F291
:107750000201884203D1FFE70120059050E00D9817
:1077600040F60001C4F20201884203D1FFE7022083
:10777000049042E00D9840F60041C4F202018842B4
:1077800003D1FFE70320039034E00D9841F200019C
:10779000C4F20201884203D1FFE70420029026E0F0
:1077A0000D9841F20041C4F20201884203D1FFE783
:1077B0000520019018E00D9841F60001C4F2020185
:1077C000884203D1FFE7062000900AE00D9941F6B8
:1077D0000042C4F202020820914208BF0720009034
:1077E000FFE700980190FFE701980290FFE70298F9
:1077F0000390FFE703980490FFE704980590FFE7E4
:1078000005980690FFE70698C0B20B9901F00301B6
:10781000890000FA01F108980843089008980B992C
:1078200021F0030143F60802C4F20102885043F636
:107830000840C4F20100006808900999089888433C
:1078400008900C988079C006002805D5FFE70999B3
:10785000089808430890FFE7089843F60841C4F2E7
:107860000101086043F60C40C4F201000068089072
:1078700009990898884308900C9880798006002818
:1078800005D5FFE70999089808430890FFE708988D
:1078900043F60C41C4F20101086043F60440C4F20F
:1078A00001000068089009990898884308900C988E
:1078B00080798007002805D5FFE7099908980843D3
:1078C0000890FFE7089843F60441C4F201010860FC
:1078D00043F60040C4F20100006808900999089836
:1078E000884308900C988079C00728B1FFE7099970
:1078F000089808430890FFE7089843F60041C4F24F
:1079000001010860FFE7FFE7FFE70B9801300B90EC
:107910002FE60EB07047000082B00190ADF8021063
:1079200001980069BDF80210084204D0FFE7012069
:107930008DF8010003E000208DF80100FFE79DF8BD
:10794000010002B07047000082B00190ADF8021053
:107950008DF801209DF8010028B1FFE7BDF8020075
:107960000199886105E0BDF8020000040199886171
:10797000FFE702B07047000042F67810C2F2010043
:107980000068704740F27030C2F20000027842F6A0
:107990007811C2F2010108681044086070470000C5
:1079A00080B543F60041C4F20201086840F400705B
:1079B0000860086840F480600860086840F48070DF
:1079C0000860032000F09AF80F2000F005F800F09E
:1079D0003BF8002080BD000080B582B0009040F2EE
:1079E0000000C2F20000006840F27031C2F20001F3
:1079F0000A784FF47A71B1FBF2F1B0FBF1F001F0CB
:107A0000F7FE20B1FFE701208DF8070018E000988D
:107A10000F280DD8FFE700994FF0FF30002200F04B
:107A200053F8009840F27431C2F20001086003E09C
:107A300001208DF8070003E000208DF80700FFE724
:107A40009DF8070002B080BD80B582B0FFE700203E
:107A5000019043F64400C4F20200016841F4804101
:107A60000160006800F4804001900198FFE7FFE7A3
:107A70000020009043F64000C4F20200016841F08B
:107A800080510160006800F0805000900098FFE78E
:107A90006FF001000F21002200F016F802B080BD47
:107AA00080B582B08DF807009DF9070007F0BAFE97
:107AB00002B080BD80B582B08DF807009DF9070047
:107AC00007F0CCFE02B080BD80B586B08DF81700FF
:107AD000049103920020029007F0D8FE02909DF9D5
:107AE0001700019002980499039A04F0DDFA014608
:107AF000019807F0D3FE06B080BD000080B582B0CB
:107B00000190019807F00EFF02B080BD80B584B0EF
:107B100002900191029820B9FFE701208DF80F0033
:107B200021E1019843F60041C4F20201096801F025
:107B30000701884212D9FFE7019943F60040C4F2D9
:107B400002000170006800F007000199884204D02B
:107B5000FFE701208DF80F0005E1FFE702980078AC
:107B6000800700282AD5FFE7029800784007002800
:107B700009D5FFE743F60801C4F20201086840F4A2
:107B8000E0500860FFE7029800780007002809D558
:107B9000FFE743F60801C4F20201086840F46040C0
:107BA0000860FFE743F60801C4F20201086820F00C
:107BB000F000029A926810430860FFE7029800788C
:107BC000C00700286ED0FFE702984068012811D155
:107BD000FFE743F60000C4F20200006800F4003141
:107BE0000020B0EB514F04D1FFE701208DF80F00CA
:107BF000B9E02CE002984068022805D0FFE702981F
:107C00004068032811D1FFE743F60000C4F20200E8
:107C1000006800F000710020B0EB516F04D1FFE765
:107C200001208DF80F009EE010E043F60000C4F242
:107C30000200006800F002010020B0EB510F04D1F7
:107C4000FFE701208DF80F008DE0FFE7FFE743F627
:107C50000801C4F20201086820F00300029A526889
:107C600010430860FFF788FE0090FFE743F6080026
:107C7000C4F20200006800F00C0002994968B0EB01
:107C8000810F0ED0FFE7FFF777FE0099401A41F20F
:107C90008931884204D3FFE703208DF80F0062E0AA
:107CA000E4E7FFE7019843F60041C4F202010968E6
:107CB00001F00701884212D2FFE7019943F6004024
:107CC000C4F202000170006800F0070001998842C8
:107CD00004D0FFE701208DF80F0044E0FFE7029891
:107CE0000078400700280CD5FFE743F60801C4F2EE
:107CF0000201086820F4E050029AD268104308603C
:107D0000FFE702980078000700280DD5FFE743F64B
:107D10000801C4F20201086820F46040029A126966
:107D200040EAC2000860FFE700F04CF843F60801A3
:107D3000C4F202010968C9B20A0947F69051C0F6B7
:107D40000101895CC84040F20001C2F200010860F4
:107D500040F27430C2F200000068FFF73DFE0020E0
:107D60008DF80F00FFE79DF80F0004B080BD000004
:107D700040F20000C2F200000068704780B5FFF7D3
:107D8000F7FF43F60801C4F202010968C1F3822239
:107D900047F6A051C0F60101895CC84080BD0000D3
:107DA00080B5FFF7E5FF43F60801C4F20201096858
:107DB00089B24A0B47F6A051C0F60101895CC84060
:107DC00080BD000080B586B000200590049003902F
:107DD000029043F60800C4F20200006800F00C00B4
:107DE0000146019140B1FFE7019804280AD0FFE75E
:107DF000019808280CD04FE042F20040C0F2F40095
:107E000002904FE041F60030C0F2B700029049E026
:107E100043F60400C4F20200016801F03F0105913D
:107E200000684002002813D5FFE743F60400C4F2BF
:107E300002000068C0F3881041F60031C0F2B701BB
:107E4000A0FB0101059A0023F8F730FA049012E034
:107E500043F60400C4F202000068C0F3881042F246
:107E60000041C0F2F401A0FB0101059A0023F8F7DC
:107E70001DFA0490FFE743F60400C4F20200006814
:107E800000F44031022000EBD130039004980399B4
:107E9000B0FBF1F0029005E042F20040C0F2F400C5
:107EA0000290FFE7029806B080BD000080B586B062
:107EB0000490049820B9FFE701208DF8170050E3E3
:107EC00004980078C007002800F0A580FFE743F67B
:107ED0000800C4F20200006800F00C00042813D06F
:107EE000FFE743F60800C4F20200006800F00C004F
:107EF00008281ED1FFE743F60400C4F20200006820
:107F00004002002815D5FFE743F60000C4F2020046
:107F1000006800F400310020B0EB514F08D0FFE7BB
:107F20000498406820B9FFE701208DF8170018E396
:107F300070E0FFE704984068B0F5803F09D1FFE7A3
:107F400043F60001C4F20201086840F48030086082
:107F500020E004984068B0F5A02F0DD1FFE743F66C
:107F60000001C4F20201086840F48020086008683B
:107F700040F4803008600CE043F60001C4F20201D6
:107F8000086820F480300860086820F480200860C9
:107F9000FFE7FFE7FFE704984068E8B1FFE7FFF776
:107FA000EBFC0390FFE743F60000C4F20200006818
:107FB00000F400310020B0EB514F0CD1FFE7FFF788
:107FC000DBFC0399401A652804D3FFE703208DF8F2
:107FD0001700C6E2E7E71CE0FFF7CEFC0390FFE7DF
:107FE00043F60000C4F20200006800F400310020F3
:107FF000B0EB514F0CD0FFE7FFF7BEFC0399401ADE
:10800000652804D3FFE703208DF81700A9E2E7E70E
:10801000FFE7FFE7FFE7049800788007002840F1BA
:108020009680FFE743F60800C4F20200006810F0F3
:108030000C0F13D0FFE743F60800C4F202000068FB
:1080400000F00C0008282CD1FFE743F60400C4F22E
:10805000020000684002002823D4FFE743F6000036
:10806000C4F20200006800F002010020B0EB510FE2
:1080700009D0FFE70498C068012804D0FFE7012079
:108080008DF817006DE243F60001C4F202010868A2
:1080900020F0F800049A126940EAC2000860FFE785
:1080A00054E00498C06870B3FFE70021C4F2472190
:1080B00001200860FFF760FC0390FFE743F6000033
:1080C000C4F20200006800F002010020B0EB510F82
:1080D0000CD1FFE7FFF750FC0399401A032804D3A3
:1080E000FFE703208DF817003BE2E7E743F60001C6
:1080F000C4F20201086820F0F800049A126940EA0C
:10810000C200086021E00021C4F24721002008607D
:10811000FFF732FC0390FFE743F60000C4F20200D1
:10812000006800F002010020B0EB510F0CD0FFE717
:10813000FFF722FC0399401A032804D3FFE703202A
:108140008DF817000DE2E7E7FFE7FFE7FFE7049888
:108150000078000700284BD5FFE70498406918B362
:10816000FFE740F68061C4F2472101200860FFF775
:1081700003FC0390FFE743F67400C4F202000068BA
:1081800000F002010020B0EB510F0CD1FFE7FFF728
:10819000F3FB0399401A032804D3FFE703208DF86B
:1081A0001700DEE1E7E722E040F68061C4F24721F4
:1081B00000200860FFF7E0FB0390FFE743F6740040
:1081C000C4F20200006800F002010020B0EB510F81
:1081D0000CD0FFE7FFF7D0FB0399401A032804D324
:1081E000FFE703208DF81700BBE1E7E7FFE7FFE7B4
:1081F000049800784007002840F1CE80FFE7002077
:108200008DF8070043F64000C4F202000068C00089
:10821000002815D4FFE7FFE70020009043F6400058
:10822000C4F20200016841F080510160006800F072
:10823000805000900098FFE701208DF80700FFE7CD
:1082400047F20000C4F200000068C005002822D4F4
:10825000FFE747F20001C4F20001086840F48070B3
:108260000860FFF789FB0390FFE747F20000C4F2C4
:1082700000000068C00500280CD4FFE7FFF77CFB76
:108280000399401A032804D3FFE703208DF8170051
:1082900067E1EAE7FFE7FFE704988068012809D172
:1082A000FFE743F67001C4F20201086840F00100E4
:1082B00008601FE00498806805280DD1FFE743F6A9
:1082C0007001C4F20201086840F004000860086808
:1082D00040F0010008600CE043F67001C4F20201B6
:1082E000086820F001000860086820F004000860B9
:1082F000FFE7FFE7FFE704988068F8B1FFE7FFF7C3
:108300003BFB0390FFE743F67000C4F202000068F5
:1083100000F002010020B0EB510F0ED1FFE7FFF794
:108320002BFB0399401A41F28931884204D3FFE7BD
:1083300003208DF8170014E1E5E71EE0FFF71CFBB2
:108340000390FFE743F67000C4F20200006800F0FB
:1083500002010020B0EB510F0ED0FFE7FFF70CFB3E
:108360000399401A41F28931884204D3FFE7032080
:108370008DF81700F5E0E5E7FFE79DF80700012815
:1083800009D1FFE743F64001C4F20201086820F07A
:1083900080500860FFE7FFE704988069002800F03C
:1083A000DC80FFE743F60800C4F20200006800F03A
:1083B0000C00082800F08580FFE7049880690228F7
:1083C0005CD1FFE76021C4F2472100200860FFF77D
:1083D000D3FA0390FFE743F60000C4F202000068FE
:1083E00000F000710020B0EB516F0CD0FFE7FFF7F9
:1083F000C3FA0399401A032804D3FFE703208DF83A
:108400001700AEE0E7E70499C869D1F820C04B6ACD
:108410008A6A40EA0C0040EA8310D2034FF6FF73E9
:108420009A43A2F580321043C96A40EA016043F6DC
:108430000401C4F2020108606021C4F24721012056
:108440000860FFF799FA0390FFE743F60000C4F2D3
:108450000200006800F000710020B0EB516F0CD1F9
:10846000FFE7FFF789FA0399401A032804D3FFE7CF
:1084700003208DF8170074E0E7E721E06021C4F2E3
:10848000472100200860FFF777FA0390FFE743F6E3
:108490000000C4F20200006800F000710020B0EBA0
:1084A000516F0CD0FFE7FFF767FA0399401A0328D2
:1084B00004D3FFE703208DF8170052E0E7E7FFE75A
:1084C0004AE004988069012804D1FFE701208DF873
:1084D000170046E043F60400C4F202000068029070
:1084E00004988069012831D0FFE7029800F48000E9
:1084F0000499C969884229D1FFE7029800F03F003A
:108500000499096A884221D1FFE7029847F6C071B1
:1085100008400499496AB0EB811F17D1FFE7029820
:1085200000F440300499896AC9034FF6FF72914301
:10853000A1F58031884209D1FFE7029800F0706010
:108540000499C96AB0EB016F04D0FFE701208DF8F0
:10855000170006E0FFE7FFE7FFE700208DF81700B0
:10856000FFE79DF8170006B080BD000080B582B01F
:108570000190019804F05EFB8DF803009DF8030064
:1085800002281BD0FFE7019804F054FB014640F29B
:108590007450C2F2000000EB4110806968B1FFE73F
:1085A000019804F047FB014640F27450C2F200000B
:1085B00000EB411080698047FFE7FFE702B080BD14
:1085C00080B584B00290029820B9FFE701208DF8B1
:1085D0000F0071E00298406A60B9FFE702984068B6
:1085E000B0F5827F01D1FFE703E002990020C86166
:1085F000FFE705E002990020086102994861FFE762
:10860000029900208862029890F8510040B9FFE773
:108610000299002081F85000029800F051F8FFE71D
:108620000299022081F8510002980168086820F040
:1086300040000860029A019211685068D2F808C0A0
:10864000D36800F482700CF4044C604403F40063BB
:108650001844136903F002031844536903F001033B
:108660001844936903F400731844D36903F0380382
:108670001844136A03F080031843926A02F400520C
:1086800010430860029A508B00F004001168526A8F
:1086900002F010021044486002980168C86920F492
:1086A0000060C861029900204865029A012182F8A1
:1086B00051108DF80F00FFE79DF80F0004B080BD4A
:1086C00080B590B00F9000200E900D900C900B9004
:1086D0000A900F98006843F20001C4F20101884239
:1086E00040F0B680FFE7FFE70020099043F6440022
:1086F000C4F20200016841F480510160006800F496
:10870000805009900998FFE7FFE70020089043F6A2
:108710003000C4F20200016841F00201016000680B
:1087200000F0020008900898FFE7FFE7002007909C
:1087300043F63000C4F20200016841F0010101601B
:10874000006800F0010007900798FFE718200A90E2
:10875000022001900B90002005900C9003200290C5
:108760000D90052003900E9040F20040C4F20200EC
:108770000AA90491FEF7F4FEDDF804C0029A0398FA
:108780000499059B4FF0800ECDF828E0CDF82CC061
:108790000C930D920E900020C4F20200FEF7E0FE52
:1087A000059941F23C00C2F20000069046F24042B8
:1087B000C4F2020202604FF0C06242608160C16098
:1087C0004FF48062026141618161C1614FF44032C6
:1087D00002624162FEF738FD18B1FFE7FCF71AFEAE
:1087E000FFE7FFE70F9841F23C01C2F20001C164CC
:1087F0000F988863FFE741F29C00C2F200000090EE
:1088000046F25841C4F2020101604FF0C06141607C
:10881000402181600021C1604FF4806202614161AA
:108820008161C1614FF4003202624162FEF70CFDCA
:1088300018B1FFE7FCF7EEFDFFE7FFE70F9841F205
:108840009C01C2F2000181640F988863FFE7FFE793
:1088500010B080BD80B588B006900591ADF81220AB
:108860000393069890F85100012804D0FFE70220F6
:108870008DF81F0011E1059820B1FFE7BDF8120047
:1088800020B9FFE701208DF81F0006E10698406837
:10889000B0F5827F16D1FFE70698806890B9FFE7B0
:1088A0000699042081F851000698059ABDF8123007
:1088B0000399EC46CCF80010114600F065FB8DF8EA
:1088C0001F00EAE0FFF758F80290FFE7069890F8DB
:1088D0005000012804D1FFE702208DF81F00DCE0E2
:1088E0000699012081F85000FFE7FFE70699042070
:1088F00081F851000699002048650599069A916310
:10890000BDF81210069A9187BDF81210069AD18709
:1089100006990863069988860699C88606990864A8
:108920000699486406988068B0F5004F0DD1FFE7BE
:1089300006980168086820F0400008600698016801
:10894000086820F480400860FFE706980068006827
:1089500000F04000402807D0FFE70698016808684B
:1089600040F040000860FFE70698C068D0BBFFE712
:10897000FFE70698C08FA0B3FFE7069800688068FD
:10898000C00778B1FFE706980068007B0699896BFD
:1089900008700699886B013088630699C88F013882
:1089A000C8871DE0FEF7E8FF0299401A0399884244
:1089B00004D3FFE70398013018B9FFE7039870B9B3
:1089C000FFE70699012081F85100FFE70699002092
:1089D00081F85000FFE703208DF81F005DE0FFE7FE
:1089E000C7E739E0FFE70698C08FA0B3FFE7069816
:1089F00000688068C00778B1FFE706980068C06823
:108A00000699896B08800699886B023088630699FD
:108A1000C88F0138C8871DE0FEF7AEFF0299401AE3
:108A20000399884204D3FFE70398013018B9FFE7A0
:108A3000039870B9FFE70699012081F85100FFE71C
:108A40000699002081F85000FFE703208DF81F00F1
:108A500023E0FFE7C7E7FFE706980399029A04F0CF
:108A600011F820B1FFE7069920204865FFE7069935
:108A7000012081F85100FFE70699002081F850009D
:108A8000FFE70698406D20B1FFE701208DF81F0039
:108A900003E000208DF81F00FFE79DF81F0008B0DD
:108AA00080BD000080B584B002900191ADF8022035
:108AB000029890F85100012804D0FFE702208DF8B9
:108AC0000F00B7E0019820B1FFE7BDF8020020B920
:108AD000FFE701208DF80F00ACE002988068A0B994
:108AE000FFE702984068B0F5827F0ED1FFE7029958
:108AF000042081F851000298019ABDF80230114615
:108B000000F014FC8DF80F0094E0FFE7029890F855
:108B10005000012804D1FFE702208DF80F0089E002
:108B20000299012081F85000FFE7FFE70299042035
:108B300081F851000299002048650199029A9163D9
:108B4000BDF80210029A9187BDF80210029AD187EF
:108B50000299086402994864029988860299C88635
:108B600002988068B0F5004F0DD1FFE702980168C8
:108B7000086820F04000086002980168086820F446
:108B800080400860FFE70298C16C4CF66900C0F6AF
:108B9000000008640298C16C4CF6B100C0F60000F9
:108BA000C8630298C16C4CF63500C0F60000C8647A
:108BB0000298C16C00200865029B19689A6BD86CFA
:108BC0000C31DB8FFEF7F8FB78B1FFE70299486DB7
:108BD00040F010004865FFE70299002081F850003E
:108BE000FFE701208DF80F0024E00298006800687C
:108BF00000F04000402807D0FFE7029801680868AD
:108C000040F040000860FFE7FFE70299002081F88C
:108C10005000FFE702980168486840F02000486073
:108C200002980168486840F00100486000208DF813
:108C30000F00FFE79DF80F0004B080BD80B582B043
:108C40000190019803F0F6FF8DF803009DF80300F2
:108C500002281BD0FFE7019803F0ECFF014640F229
:108C60007450C2F2000000EB4110406868B1FFE7A9
:108C7000019803F0DFFF014640F27450C2F2000099
:108C800000EB411040688047FFE7FFE702B080BD7E
:108C900080B582B00190019803F0CCFF8DF80300FD
:108CA0009DF8030002281BD0FFE7019803F0C2FFE4
:108CB000014640F27450C2F2000000EB411000691E
:108CC00068B1FFE7019803F0B5FF014640F2745028
:108CD000C2F2000000EB411000698047FFE7FFE7A8
:108CE00002B080BD80B588B006900591ADF8122025
:108CF0000393FEF741FE0290BDF81200ADF80600A6
:108D0000069890F85100012804D0FFE702208DF862
:108D10001F0034E1059820B1FFE7BDF8120020B92B
:108D2000FFE701208DF81F0029E1FFE7069890F882
:108D30005000012804D1FFE702208DF81F001EE13A
:108D40000699012081F85000FFE7FFE7069903200C
:108D500081F851000699002048650599069A11632B
:108D6000BDF81210069A9186BDF81210069AD186A7
:108D700006998863069988870699C8870699486482
:108D80000699086406988068B0F5004F0DD1FFE79A
:108D900006980168086820F040000860069801689D
:108DA000086840F480400860FFE7069800680068A3
:108DB00000F04000402807D0FFE7069801680868E7
:108DC00040F040000860FFE70698C068B0F5006F0B
:108DD00051D1FFE70698406828B1FFE7BDF80600CB
:108DE00001280ED1FFE706980168006B0088C86073
:108DF0000699086B023008630699C88E0138C88648
:108E0000FFE7FFE70698C08EA0B3FFE7069800686B
:108E10008068800700280ED5FFE706980168006B80
:108E20000088C8600699086B023008630699C88EEE
:108E30000138C8861DE0FEF79FFD0299401A03998C
:108E4000884204D3FFE70398013018B9FFE703987D
:108E500070B9FFE70699012081F85100FFE70699F4
:108E6000002081F85000FFE703208DF81F0086E006
:108E7000FFE7C7E750E00698406828B1FFE7BDF874
:108E8000060001280ED1FFE706980168006B007804
:108E900008730699086B013008630699C88E01387B
:108EA000C886FFE7FFE70698C08EA0B3FFE70698E5
:108EB00000688068800700280ED5FFE706980168E3
:108EC000006B007808730699086B013008630699F7
:108ED000C88E0138C8861DE0FEF74EFD0299401A83
:108EE0000399884204D3FFE70398013018B9FFE7DC
:108EF000039870B9FFE70699012081F85100FFE758
:108F00000699002081F85000FFE703208DF81F002C
:108F100035E0FFE7C7E7FFE706980399029A03F0F9
:108F200023FE20B1FFE7069920204865FFE7069859
:108F3000806870B9FFE7FFE700200090069800689E
:108F4000C068009006980068806800900098FFE76D
:108F5000FFE70699012081F85100FFE706990020FC
:108F600081F85000FFE70698406D20B1FFE701202F
:108F70008DF81F0003E000208DF81F00FFE79DF82B
:108F80001F0008B080BD000080B58CB0DDF838C08F
:108F90000A9009910892ADF81E3001200390FEF767
:108FA000EBFC04900A9890F851008DF817000A988D
:108FB00040680690BDF81E00ADF81C009DF8170033
:108FC000012812D0FFE70698B0F5827F09D1FFE7AC
:108FD0000A98806828B9FFE79DF81700042804D094
:108FE000FFE702208DF82F009BE1099838B1FFE7D9
:108FF000089820B1FFE7BDF81E0020B9FFE7012067
:109000008DF82F008DE1FFE70A9890F850000128B5
:1090100004D1FFE702208DF82F0082E10A99012098
:1090200081F85000FFE7FFE70A9890F85100042804
:1090300005D0FFE70A99052081F85100FFE70A995A
:109040000020486508990A9A9163BDF81E100A9A93
:10905000D187BDF81E100A9A918709990A9A11635F
:10906000BDF81E100A9AD186BDF81E100A9A918684
:109070000A9908640A9948640A980068006800F030
:109080004000402807D0FFE70A980168086840F0D0
:1090900040000860FFE70A98C068B0F5006F40F034
:1090A0008180FFE70A98406828B1FFE7BDF81C00FF
:1090B00001280ED1FFE70A980168006B0088C8609C
:1090C0000A99086B023008630A99C88E0138C8866D
:1090D000FFE7FFE70A98C18E0120019039B9FFE749
:1090E0000A98C08F002818BF01200190FFE701985F
:1090F000C007002855D0FFE70A98006880688007FD
:10910000002818D5FFE70A98C08EA0B1FFE70398A2
:10911000012810D1FFE70A980168006B0088C86039
:109120000A99086B023008630A99C88E0138C8860C
:1091300000200390FFE70A9800688068C007A8B184
:10914000FFE70A98C08F88B1FFE70A980068C068F7
:109150000A99896B08800A99886B023088630A999A
:10916000C88F0138C88701200390FFE7FEF704FC91
:109170000499401A0E99884212D3FFE70E980130E5
:1091800070B1FFE70A99012081F85100FFE70A99C1
:10919000002081F85000FFE703208DF82F00C0E089
:1091A00098E782E00A98406828B1FFE7BDF81C0004
:1091B00001280ED1FFE70A980168006B0078087358
:1091C0000A99086B013008630A99C88E0138C8866D
:1091D000FFE7FFE70A98C18E0120009039B9FFE749
:1091E0000A98C08F002818BF01200090FFE7009860
:1091F000C007002858D0FFE70A98006880688007F9
:10920000002818D5FFE70A98C08EA0B1FFE70398A1
:10921000012810D1FFE70A980168006B00780873F5
:109220000A99086B013008630A99C88E0138C8860C
:1092300000200390FFE70A9800688068C007A8B183
:10924000FFE70A98C08F88B1FFE70A980068C068F6
:109250000A99896B08700A99886B013088630A99AA
:10926000C88F0138C88701200390FFE7FEF784FB11
:109270000499401A0E99884204D3FFE70E980130F2
:1092800018B9FFE70E9870B9FFE70A99012081F835
:109290005100FFE70A99002081F85000FFE7032002
:1092A0008DF82F003DE095E7FFE70A980E99049AA4
:1092B00003F05AFC68B1FFE70A9920204865FFE7F0
:1092C0000A99002081F85000FFE701208DF82F0057
:1092D00027E00A98806870B9FFE7FFE70020029056
:1092E0000A980068C06802900A9800688068029036
:1092F0000298FFE7FFE70A99012081F85100FFE794
:109300000A99002081F85000FFE70A98406D20B1CB
:10931000FFE701208DF82F0003E000208DF82F00DB
:10932000FFE79DF82F000CB080BD000080B588B02D
:10933000069005910492ADF80E30069890F8510011
:109340008DF807000698406802909DF807000128F4
:1093500012D0FFE70298B0F5827F09D1FFE70698A7
:10936000806828B9FFE79DF80700042804D0FFE7CC
:1093700002208DF81F00DFE0059838B1FFE7049860
:1093800020B1FFE7BDF80E0020B9FFE701208DF8FE
:109390001F00D1E0FFE7069890F85000012804D1A3
:1093A000FFE702208DF81F00C6E00699012081F832
:1093B0005000FFE7FFE7069890F85100042805D019
:1093C000FFE70699052081F85100FFE70699002084
:1093D00048650599069A1163BDF80E10069A9186A4
:1093E000BDF80E10069AD1860499069A9163BDF8CD
:1093F0000E10069A9187BDF80E10069AD18706992D
:10940000086406994864069890F8510004280FD122
:10941000FFE70698C16C4CF66900C0F600000864CE
:109420000698C16C4CF6B100C0F60000C8630EE0AF
:109430000698C16C4CF69900C0F6000008640698C6
:10944000C16C4CF6FD10C0F60000C863FFE706983B
:10945000C16C4CF63500C0F60000C8640698C16CBB
:1094600000200865069B19689A6BD86C0C31DB8F5D
:10947000FDF7A2FF78B1FFE70699486D40F01000B4
:109480004865FFE70699002081F85000FFE70120BA
:109490008DF81F0050E006980168486840F0010010
:1094A00048600698816C002008640699896CC8633E
:1094B0000699896CC8640699896C0865069B1A68C8
:1094C000196B986C0C32DB8EFDF776FF78B1FFE7F5
:1094D0000699486D40F010004865FFE706990020A6
:1094E00081F85000FFE701208DF81F0024E0069866
:1094F0000068006800F04000402807D0FFE70698A9
:109500000168086840F040000860FFE7FFE706993F
:10951000002081F85000FFE706980168486840F095
:109520002000486006980168486840F002004860E2
:1095300000208DF81F00FFE79DF81F0008B080BDD8
:1095400080B584B002900191ADF80220029890F8A5
:109550005100012804D0FFE702208DF80F00A1E0A0
:10956000019820B1FFE7BDF8020020B9FFE7012014
:109570008DF80F0096E0FFE7029890F85000012860
:1095800004D1FFE702208DF80F008BE00299012043
:1095900081F85000FFE7FFE70299032081F85100AE
:1095A0000299002048650199029A1163BDF80210E2
:1095B000029A9186BDF80210029AD18602998863B8
:1095C0000299486402990864029988870299C887B9
:1095D00002988068B0F5004F0DD1FFE7029801684E
:1095E000086820F04000086002980168086840F4AC
:1095F00080400860FFE70298816C4CF68100C0F65D
:10960000000008640298816C4CF65510C0F600000A
:10961000C8630298816C4CF63500C0F60000C8643F
:109620000298816C00200865029B1A68196B986C7F
:109630000C32DB8EFDF7C0FE78B1FFE70299486D72
:1096400040F010004865FFE70299002081F85000C3
:10965000FFE701208DF80F0024E002980068006801
:1096600000F04000402807D0FFE702980168086832
:1096700040F040000860FFE7FFE70299002081F812
:109680005000FFE702980168486840F020004860F9
:1096900002980168486840F00200486000208DF898
:1096A0000F00FFE79DF80F0004B080BD80B582B0C9
:1096B0000190019803F0BEFA8DF803009DF80300B5
:1096C000022815D0FFE79DF80300410140F27450D5
:1096D000C2F20000405850B1FFE79DF8030041017D
:1096E00040F27450C2F2000040588047FFE7FFE7A5
:1096F00002B080BD80B582B00190019803F09AFA63
:109700008DF803009DF8030002281BD0FFE70198A5
:1097100003F090FA014640F27450C2F2000000EBF0
:109720004110C06868B1FFE7019803F083FA014671
:1097300040F27450C2F2000000EB4110C068804754
:10974000FFE7FFE702B080BD80B582B001900198CD
:1097500003F070FA8DF803009DF8030002281BD077
:10976000FFE7019803F066FA014640F27450C2F236
:10977000000000EB4110806868B1FFE7019803F03A
:1097800059FA014640F27450C2F2000000EB411059
:1097900080688047FFE7FFE702B080BD80B582B0F8
:1097A0000190019803F046FA8DF803009DF803003C
:1097B00002281BD0FFE7019803F03CFA014640F273
:1097C0007450C2F2000000EB4110406968B1FFE73D
:1097D000019803F02FFA014640F27450C2F20000E3
:1097E00000EB411040698047FFE7FFE702B080BD12
:1097F00080B582B00190019804F020FC02B080BDD9
:1098000080B582B00090009820B9FFE701208DF864
:1098100007003FE0009890F83D0040B9FFE700994D
:10982000002081F83C00009800F038F8FFE700992C
:10983000022081F83D00009951F8040B04F09CFCD3
:109840000099012081F84600FFE70099012081F886
:109850003E00009981F83F00009981F8400000998E
:1098600081F84100FFE7FFE70099012081F84200FD
:10987000009981F84300009981F84400009981F82B
:109880004500FFE70099012081F83D0000208DF898
:109890000700FFE79DF8070002B080BD82B001908D
:1098A0000198006844F20041C4F20101884212D1DB
:1098B000FFE7FFE70020009043F64400C4F20200F7
:1098C000016841F400310160006800F4003000904C
:1098D0000098FFE7FFE702B07047000080B588B04E
:1098E000079000200690059004900390029007983E
:1098F000006844F20041C4F20101884222D1FFE72E
:10990000FFE70020019043F63000C4F20200016836
:1099100041F020010160006800F0200001900198F2
:10992000FFE740200290022003900021049105905F
:109930000320069041F20040C4F2020002A9FDF7A4
:109940000FFEFFE708B080BD80B586B0049003919C
:10995000029200208DF80700FFE7049890F83C0081
:10996000012804D1FFE702208DF8170089E004994F
:10997000012081F83C00FFE7FFE7029800900C28E7
:1099800000F270800099DFE801F0076D6D6D206DC9
:109990006D6D3A6D6D6D530004980068039904F085
:1099A000D9FC04980168886940F00800886104982F
:1099B0000168886920F004008861039802690498AE
:1099C000016888691043886150E004980068039931
:1099D00004F036FD04980168886940F400608861ED
:1099E00004980168886920F480608861039802699E
:1099F00004980168886940EA0220886136E004988A
:109A00000068039904F096FD04980168C86940F065
:109A10000800C86104980168C86920F00400C861A2
:109A20000398026904980168C8691043C8611DE081
:109A300004980068039904F0F7FD04980168C86968
:109A400040F40060C86104980168C86920F480602F
:109A5000C8610398026904980168C86940EA022055
:109A6000C86103E001208DF80700FFE7FFE70499D4
:109A7000002081F83C00FFE79DF807008DF81700F3
:109A8000FFE79DF8170006B080BD000080B582B0EA
:109A90000090009820B9FFE701208DF807003FE013
:109AA000009890F83D0040B9FFE70099002081F848
:109AB0003C00009800F038F8FFE70099022081F898
:109AC0003D00009951F8040B04F056FB0099012069
:109AD00081F84600FFE70099012081F83E000099D7
:109AE00081F83F00009981F84000009981F8410019
:109AF000FFE7FFE70099012081F84200009981F813
:109B00004300009981F84400009981F84500FFE77F
:109B10000099012081F83D0000208DF80700FFE743
:109B20009DF8070002B080BD81B0009001B0704781
:109B300080B58CB00A900991099828B9FFE70A9876
:109B400090F83E0007901CE00998042805D1FFE733
:109B50000A9890F83F00069010E00998082805D16F
:109B6000FFE70A9890F84000059004E00A9890F802
:109B700041000590FFE705980690FFE706980790DB
:109B8000FFE70798012804D0FFE701208DF82F0098
:109B9000AFE0099828B9FFE70A99022081F83E0052
:109BA0001EE00998042806D1FFE70A99022081F8EF
:109BB0003F00049012E00998082806D1FFE70A99AF
:109BC000022081F84000039005E00A99022081F804
:109BD00041000390FFE703980490FFE70498FFE734
:109BE0000A98006809990122019204F097FB0198F4
:109BF0000A9909680022C4F20102914202900CD035
:109C0000FFE70A9800684FF60041CBF6FE71084462
:109C1000B0FA80F040090290FFE70298C00738B11F
:109C2000FFE70A980168486C40F400404864FFE789
:109C30000A9800680021C4F2010188423CD0FFE785
:109C40000A980068B0F1804F36D0FFE70A980068A4
:109C500040F20041C4F2000188422DD0FFE70A988B
:109C6000006840F60001C4F20001884224D0FFE7FA
:109C70000A98006840F60041C4F2000188421BD0F7
:109C8000FFE70A98006840F20041C4F201018842EF
:109C900012D0FFE70A98006844F20001C4F2010103
:109CA000884209D0FFE70A98006841F60001C4F233
:109CB0000001884212D1FFE70A980068806800F02E
:109CC000070008900898062807D0FFE70A9801685F
:109CD000086840F001000860FFE706E00A980168A4
:109CE000086840F001000860FFE700208DF82F00B1
:109CF000FFE79DF82F000CB080BD000082B00190FE
:109D0000ADF8021002B0704780B582B001900198A2
:109D100005F0AAFA8DF803009DF8030003281BD074
:109D2000FFE79DF8030000EBC00140F29850C2F23B
:109D3000000000EB8100006968B1FFE79DF80300B7
:109D400000EBC00140F29850C2F2000000EB81002D
:109D500000698047FFE7FFE702B080BD80B592B0A1
:109D60001190119800680068109011980068C06800
:109D70000F901198006840690E9000200D900C9093
:109D8000109800F00F000D900D9888B9FFE79DF82E
:109D90004000800600280AD5FFE79DF83C008006B9
:109DA000002804D5FFE7119805F082FA02E2FFE7E8
:109DB0000D98002800F0C280FFE79DF83800C0072A
:109DC00038B9FFE7BDF83C0010F4907F00F0B68092
:109DD000FFE79DF84000C00758B1FFE79DF83D0040
:109DE000C00730B1FFE71199486C40F001004864AA
:109DF000FFE79DF84000400700280BD5FFE79DF8DE
:109E00003800C00730B1FFE71199486C40F00200FC
:109E10004864FFE79DF84000800700280BD5FFE766
:109E20009DF83800C00730B1FFE71199486C40F049
:109E300004004864FFE79DF840000007002811D5A2
:109E4000FFE79DF83C008006002805D4FFE79DF859
:109E50003800C00730B1FFE71199486C40F00800A6
:109E60004864FFE71198406C002866D0FFE79DF832
:109E70004000800600280AD5FFE79DF83C008006D8
:109E8000002804D5FFE7119805F012FAFFE71198B2
:109E900000684069C0F380100C901198406C000776
:109EA000002804D4FFE70C9800283ED0FFE7119863
:109EB00005F060F9119800684069400600282FD528
:109EC000FFE7FFE7FFE71198006850E8050F20F073
:109ED00040000B90FFE70B991198026842E80510CB
:109EE0000028F0D1FFE7FFE71198C06B98B1FFE7BA
:109EF0001198C16B4EF6B570C0F600000865119858
:109F0000C06BFCF7EFFF28B1FFE71198C06B016D44
:109F10008847FFE703E01198FFF7F6FEFFE703E04D
:109F20001198FFF7F1FEFFE706E01198FFF7ECFE4E
:109F3000119900204864FFE7FFE73BE11198006BAF
:109F4000012840F01781FFE79DF84000C006002877
:109F500040F11081FFE79DF83C00C006002840F169
:109F60000981FFE7FFE700200A9011980068006868
:109F70000A901198006840680A900A98FFE71198C3
:109F8000006840694006002840F19A80FFE7119878
:109F9000C06B00684068ADF82600BDF826000028B8
:109FA00075D0FFE7BDF826001199898D88426EDAD9
:109FB000FFE7BDF826001199C8851198C06BC069EC
:109FC000B0F5807F58D0FFE7FFE7FFE71198006802
:109FD00050E8030F20F480700890FFE7089911986B
:109FE000026842E803100028F0D1FFE7FFE7FFE72F
:109FF000FFE71198006850E8050F20F00100079076
:10A00000FFE707991198026842E805100028F0D18F
:10A01000FFE7FFE7FFE7FFE71198006850E8050F4B
:10A0200020F040000690FFE706991198026842E888
:10A0300005100028F0D1FFE7FFE71199202081F8F3
:10A040004200119900200863FFE7FFE711980068BC
:10A0500050E8030F20F010000590FFE705991198D4
:10A06000026842E803100028F0D1FFE7FFE71198EB
:10A07000C06BFCF7C1FEFFE71199022048631198FD
:10A08000818DC28D891A89B2FFF738FE17E0BDF8BD
:10A0900026001199898D884210D1FFE71198C06B75
:10A0A000C069B0F5807F08D1FFE7119902204863AD
:10A0B0001198818DFFF722FEFFE7FFE7FFE779E0C8
:10A0C0001199888DC98D401AADF812001198C08D74
:10A0D00000284ED0FFE7BDF81200002849D0FFE766
:10A0E000FFE7FFE71198006850E8030F20F4907035
:10A0F0000390FFE703991198026842E803100028D3
:10A10000F0D1FFE7FFE7FFE7FFE71198006850E8AD
:10A11000050F20F001000290FFE7029911980268F4
:10A1200042E805100028F0D1FFE7FFE71199202051
:10A1300081F84200119900200863FFE7FFE71198BA
:10A14000006850E8030F20F010000190FFE701992C
:10A150001198026842E803100028F0D1FFE7FFE7FA
:10A160001199022048631198BDF81210FFF7C6FD3F
:10A17000FFE71FE09DF84000000600280AD5FFE732
:10A180009DF83C000006002804D5FFE7119805F073
:10A1900079FA0FE09DF84000400600280AD5FFE755
:10A1A0009DF83C004006002804D5FFE7119805F013
:10A1B0002BF8FFE712B080BD80B582B00090009808
:10A1C00020B9FFE701208DF8070040E00098806982
:10A1D00008B1FFE700E0FFE7009890F8410040B9C0
:10A1E000FFE70099002081F84000009800F034F863
:10A1F000FFE70099242081F8410000980168C868B1
:10A2000020F40050C860009805F006F90098016835
:10A21000086920F49040086100980168486920F0BE
:10A220002A00486100980168C86840F40050C8607E
:10A23000009900204864009A202182F84110009A79
:10A2400082F84210009948638DF80700FFE79DF8F7
:10A25000070002B080BD000080B59CB01B900020BC
:10A260001A9019901890179016901B98006841F258
:10A270000001C4F20101884240F09380FFE7FFE74C
:10A280000020159043F64400C4F20200016841F03A
:10A2900010010160006800F0100015901598FFE7AC
:10A2A000FFE70020149043F63000C4F2020001687A
:10A2B00041F002010160006800F00200149014985F
:10A2C000FFE7FFE70020139043F63000C4F20200DE
:10A2D000016841F001010160006800F00100139085
:10A2E0001398FFE780201690022009901790002015
:10A2F0000D90189003200A90199007200B901A9047
:10A3000040F20040C4F2020016A90C91FDF728F9B2
:10A31000DDF824C00A9A0B980C990D9B4FF4007E2F
:10A32000CDF858E0CDF85CC0189319921A9000202F
:10A33000C4F20200FDF714F90D9941F2FC00C2F2DB
:10A3400000000E9046F28842C4F2020202604FF012
:10A35000006242608160C1604FF4806202614161CD
:10A360008161C1614FF4403202624162FCF76CFFCF
:10A3700018B1FFE7FBF74EF8FFE7FFE71B9841F244
:10A38000FC01C2F20001C1631B988863FFE725202E
:10A39000089005210022FDF797FB0898FDF78AFB3E
:10A3A00014E11B98006844F60001C4F200018842E1
:10A3B0006AD1FFE7FFE70020129043F64000C4F2A5
:10A3C0000200016841F480210160006800F48020EF
:10A3D00012901298FFE7FFE70020119043F630003B
:10A3E000C4F20200016841F004010160006800F05D
:10A3F000040011901198FFE74FF44060169002207E
:10A4000017900020069018900320199007201A90AA
:10A4100040F60000C4F2020016A9FDF7A1F8069963
:10A4200041F25C10C2F20000079046F22802C4F22A
:10A43000020202604FF0006242608160C1604FF42E
:10A4400080620261416181614FF48072C261016288
:10A450004162FCF7F9FE18B1FFE7FAF7DBFFFFE70F
:10A46000FFE71B9841F25C11C2F20001C1631B9827
:10A470008863FFE72720059005210022FDF724FBD4
:10A480000598FDF717FBA0E01B98006841F200411A
:10A49000C4F20101884240F09780FFE7FFE7002007
:10A4A000109043F64400C4F20200016841F020011C
:10A4B0000160006800F0200010901098FFE7FFE7AF
:10A4C00000200F9043F63000C4F20200016841F012
:10A4D00040010160006800F040000F900F98FFE716
:10A4E0004FF484401690022017900020039018909B
:10A4F0000320199008201A9041F60000C4F20200CF
:10A5000016A9FDF72DF8039941F2BC10C2F2000024
:10A51000049046F22842C4F2020202604FF0206228
:10A5200042608160C1604FF480620261416181617B
:10A53000C1614FF4803202624162FCF785FE18B1BE
:10A54000FFE7FAF767FFFFE7FFE71B9841F2BC114F
:10A55000C2F20001C1631B988863FFE741F21C202F
:10A56000C2F20000029046F2A041C4F20201016072
:10A570004FF020614160402181600021C1604FF4B3
:10A580008062026141618161C1614FF48032026287
:10A590004162FCF759FE18B1FFE7FAF73BFFFFE70E
:10A5A000FFE71B9841F21C21C2F2000181631B9856
:10A5B0008863FFE74720019005210022FDF784FA18
:10A5C0000198FDF777FAFFE7FFE7FFE71CB080BDD2
:10A5D00080B584B002900191ADF80220029890F805
:10A5E0004200202817D1FFE7019820B1FFE7BDF80E
:10A5F000020020B9FFE701208DF80F000FE002995B
:10A600000020086302980199BDF8022004F0A2FF1F
:10A610008DF80F0003E002208DF80F00FFE79DF892
:10A620000F0004B080BD000080B582B00190019899
:10A6300004F01AFE8DF803009DF8030003281BD0D8
:10A64000FFE79DF8030000EBC00140F29850C2F212
:10A65000000000EB8100C06868B1FFE79DF80300CF
:10A6600000EBC00140F29850C2F2000000EB810004
:10A67000C0688047FFE7FFE702B080BD80B582B0C9
:10A680000190019804F0F0FD8DF803009DF803009F
:10A6900003281BD0FFE79DF8030000EBC00140F248
:10A6A0009850C2F2000000EB8100806868B1FFE7BB
:10A6B0009DF8030000EBC00140F29850C2F2000088
:10A6C00000EB810080688047FFE7FFE702B080BDB4
:10A6D00080B582B00190019804F0C6FD8DF80300AA
:10A6E0009DF8030003281BD0FFE79DF8030000EB53
:10A6F000C00140F29850C2F2000000EB81004068B7
:10A7000068B1FFE79DF8030000EBC00140F29850EC
:10A71000C2F2000000EB810040688047FFE7FFE7DE
:10A7200002B080BDFFE7FEE784B08DED030A9DED2A
:10A73000030AB6EE001A20EE010A8DED020A039814
:10A74000019001980090009945F6DF10C5F637702A
:10A75000A0EB61000090009801909DED010A9DED35
:10A76000021A21EE001A21EE002AB7EE081A31EE85
:10A77000422A20EE020A8DED010A9DED010A9DEDAF
:10A78000022A22EE002A22EE002A31EE421A20EEA0
:10A79000010A8DED010A9DED010A04B07047000029
:10A7A00083B0ADF80A00BDF90A0040F26111884299
:10A7B00003D1FFE70120019015E0BDF90A00B0F5D3
:10A7C000806F03D1FFE70320009009E0BDF90A0084
:10A7D000A0F29F60B0FA80F0400940000090FFE7CF
:10A7E00000980190FFE70198C0B203B070470000E5
:10A7F00080B586B004908DED030A049818B9FFE780
:10A80000002005904CE09DED030A049890ED014A6C
:10A8100090ED022A90ED063A90ED071A23EE043AE5
:10A8200030EE430A21EE021A30EE410A8DED020AA3
:10A83000002028B9FFE7029804F0E6FF58B90DE0C0
:10A8400002980DF015F841EC100B51EC100B04F0D0
:10A85000C1FF18B1FFE703980290FFE79DED020AE0
:10A86000049890ED034A90ED043A90ED052A90ED9E
:10A87000061A20EE040A21EE031A30EE010A90EDCA
:10A88000071A21EE021A30EE010A8DED010A049931
:10A890008869C86102980499886101980590FFE76A
:10A8A0009DED050A06B080BD80B588B007908DED9E
:10A8B000060ACDED050A079808B9FFE78BE0059871
:10A8C000079908600799002088610799C86107986F
:10A8D00090ED000AB5EE400AF1EE10FA0EDCFFE74B
:10A8E00007994FF07E50C8600799002008610799CA
:10A8F000486107994860079988606CE09DED060AF9
:10A90000079890ED001A80EE010A8DED040A9DED86
:10A91000041A9FED320A80EE010A0BF04BFA8DED1E
:10A92000030A9FED2F0A8DED000A0AF07DF9B0EEC3
:10A93000401A9DED000A31EE011A9DED033A21EE19
:10A94000031AB7EE002A8DED012A31EE021A23EE2A
:10A95000033A31EE031A8DED021A9DED031A21EE32
:10A96000011A9DED023A81EE031A079880ED031A51
:10A97000079890ED031A31EE011A80ED041A079939
:10A98000C86848619DED031A21EE011A31EE421AA2
:10A9900031EE011A9DED022A81EE021A079880ED30
:10A9A000011A0AF041F9B0EE401A9DED010A31EEAC
:10A9B000012A9DED031A22EE012A30EE420A21EE11
:10A9C000011A30EE010A9DED021A80EE010A079885
:10A9D00080ED020AFFE708B080BD00BFDB0F4940F1
:10A9E000DB0F493F80B584B002908DED010A0298DB
:10A9F00018B9FFE70020039039E09DED010A0298A5
:10AA000090ED031A90ED043A90ED052A31EE031A09
:10AA100031EE021A80EE010A8DED000A002028B9FD
:10AA2000FFE7009804F0BEFE58B911E000980CF062
:10AA30001FFF41EC100B51EC100B04F093FE38B1EA
:10AA4000FFE700980299886100980299C86106E0C2
:10AA500001980299886101980299C861FFE70298FC
:10AA60009DED010AFFF7C4FE8DED030AFFE79DEDA2
:10AA7000030A04B080BD000080B582B08DF80600E6
:10AA80009DF80600022804DBFFE7FF208DF8070091
:10AA900039E09DF8061040F24460C2F2000050F820
:10AAA000210020B1FFE700208DF807002BE088206F
:10AAB000F8F74AFA01469DF8062040F24460C2F2D7
:10AAC000000040F822109DF8061050F8210020B92F
:10AAD000FFE7FF208DF8070015E09DF8061040F213
:10AAE0004460C2F20000009050F821008821F5F780
:10AAF000F2FC00999DF8060051F820100870002023
:10AB00008DF80700FFE79DF9070002B080BD000047
:10AB100080B588B00690069820B9FFE7FE208DF832
:10AB20001F002EE0069800F049F80590059820B91E
:10AB3000FFE7FC208DF81F0023E005988088019036
:10AB400008208DF80800FF208DF809008DF80A0014
:10AB50008DF80B008DF80C008DF80D008DF80E00AF
:10AB60008DF80F00FC208DF810000598007801A9E1
:10AB7000F7F7A2FF002818BF4FF0FF308DF81F0035
:10AB8000FFE79DF91F0008B080BD000082B08DF87E
:10AB900003009DF80300022803DBFFE7002001907B
:10ABA00009E09DF8031040F24460C2F2000050F842
:10ABB00021000190FFE7019802B0704780B586B090
:10ABC0000490049818B9FFE70020059036E0049837
:10ABD0000078FFF7DBFF0390039818B9FFE7002028
:10ABE00005902BE000200290FFE70298039991F86E
:10ABF000841088421FDAFFE70398029900EB810076
:10AC000040680190019888B1FFE7019800780499A5
:10AC1000097888420AD1FFE7019840880499498859
:10AC2000884203D1FFE70198059007E0FFE702980B
:10AC300001300290D9E700200590FFE7059806B0A3
:10AC400080BD000080B584B002900191029818B1D7
:10AC5000FFE7019820B9FFE7FE208DF80F0011E013
:10AC60000298FFF7ABFF0090009820B9FFE7FC20A7
:10AC70008DF80F0006E00098019900F049F98DF871
:10AC80000F00FFE79DF90F0004B080BD80B586B0CE
:10AC900004900391049818B1FFE7039820B9FFE7E7
:10ACA000FE208DF8170090E003984178807840EA04
:10ACB0000120ADF80A00BDF80A009FED460ADFED5D
:10ACC000460A102106F04EFF049880ED070A03990A
:10ACD000C8780979000140EA1110ADF80800BDF804
:10ACE0000800BBEE0E0AF3EE0E0A0C21009106F0EE
:10ACF00039FF0099049880ED080A03980279407999
:10AD000002F00F0240EA0220ADF80600BDF806008E
:10AD1000BAEE080AF2EE080A06F024FF049880ED65
:10AD2000090A0398807900EE100AB8EE400A0498E8
:10AD300080ED0A0AFFE7049890ED070AB5EE400A95
:10AD4000F1EE10FA0ADAFFE7049890ED070A9FED9A
:10AD5000231A30EE010A80ED070AECE7FFE70498BA
:10AD600090ED070A9FED1D1AB4EE410AF1EE10FABC
:10AD70000ADBFFE7049890ED070A9FED191A30EE01
:10AD8000010A80ED070AEAE70498C079C007C0B15C
:10AD9000FFE7049890ED071A9FED100A30EE410A84
:10ADA00080ED070A049890ED080AB1EE400A80EDA4
:10ADB000080A049890ED090AB1EE400A80ED090AEC
:10ADC000FFE700208DF81700FFE79DF9170006B098
:10ADD00080BD00BFDA0F49C1DA0F4941DB0FC9401E
:10ADE000DB0FC9C080B586B00490049820B9FFE796
:10ADF000FE208DF8170087E004980078FFF73CFEEE
:10AE000020B1FFE7FF208DF817007DE0049800785F
:10AE1000FFF7BCFE0390039820B9FFE7FF208DF8F1
:10AE2000170071E000200290FFE70298039991F863
:10AE3000841088421BDAFFE70398029900EB810037
:10AE4000406878B1FFE70398029900EB8100406801
:10AE5000408804994988884204D1FFE7FD208DF895
:10AE6000170051E0FFE7029801300290DDE70398F8
:10AE700090F88400202804DBFFE7FF208DF81700FE
:10AE800042E03020F8F760F80190019820B9FFE720
:10AE9000FF208DF8170037E001983021F5F71BFBF4
:10AEA0000199049A106852684A600860019900206C
:10AEB00008720498C079019900F00100087604989E
:10AEC0004088ADF8020004980078BDF80210032213
:10AED000F7F730FC38B1FFE70198F7F743FFFF20A1
:10AEE0008DF8170010E00198039991F8842001EB88
:10AEF00082014860039991F88400013081F8840050
:10AF000000208DF81700FFE79DF9170006B080BDFF
:10AF100080B58EB00C900B910C9818B1FFE70B9890
:10AF200020B9FFE7FE208DF8370087E00C98808875
:10AF3000ADF818000B9890ED020ADFED420A9FED84
:10AF4000421A102004F0CEFEADF822000B9890EDCE
:10AF5000010AFBEE0E0AB3EE0E1A0C20019004F06B
:10AF6000C1FE01460198ADF820100B9991ED030A3E
:10AF7000DFED360ACDED000A9FED351A04F0B2FE82
:10AF8000DDED000A01460198ADF81E100B9991ED18
:10AF9000040AB1EE041A04F0A5FE01460198ADF8CA
:10AFA0001C100B9991ED000AFAEE080AB2EE081A8D
:10AFB00004F098FEADF81A009DF823008DF82400E7
:10AFC0009DF822008DF82500BDF8200000098DF8BD
:10AFD0002600BDF820109DF81F0040EA01108DF8F2
:10AFE00027009DF81E008DF82800BDF81C00000900
:10AFF0008DF82900BDF81C109DF81B0040EA0110D7
:10B000008DF82A009DF81A008DF82B000C98808886
:10B01000029008208DF80C0009980A99CDF81110BB
:10B02000CDF80D000C98007802A9F7F745FD00282F
:10B0300018BF4FF0FF308DF83700FFE79DF937005C
:10B040000EB080BDDA0F49C1DA0F4941000000009F
:10B050000000FA4380B590B00E900E9820B9FFE73B
:10B06000FE208DF83F0077E00E980078FFF78EFD08
:10B070000D900D9820B9FFE7FC208DF83F006BE0A4
:10B0800000200C900B90FFE70B980D9991F884101D
:10B0900088421EDAFFE70D980B9900EB81004068AB
:10B0A00090B1FFE70D980B9900EB81004068408854
:10B0B0000E994988884207D1FFE70D980B9900EB5C
:10B0C000810040680C9004E0FFE70B9801300B9082
:10B0D000DAE70C9820B9FFE7FC208DF83F003BE051
:10B0E0000E984088ADF82A000E980078BDF82A1016
:10B0F00003AA0023F7F7B0F9E0B1FFE7F8F7ECF89F
:10B1000001910090009901980C9A13695269C91A2B
:10B11000904148F2A162C0F20102891A70F1000068
:10B1200004D3FFE70C9900200872FFE7FF208DF899
:10B130003F0011E00C9901200872F8F7CDF80A469B
:10B140000C994A6108610C9803A90D31FFF79EFD27
:10B1500000208DF83F00FFE79DF93F0010B080BD53
:10B1600082B00090009820B9FFE74FF04040019076
:10B1700003E0009840690190FFE79DED010A02B0ED
:10B180007047000082B00090009820B9FFE74FF0B0
:10B190004040019003E0009880690190FFE79DED39
:10B1A000010A02B07047000080B582B08DF8060039
:10B1B0009DF80600022804DBFFE7FF208DF807005A
:10B1C00039E09DF8061040F24C60C2F2000050F8E1
:10B1D000210020B1FFE700208DF807002BE0482078
:10B1E000F7F7B2FE01469DF8062040F24C60C2F22D
:10B1F000000040F822109DF8061050F8210020B9F8
:10B20000FFE7FF208DF8070015E09DF8061040F2DB
:10B210004C60C2F20000009050F821004821F5F780
:10B220005AF900999DF8060051F820100870002086
:10B230008DF80700FFE79DF9070002B080BD000010
:10B2400080B58EB00C900C9820B9FFE7FE208DF8E9
:10B250003700A9E00C98007800F0AAF80B900B9842
:10B2600020B9FFE7FC208DF837009DE00B980230F5
:10B270000A900C984088ADF81600BDF81610A1F29F
:10B280000120019104280CD3FFE70198A0F20520CA
:10B29000042829D3FFE70198A0F20920032849D305
:10B2A00072E04FF40070069008208DF81C0000201A
:10B2B0000490FFE70498032815DCFFE70A98049A36
:10B2C00000EB4200407806A9053101F812000A9807
:10B2D000049A30F8120001EB42014870FFE704982D
:10B2E00001300490E6E753E040F2FF10069008209A
:10B2F0008DF81C0004200390FFE70398072818DC52
:10B30000FFE70A98039A00EB4200407806A905314E
:10B3100001EB420202F8080C0A98039A30F8120076
:10B3200001EB420101F8070CFFE70398013003909D
:10B33000E3E72DE040F2FF20069008208DF81C0086
:10B340000290FFE702980A2818DCFFE70A98029AA1
:10B3500000EB4200407806A9053101EB420202F8F9
:10B36000100C0A98029A30F8120001EB420101F821
:10B370000F0CFFE7029801300290E3E700208DF800
:10B3800023008DF8240003E0FF208DF837000BE048
:10B390000C98007806A9F7F78FFB002818BF4FF02C
:10B3A000FF308DF83700FFE79DF937000EB080BD04
:10B3B00082B08DF803009DF80300022803DBFFE74D
:10B3C0000020019009E09DF8031040F24C60C2F2A9
:10B3D000000050F821000190FFE7019802B070478B
:10B3E00082B08DF805009DF805000146009140B13E
:10B3F000FFE70098012809D0FFE7009802280AD04B
:10B400000EE042F21070ADF806000EE04FF48040FE
:10B41000ADF8060009E047F23050ADF8060004E050
:10B420004FF6FF70ADF80600FFE7BDF9060002B069
:10B430007047000083B0ADF808008DF807109DF844
:10B44000070001460091022804D3FFE70098022874
:10B4500013D026E0BDF80800B0F5007F0CDDFFE753
:10B46000BDF80800B0F5027F06DAFFE7BDF8080076
:10B4700001388DF80B0019E014E0BDF80800B0F5B4
:10B48000017F0DDDFFE7BDF8080040F20A21884288
:10B4900006DCFFE7BDF8080001388DF80B0005E079
:10B4A00000E0FFE7FF208DF80B00FFE79DF90B00A0
:10B4B00003B0704780B586B00490049818B9FFE7D0
:10B4C000002005902FE004980078FFF771FF0390AB
:10B4D000039818B9FFE70020059024E000200290AF
:10B4E000FFE70298039991F84410884218DAFFE7C1
:10B4F0000398029900EB810080690190019850B196
:10B50000FFE70198408804994988884203D1FFE702
:10B510000198059007E0FFE7029801300290E0E70C
:10B5200000200590FFE7059806B080BD83B08DF838
:10B5300007009DF807000146009140B1FFE7009821
:10B54000012809D0FFE7009802280BD00EE0002068
:10B55000C4F2102002900DE043F63C40C4F27C108F
:10B56000029007E04FF07E50029003E04FF07E50D3
:10B570000290FFE79DED020A03B0704780B586B0E8
:10B580000490049820B9FFE7FE208DF8170081E0B1
:10B5900004980078FFF708FE20B1FFE7FF208DF840
:10B5A000170077E004980078FFF702FF03900398F4
:10B5B00020B9FFE7FF208DF817006BE00020029014
:10B5C000FFE70298039991F8441088421BDAFFE7DD
:10B5D0000398029900EB8100806978B1FFE7039836
:10B5E000029900EB8100806940880499498888426B
:10B5F00004D1FFE7FD208DF817004BE0FFE702982C
:10B6000001300290DDE7039890F844000B2804DB3A
:10B61000FFE7FF208DF817003CE05020F7F794FC7F
:10B620000190019820B9FFE7FF208DF8170031E065
:10B630000199049A106852684A60086001981830AD
:10B640002821F4F748FF04984079019900F001009F
:10B6500081F828000499087849880322F7F76AF8E6
:10B6600038B1FFE70198F7F77DFBFF208DF8170051
:10B6700010E00198039991F8442001EB8201886160
:10B68000039991F84400013081F8440000208DF8BE
:10B690001700FFE79DF9170006B080BD80B582B0A6
:10B6A000019001989FED020A00F004F802B080BDFD
:10B6B0000000000080B58AB007A9019101460198F9
:10B6C000089180ED000A089820B9FFE7FE208DF868
:10B6D000270078E008980078FFF76AFE0690069841
:10B6E00020B9FFE7FC208DF827006CE0019890ED71
:10B6F000000AB7EE001AB4EE410AF1EE10FA04DDCA
:10B70000FFE74FF07E500790FFE7019890ED000AA9
:10B71000BFEE001AB4EE410AF1EE10FA05DAFFE7C7
:10B720000020CBF680700790FFE708984079C007AB
:10B7300040B1FFE7019890ED000AB1EE400A80EDBC
:10B74000000AFFE70898FFF7B5FE0590059820B9B5
:10B75000FFE7FC208DF8270035E008994888097933
:10B76000FFF768FE8DF813009DF91300B0F1FF3F5D
:10B7700004DCFFE7FF208DF8270024E001980699FC
:10B780000231039190ED000A8DED000A08980079CE
:10B79000FFF726FE9DED000A01EE100AB8EEC11A71
:10B7A00020EE010ABDEEC00A10EE100AADF80A0044
:10B7B000BDF80A0003999DF9132021F8120000201A
:10B7C0008DF82700FFE79DF927000AB080BD000033
:10B7D00080B590B00E900E9820B9FFE7FE208DF84E
:10B7E0003F0072E00E980078FFF7E2FD0D900D9893
:10B7F00020B9FFE7FC208DF83F0066E000200C90A8
:10B80000FFE70C980D9991F84410884259DAFFE748
:10B810000D980C9900EB810080690B900B98002823
:10B820004AD0FFE70B9840880E994988884243D157
:10B83000FFE70E990878498804AA0023F6F70CFE62
:10B84000E8B1FFE7F7F748FD0391029002990398EA
:10B850000B9A136A526AC91A904140F2E932891A66
:10B8600070F1000007D3FFE70B9900200876FC2059
:10B870008DF83F0029E0FF208DF83F0025E00B996F
:10B8800001200876F7F728FD0A460B994A620862FC
:10B890000B9804A900F0F8FA0B9901918868CA681E
:10B8A0000B69D1F814C0C1F838C04B630A63C86291
:10B8B00000208DF83F0008E0FFE70C9801300C9065
:10B8C0009FE7FC208DF83F00FFE79DF93F0010B097
:10B8D00080BD000080B586B000208DF81700049070
:10B8E000FFE70498012830DCFFE79DF81000FFF720
:10B8F0005FFD0390039808B9FFE722E00020029063
:10B90000FFE70298039991F84410884218DAFFE79C
:10B910000398029900EB810080690190019850B171
:10B92000FFE70198FFF754FF20B1FFE7FF208DF8F4
:10B930001700FFE7FFE7FFE7029801300290E0E71A
:10B94000FFE7049801300490CBE79DF9170006B09B
:10B9500080BD000080B582B040F6EC70C2F20000FD
:10B96000009046F20041C4F20001016003214160F1
:10B97000002101918160C1604FF4A02202614FF467
:10B98000C0024261017641768176C17601774177C6
:10B99000FAF748FE18B1FFE7F9F73CFDFFE702B000
:10B9A00080BD000080B582B041F21400C2F20000F8
:10B9B000009046F60001C4F20001016003214160DD
:10B9C000002101918160C1604FF4A02202614FF417
:10B9D000C0024261017641768176C1760177417776
:10B9E000FAF720FE18B1FFE7F9F714FDFFE702B000
:10B9F00080BD000080B58AB0FFE70020099043F6C3
:10BA00003000C4F20200016841F480010160006866
:10BA100000F4800009900998FFE7FFE700200890F4
:10BA200043F63000C4F20200016841F400110160E5
:10BA3000006800F4001008900898FFE70C200090C0
:10BA40000521059100220692FCF73EF80098FCF7CC
:10BA500031F80599069A39200190FCF735F80198DC
:10BA6000FCF728F80599069A3A200290FCF72CF882
:10BA70000298FCF71FF80599069A3B200390FCF703
:10BA800023F80398FCF716F80599069A44200490C9
:10BA9000FCF71AF80498FCF70DF80599069A45206A
:10BAA0000790FCF711F80798FCF704F80AB080BD7E
:10BAB00080B582B04EF22900C0F6000047F604724D
:10BAC000C0F601020021019104F026FE019940F622
:10BAD0001052C2F2000210604EF2CD60C0F60000BB
:10BAE00047F68862C0F6010204F016FE02B080BD7F
:10BAF00080B59AB000201990189017901690159064
:10BB0000FFE70020149043F63000C4F20200016801
:10BB100041F002010160006800F0020014901498E6
:10BB2000FFE7FFE70020139043F63000C4F2020065
:10BB3000016841F040010160006800F0400013908E
:10BB40001398FFE7FFE70020129043F63000C4F29D
:10BB50000200016841F001010160006800F001008D
:10BB600012901298FFE7FFE70020119043F6300093
:10BB7000C4F20200016841F008010160006800F0B1
:10BB8000080011901198FFE7FFE70020109043F69E
:10BB90003000C4F20200016841F004010160006855
:10BBA00000F0040010901098FFE7FFE700200F90CE
:10BBB00043F63000C4F20200016841F080010160E8
:10BBC000006800F080000F900F98FFE7FFE700206B
:10BBD0000E9043F63000C4F20200016841F02001EB
:10BBE0000160006800F020000E900E98FFE741F61B
:10BBF0000040C4F2020002904FF4E0510191002293
:10BC00000C92FBF7A1FE0020C4F202000490102168
:10BC1000039101220692FBF797FE069A40F200403C
:10BC2000C4F2020007901146FBF78EFE019B0298BA
:10BC3000069A0C991593169217910221189115A93D
:10BC40000891FBF78DFC0498069A089915924FF419
:10BC50008813059316931792FBF782FC039B0498B5
:10BC6000069A08991593169217921892FBF778FC8A
:10BC7000059A06980899302315931692179040F666
:10BC80000000C4F20200FBF76BFC069A07980899C3
:10BC90001592169217921892FBF762FC0C9A0620E6
:10BCA000099005210B91FBF70FFF0998FBF702FFA5
:10BCB0000B990C9A0A200A90FBF706FF0A98FBF7EB
:10BCC000F9FE0B990C9A17200D90FBF7FDFE0D98CD
:10BCD000FBF7F0FE1AB080BD80B582B041F27C2047
:10BCE000C2F20000019043F20001C4F201010160C0
:10BCF0004FF48271416000218160C16001610122C5
:10BD000042614FF4007282611822C2610162416295
:10BD100081620A21C162FCF753FC18B1FFE7F9F711
:10BD200079FBFFE702B080BD80B588B000210091AB
:10BD3000079106910591049103910291019141F2BD
:10BD4000D420C2F2000044F20042C4F201020260B8
:10BD50004160816041F28732C26001618161FDF71B
:10BD60004FFD18B1FFE7F9F755FBFFE741F2D4208B
:10BD7000C2F20000FDF78AFE18B1FFE7F9F74AFBAF
:10BD8000FFE760200190002202920392059241F2A7
:10BD9000D420C2F2000001A9FDF7D6FD18B1FFE7DB
:10BDA000F9F738FBFFE741F2D420C2F20000FDF7BB
:10BDB00095FD08B080BD000080B582B041F21C3016
:10BDC000C2F20000019041F20001C4F201010160E1
:10BDD0004FF4E131416000218160C16001610C22BA
:10BDE00042618161C161FEF7E7F918B1FFE7F9F738
:10BDF00011FBFFE702B080BD80B582B041F2643034
:10BE0000C2F20000019044F60001C4F2000101609A
:10BE100048F2A061C0F2010141604FF4805181609D
:10BE20000021C1604FF4806202610C224261816195
:10BE3000C161FEF7C1F918B1FFE7F9F7EBFAFFE7C7
:10BE400002B080BD80B582B041F2AC30C2F20000D9
:10BE5000019041F20041C4F2010101604FF4E1316F
:10BE6000416000218160C16001610C2242618161F9
:10BE7000C161FEF7A1F918B1FFE7F9F7CBFAFFE7C7
:10BE800002B080BDFFE7FEE780B58AB00990089157
:10BE90000898417B807B40EA0120ADF81E0008989D
:10BEA000C17B007C40EA0120ADF81C000898417C71
:10BEB000807C40EA0120ADF81A0009980079FFF76C
:10BEC0008FFAADF8180009980079FFF72FFB8DED78
:10BED000050ABDF81E0000EE100AB8EEC00A9FED7C
:10BEE0006D1A80EE010A9FED6C1A20EE010A8DEDAD
:10BEF000040ABDF91C0000EE100AB8EEC00A8DED70
:10BF0000030ABDF91A00BDF91810484300EE100AE3
:10BF1000B8EEC00A9FED611A80EE010A8DED020AAB
:10BF200009988079C00700284CD0FFE7BDF81E00B3
:10BF30000999B1F84010401A01900198B0F5805F5E
:10BF400005DDFFE70999486C013848640AE001986B
:10BF500010F5805F05DAFFE70999486C0130486405
:10BF6000FFE7FFE7BDF81E000999A1F8400004981B
:10BF70000090099890ED110AB8EEC00A9FED461A9C
:10BF800020EE010A9DED001A30EE010A9DED051A22
:10BF900080EE010A80ED120A0999886C88609DED97
:10BFA000030A9DED051A80EE010A099880ED030A47
:10BFB0009DED020A9DED051A20EE010A099880ED1B
:10BFC000040A13E0099900204864BDF81E10099A7C
:10BFD000A2F8401009998864049809998860039828
:10BFE0000999C860029809990861FFE7FFE7099875
:10BFF00090ED020AB5EE400AF1EE10FA0ADAFFE718
:10C00000099890ED020A9FED241A30EE010A80EDA6
:10C01000020AECE7FFE7099890ED020A9FED1E1A6D
:10C02000B4EE410AF1EE10FA0ADBFFE7099890ED51
:10C03000020A9FED1B1A30EE010A80ED020AEAE7C0
:10C04000099890F82800C007C0B1FFE7099890ED63
:10C05000021A9FED110A30EE410A80ED020A09989A
:10C0600090ED030AB1EE400A80ED030A099890EDC5
:10C07000040AB1EE400A80ED040AFFE70898C07C8C
:10C0800000EE100AB8EE400A099880ED050A0AB0E1
:10C0900080BD00BF00000046DB0FC94000008046A5
:10C0A000DB0FC9C0FFE7FEE788B007900691059255
:10C0B000079800F0070004900498C0F107000528D5
:10C0C00003D3FFE70420019004E00498C0F10700C7
:10C0D0000190FFE70198039004980430062803D8E4
:10C0E000FFE70020009003E0049803380090FFE78A
:10C0F0000098029006980399012202FA01F1013991
:10C100000840029B984005999A40013A1140084323
:10C1100008B0704780B590B00E908DED0D0ACDED52
:10C120000C0A8DED0B1ACDED0A1A002028B9FFE795
:10C130000D9803F043FB58B943E00D980BF098FBC2
:10C1400041EC100B51EC100B03F01CFBC8B3FFE7E4
:10C15000002028B9FFE70C9803F030FB58B930E015
:10C160000C980BF085FB41EC100B51EC100B03F01D
:10C1700009FB30B3FFE7002028B9FFE70B9803F075
:10C180001DFB58B91DE00B980BF072FB41EC100B36
:10C1900051EC100B03F0F6FA98B1FFE7002028B934
:10C1A000FFE70A9803F00AFB78B90AE00A980BF057
:10C1B0005FFB41EC100B51EC100B03F0E3FA20B9DC
:10C1C000FFE70E9880690F9016E19DED0D0ADDEDF9
:10C1D0000C0A0E98406890ED071AF8F7E9FD8DED0E
:10C1E000090A9DED090A0E98406890ED001A20EEAC
:10C1F000010A8DED080A0E98406890ED000A9DED49
:10C200000C1A20EE010A8DED070A0E981C309DEDE8
:10C21000070AFEF7EDFA8DED060A0E980078014642
:10C22000019110B3FFE70198012804D0FFE70198BE
:10C23000022817D01CE09DED060A0E9890ED021A18
:10C2400090ED052A30EE420A9DED0A2AB4EE412A0D
:10C25000F1EE10FAC8BFB0EE421A80EE010A8DED81
:10C26000050A05E00B98059002E000200590FFE725
:10C2700009980E99086106980E994861002028B91E
:10C28000FFE7059803F09AFA70B90AE005980BF0F9
:10C29000EFFA41EC100B51EC100B03F073FA18B9E4
:10C2A000FFE700200590FFE79DED080A0E98406823
:10C2B00090ED011A90ED032A20EE010A9DED051A7A
:10C2C00021EE021A30EE410A8DED040A0E9890ED2F
:10C2D000030A9DED081A9DED0A2A21EE021A30EE9E
:10C2E000010A8DED030A9DED030A0E98406890ED5A
:10C2F000021A20EE010A8DED020A0E98406890EDB8
:10C30000020A9FED3F1AB4EE410AF1EE10FA39DD50
:10C31000FFE7002028B9FFE7039803F04FFA58B968
:10C320002FE003980BF0A4FA41EC100B51EC100B2A
:10C3300003F028FA28B3FFE79DED040A9DED021AE9
:10C3400030EE010AB0EEC00A0E98406890ED051A72
:10C35000B4EE410AF1EE10FA12DCFFE79DED030A9C
:10C36000B0EEC00A0E98406890ED041AB4EE410A8F
:10C37000F1EE10FA04DCFFE703980E99C860FFE7BE
:10C38000FFE7FFE79DED021A9DED040A30EE010A7A
:10C390008DED040A002028B9FFE7049803F00EFA97
:10C3A00058B925E004980BF063FA41EC100B51ECFE
:10C3B000100B03F0E7F9D8B1FFE70E98406890ED55
:10C3C000050A9FED0F1AB4EE410AF1EE10FA0BDDEB
:10C3D000FFE79DED040A0E984068D0ED050AF5F7D9
:10C3E000D9FB8DED040AFFE704980E998861FFE7F9
:10C3F0000E9880690F90FFE79DED0F0A10B080BD89
:10C40000BD37863580B586B004908DF80F108DED60
:10C41000020A0192049820B9FFE7FF208DF8170067
:10C42000B7E0002030B9FFE70198406803F0C6F993
:10C4300080B90BE0019840680BF01AFA41EC100B40
:10C4400051EC100B03F09EF920B9FFE7FF208DF8A7
:10C4500017009EE0002030B9FFE70198806803F0E4
:10C46000ADF980B90BE0019880680BF001FA41EC5E
:10C47000100B51EC100B03F085F920B9FFE7FF20FA
:10C480008DF8170085E0002030B9FFE70198C068FB
:10C4900003F094F980B90BE00198C0680BF0E8F95B
:10C4A00041EC100B51EC100B03F06CF920B9FFE7D5
:10C4B000FF208DF817006CE0002030B9FFE70198ED
:10C4C000006903F07BF980B90BE0019800690BF07B
:10C4D000CFF941EC100B51EC100B03F053F920B9DC
:10C4E000FFE7FF208DF8170053E0002030B9FFE789
:10C4F0000198406903F062F980B90BE00198406946
:10C500000BF0B6F941EC100B51EC100B03F03AF9BB
:10C5100020B9FFE7FF208DF817003AE00198049951
:10C5200048609DED021AB7EE000A80EE010A8DED1B
:10C53000000A002028B9FFE7009803F03FF958B936
:10C540000EE000980BF094F941EC100B51EC100B3D
:10C5500003F018F920B1FFE700980499886003E020
:10C56000FF208DF8170014E0049901F11C009DEDE7
:10C57000020A4968D1ED060AFEF796F99DF80F0008
:10C5800004990870049800F009F800208DF817004D
:10C59000FFE79DF9170006B080BD000080B584B0AC
:10C5A0000290029820B9FFE7FF208DF80F0013E0FA
:10C5B000029900200190C8600299086102994861BF
:10C5C0000299886102981C309FED050AFEF70AFA6D
:10C5D00001988DF80F00FFE79DF90F0004B080BDB2
:10C5E0000000000082B00090009820B9FFE7FF2013
:10C5F0008DF8070005E000990020C8608DF807005D
:10C60000FFE79DF9070002B070470000000000003E
:10C61000EFF30980BFF36F8F154B1A681EF0100FF0
:10C6200008BF20ED108A20E9F04F10602DE90900C5
:10C630004FF0500080F31188BFF34F8FBFF36F8F1F
:10C6400005F0C4FF4FF0000080F31188BDE8090039
:10C6500019680868B0E8F04F1EF0100F08BFB0EC82
:10C66000108A80F30988BFF36F8F704700BF00BF47
:10C670004C15002080B582B004F046F842F25C11FF
:10C68000C2F20001086020B9FFE7FE208DF8070024
:10C6900017E04CF2D172C0F6000200200090032196
:10C6A000F6F7C6FE009840F25461C2F20001087627
:10C6B00048610861C8608860486008608DF80700BC
:10C6C000FFE79DF9070002B080BD000080B584B08F
:10C6D000029001910092029820B9FFE7FE208DF8A8
:10C6E0000F0071E0009820B9FFE7FE208DF80F00E1
:10C6F0006AE00199022008700098F8F705FD00989B
:10C7000001998068C1F81B0000980199C068C1F8C0
:10C710001F00009801990068C1F813000098019962
:10C720004068C1F817000098B0F91000FEF738F81B
:10C73000019981F823000098B0F91200FEF730F853
:10C74000019981F824000098B0F91400FEF728F848
:10C75000019981F825000098B0F91600FEF720F83D
:10C76000019981F826000098B0F91800FEF718F832
:10C77000019981F827000098B0F91A00FEF710F827
:10C78000019981F828000098B0F91C00FEF708F81C
:10C79000019981F829000098B0F91E00FEF700F811
:10C7A000019981F82A000098B0F9160040F29F61C3
:10C7B000884205D1FFE700980199F8F773FCFFE77D
:10C7C00000208DF80F00FFE79DF90F0004B080BD39
:10C7D00080B542F25C10C2F200000068012103F053
:10C7E000B3FE80BD80B582B00020F6F7CBFD40F2ED
:10C7F0005461C2F200011922FDF7EAFE20B9FFE7F9
:10C8000000208DF8070003E0FF208DF80700FFE708
:10C810009DF9070002B080BD80B582B00190019AF9
:10C820000121084603F0E2FE0138B0FA80F0400929
:10C8300002B080BD80B582B001900198806B0090FD
:10C8400000980168486820F0030048600099486D2E
:10C8500040F0100048650099012081F851000098CF
:10C86000FBF784FE02B080BD80B582B001900198D4
:10C87000806B00900098FCF70BFA02B080BD0000BE
:10C8800080B582B001900198806B00900098FCF711
:10C8900031FF02B080BD000080B582B001900198E8
:10C8A000806B00900098FCF779FF02B080BD00001B
:10C8B00080B584B003900398806B0290FBF75CF81E
:10C8C000019003980068006800F48070B0F5807FE4
:10C8D00039D0FFE702980168486820F020004860DE
:10C8E0000298806868B9FFE702984068B0F5827FD7
:10C8F00007D1FFE702980168486820F0030048600C
:10C9000006E002980168486820F001004860FFE7EF
:10C910000298019A642100F0B5F820B1FFE702996E
:10C9200020204865FFE702990020C887029901206E
:10C9300081F851000298406D20B1FFE70298FBF7A3
:10C9400015FE04E0FFE70298FCF778F9FFE704B072
:10C9500080BD000080B584B003900398806B029086
:10C96000FBF70AF8019003980068006800F48070F3
:10C97000B0F5807F3BD0FFE702980168486820F05F
:10C980002000486002980168486820F00200486072
:10C990000298019A642100F0E7F830B1FFE70299AC
:10C9A000486D40F020004865FFE70298806870B944
:10C9B000FFE7FFE70020009002980068C068009041
:10C9C00002980068806800900098FFE7FFE70299EE
:10C9D0000020C8860299012081F851000298406D1C
:10C9E00020B1FFE70298FBF7C1FD04E0FFE70298E2
:10C9F000FCF75CFEFFE704B080BD000080B584B0AA
:10CA000003900398806B0290FAF7B6FF01900398A9
:10CA10000068006800F48070B0F5807F2BD0FFE7DD
:10CA200002980168486820F0200048600298019A46
:10CA3000642100F099F830B1FFE70299486D40F0A9
:10CA400020004865FFE702980168486820F003006D
:10CA5000486002990020C8860299C887029901207F
:10CA600081F851000298406D20B1FFE70298FBF772
:10CA70007DFD04E0FFE70298FCF766FEFFE704B0E7
:10CA800080BD000080B586B00490039102920498A6
:10CA90004068B0F5827F13D1FFE704988068B0F555
:10CAA000004F06D0FFE704988068B0F5806F07D18B
:10CAB000FFE704980168086820F040000860FFE77D
:10CAC00004984068B0F5827F31D1FFE70498806810
:10CAD000B0F5806F15D0FFE70498039B02996A4672
:10CAE00011608021002200F0BDF848B1FFE70499F1
:10CAF000486D40F02000486503208DF817002FE0B6
:10CB000014E00498039B02996A46116001210022F7
:10CB100000F0A8F848B1FFE70499486D40F0200004
:10CB2000486503208DF817001AE0FFE714E0049829
:10CB3000039B02996A4611600121002200F092F8DD
:10CB400048B1FFE70499486D40F020004865032094
:10CB50008DF8170004E0FFE700208DF81700FFE7CD
:10CB60009DF8170006B080BD80B586B00490039193
:10CB700002920498039B02996A46116002210122E5
:10CB800000F070F848B1FFE70499486D40F02000CC
:10CB9000486503208DF8170048E040F20000C2F21B
:10CBA000000000684AF6AB21CAF6AA21A0FB0110DA
:10CBB00000094DF68361C4F21B31A0FB0110800C0B
:10CBC0004FF47A714843019004984068B0F5827F31
:10CBD00015D1FFE70498039B02996A4611608021F2
:10CBE000002200F03FF848B1FFE70499486D40F09B
:10CBF0002000486503208DF8170017E012E0FFE7DA
:10CC0000019808B9FFE70CE0019801380190FFE7AF
:10CC1000049800688068C1B20020B0EBD11FEFD14A
:10CC2000FFE7FFE700208DF81700FFE79DF81700EA
:10CC300006B080BD82B000900098006843F2000109
:10CC4000C4F20101884204D1FFE700208DF80700FB
:10CC500003E002208DF80700FFE79DF8070002B00F
:10CC60007047000080B58AB0DDF830C008900791A9
:10CC70008DF81B20059305980190FAF77DFE02467A
:10CC800001980C99891A08440390FAF775FE0290EE
:10CC9000039840F20001C2F200010968C1F3CB31F0
:10CCA00048430490FFE708980068806807990840A7
:10CCB000401AB0FA80F040099DF81B1088425FD0FE
:10CCC000FFE705980130002859D0FFE7FAF754FE36
:10CCD0000299401A0399884204D2FFE7039800287A
:10CCE00042D1FFE708980168486820F0E0004860FA
:10CCF00008984068B0F5827F13D1FFE708988068F4
:10CD0000B0F5004F06D0FFE708988068B0F5806F57
:10CD100007D1FFE708980168086820F04000086024
:10CD2000FFE70898806AB0F5005F0FD1FFE7FFE7E3
:10CD300008980168086820F40050086008980168A5
:10CD4000086840F400500860FFE7FFE708990120F9
:10CD500081F85100FFE70899002081F85000FFE7B3
:10CD600003208DF827000FE0049818B9FFE7002092
:10CD7000039003E0049801380490FFE7FFE792E78F
:10CD800000208DF82700FFE79DF827000AB080BD3E
:10CD9000074B19680868B0E8F04F80F30988BFF3C3
:10CDA0006F8F4FF0000080F31188704700BF00BF05
:10CDB0004C15002080B56FF00400002102F090FDBA
:10CDC00080BD000084B003900291039890ED000AAA
:10CDD000029890ED001A30EE010A8DED010A9DEDEA
:10CDE000010AB7EE001AB4EE410AF1EE10FA1BDDAB
:10CDF000FFE79DED011AB7EE000A80EE010A8DED06
:10CE0000000A9DED001A039890ED000A20EE010A39
:10CE100080ED000A9DED001A029890ED000A20EEC8
:10CE2000010A80ED000AFFE704B07047000000002F
:10CE300080B586B004908DF80F10049828B9FFE7EC
:10CE40000020CBF68070059065E00498806900783A
:10CE50000146009120B1FFE70098012805D009E0C4
:10CE60000020C4F24820029007E00020C4F2C8303D
:10CE7000029002E0002005904DE0049882699DF840
:10CE80000F1002EB810292ED020A90ED671A20EE7C
:10CE9000010A00EB011090ED091A30EE410A10EE84
:10CEA000100A0AF0E5FC41EC100B51EC100B9FED61
:10CEB0001C0B52EC103BD20F62F3DF7141EC100BF4
:10CEC00051EC100B09F0AEFD01909DED010A9DEDB6
:10CED000021AB4EE410AF1EE10FA12DAFFE79DED04
:10CEE000010A20EE000A9DED021A21EE011A80EEE1
:10CEF000011AB7EE000A30EE410A049880ED460AA6
:10CF000004E004990020C1F81801FFE70498D0F864
:10CF100018010590FFE79DED050A06B080BD00BF32
:10CF2000000000000000000080B586B0049003916E
:10CF3000049828B1FFE70498B0F8200120B9FFE772
:10CF4000FF208DF817004FE0049890ED000A90ED57
:10CF5000471A30EE410A8DED020A0498D0ED490AD5
:10CF600090ED680A9FED221AF7F722FF8DED010A76
:10CF70009DED020A0498806990ED062AB7EE001A2A
:10CF800081EE021AB4EE410AF1EE10FA28DBFFE757
:10CF900003988078C00718B3FFE79DED010AB7EE4C
:10CFA000001AB4EE410AF1EE10FA19DCFFE7049919
:10CFB0000868C1F81C01049901F5D070896991EDE8
:10CFC000050AB8EE400ADFED0A0A80EE800AF7F79C
:10CFD000ADFE0499B1F820010138A1F82001FFE766
:10CFE00000208DF81700FFE79DF9170006B080BDFF
:10CFF000DB0FC94084B002908DED010A029820B980
:10D00000FFE7FF208DF80F001DE00298806900788F
:10D010000146009120B1FFE70098012808D00EE0FA
:10D02000029944F20000C4F29C50C1F89C0106E051
:10D0300002990020C4F27A50C1F89C01FFE7002059
:10D040008DF80F00FFE79DF90F0004B07047000056
:10D0500080B586B004900391049818B1FFE7039857
:10D0600020B9FFE7FF208DF8170035E0F6F734F917
:10D070000AF053FC00EE100A9FED191A8DED011A0B
:10D0800080EE010A049880ED000AF6F725F9049A6B
:10D0900002929368D268C01A91410AF03EFC9DED5D
:10D0A000011A0146029800EE101A80EE010A80ED86
:10D0B000040AF6F711F90A460499CA6088600498D0
:10D0C0009FED080AFFF796FF0498039900F0E8F82F
:10D0D00000208DF81700FFE79DF9170006B080BD0E
:10D0E000002474490000694380B58AB00890079114
:10D0F0008DED060A089858B1FFE7079840B1FFE7A1
:10D100009DED060AB5EE400AF1EE10FA04DCFFE7E9
:10D11000FF208DF82700BFE0079840688DF81700C2
:10D12000079808998861F5F7E7F900200490FFE770
:10D1300004989DF81710884248DAFFE70798049989
:10D1400001EB810100EB41002C30FEF717FA089843
:10D150000499C1EB011100EB810000F5D2709DED47
:10D16000060A079901F1700201210391FFF74AF9BC
:10D1700003990898049AC2EB021200EB820000F5B2
:10D1800043709DED060A079A9032FFF73BF9089924
:10D19000049801EB401000F2EC409DED060A89690D
:10D1A000D1ED4C0AFDF780FB0899049801EB401083
:10D1B00000F2AC509DED060A8969D1ED4D0AFDF7EC
:10D1C00073FBFFE7049801300490B1E707986830DB
:10D1D000FEF7D4F90898806990F86C000146029136
:10D1E000E0B1FFE7029801282FD1FFE7089800F28D
:10D1F00074409DED060A079901F1F00201210191A9
:10D20000FFF700F90199089800F596609DED060A70
:10D21000079A02F58872FFF7F5F81AE0089800F20D
:10D2200074409DED060A079901F1B00201210091B9
:10D23000FFF7E8F80099089800F596609DED060A5A
:10D24000079AD032FFF7DEF803E0FC208DF82700C4
:10D2500022E0089901F26C609DED060A8969D1ED22
:10D260004E0AFDF721FB089901F28C609DED060A3C
:10D270008969D1ED4F0AFDF717FB08990020C1F825
:10D280002C01C1F82801C1F82401C1F82001C1F81E
:10D290001C018DF82700FFE79DF927000AB080BD2B
:10D2A00080B584B002900191029820B9FFE7FF2079
:10D2B0008DF80F00C2E00298806990F82000C00746
:10D2C000002800F0AB80FFE7029890F8DC000146F0
:10D2D0000091032800F29C800099DFE801F0022011
:10D2E0005471029890ED240A9FED581A80EE010ABD
:10D2F000806990ED091AB4EE410AF1EE10FA09DDE9
:10D30000FFE70299012081F8DC0002990868C1F862
:10D31000D800FFE70298019900F090F97DE00298AB
:10D3200090ED240A9FED491A80EE010A806990ED84
:10D33000091AB4EE410AF1EE10FA05DAFFE7029994
:10D34000002081F8DC0068E0029890ED000A90ED82
:10D35000361A30EE410A806990ED0A1AB4EE410A9D
:10D36000F1EE10FA09DBFFE70299012081F8D40001
:10D370000299022081F8DC004FE0FFE70298019952
:10D3800000F05CF949E002990020A1F82001029820
:10D3900090ED490A816991ED051AB8EE412A9FED99
:10D3A000291A81EE021A30EE010A80ED680A02990C
:10D3B000032081F8DC0002990868C1F8D800FFE773
:10D3C0000298019900F03AF9029890ED000A90ED68
:10D3D000361A30EE410A9FED1C1AB4EE410AF1EE06
:10D3E00010FA14DBFFE7029890ED240A9FED171A5C
:10D3F00080EE010AB3EE041AB4EE410AF1EE10FA1F
:10D4000005DAFFE70299002081F8DC00FFE704E07D
:10D410000299002081F8DC00FFE70BE00299002070
:10D4200081F8DC00029981F8D4000298019900F09B
:10D4300005F9FFE700208DF80F00FFE79DF90F00C9
:10D4400004B080BDDB0FC9C09A99993E00007A44B0
:10D4500080B586B00490049820B9FFE7FF208DF8CE
:10D4600017005AE00498806940688DF80F0000208A
:10D470000290FFE702989DF80F1088422FDAFFE72D
:10D4800004980299C1EB011100EB810000F5D27004
:10D49000FFF784F804980299C1EB011100EB8100B9
:10D4A00000F54370FFF77AF80498029900EB4110F9
:10D4B00000F2EC409FED1B0A8DED010AFDF792FA98
:10D4C0009DED010A0498029900EB411000F2AC5066
:10D4D000FDF788FAFFE7029801300290CAE7049846
:10D4E00000F27440FFF75AF8049800F59660FFF7D1
:10D4F00055F8049800F26C609FED0A0A8DED000A61
:10D50000FDF770FA9DED000A049800F28C60FDF7BB
:10D5100069FA00208DF81700FFE79DF9170006B0A3
:10D5200080BD00BF0000000080B584B0029002986A
:10D5300020B9FFE7FF208DF80F0034E002988069E2
:10D5400040688DF8070000200090FFE700989DF8E4
:10D550000710884219DAFFE702980099C1EB011120
:10D5600000EB810000F5D270FFF73CF802980099BB
:10D57000C1EB011100EB810000F54370FFF732F8B9
:10D58000FFE7009801300090E0E7029800F2744055
:10D59000FFF728F8029800F59660FFF723F80020BF
:10D5A0008DF80F00FFE79DF90F0004B080BD00006B
:10D5B00084B00290029820B9FFE7FF208DF80F0099
:10D5C00038E00298806940688DF8070000200090DC
:10D5D000FFE700989DF8071088421EDAFFE70298DF
:10D5E000009900EB81010020C1F830010299009AF6
:10D5F00001EB8201C1F848010299009A01EB820116
:10D60000C1F860010299009A01EB8201C1F878012A
:10D61000FFE7009801300090DBE702990020C1F895
:10D6200090010299C1F894010299C1F898018DF80E
:10D630000F00FFE79DF90F0004B0704780B598B068
:10D6400016901591169818B1FFE7159820B9FFE7C5
:10D65000FF208DF85F004EE31698806940688DF8D2
:10D6600053001698007F48BBFFE700201390FFE7A8
:10D6700013989DF8531088420FDAFFE716988069D7
:10D68000139901EB810100EB41002C30FEF706F805
:10D69000FFE7139801301390EAE716988069683025
:10D6A000FDF7FCFF169890ED490A80ED680A40F2FC
:10D6B0009450C2F2000080ED000AF9E2169890F84A
:10D6C000D0000146099150B1FFE70998012800F008
:10D6D000AB80FFE70998022800F0DC81E2E200203D
:10D6E0001290FFE712989DF85310884251DAFFE735
:10D6F00016981299C1EB011100EB810000F5D27070
:10D70000FEF770FF1699129AC2EB021001EB80002F
:10D7100000F5D27001EB8202D2ED3E0AD1ED041A7F
:10D720009FEDE31AB0EE410AFEF7F4FC1698129949
:10D7300000EB810080ED4C0A1698129900EB8101F4
:10D74000D1F83001C1F860011699129A01EB42102C
:10D7500000F2AC5001EB820191ED580AFDF748F858
:10D760001698129900EB810080ED5E0A169988697F
:10D77000129A02EB820300EB43002C3001EB820192
:10D7800091ED5E0AFDF796FFFFE7129801301290C7
:10D79000A8E7169901F2744040F29452C2F20002D6
:10D7A00092ED000AD1ED041AD1ED490A9FEDC01A9D
:10D7B0008DED081AFEF7AEFC9DED081A169880ED67
:10D7C000640A169901F59660D1ED041AD1ED4B0A61
:10D7D00091ED640AFEF79EFC169880ED650A169995
:10D7E00001F28C6091ED650AFDF702F8169880ED64
:10D7F000660A16998869683091ED660AFDF75AFF46
:10D8000015984078C00770B1FFE71698FFF720FE23
:10D810001698FFF789FE1698FFF7CAFE16990120A1
:10D8200081F8D000FFE742E200201190FFE7119855
:10D830009DF85310884280F2AD80FFE7169880690A
:10D84000119901EB810100EB410090F8340001389F
:10D850008DF84300169881699DF8432001EB820101
:10D8600091ED020A90ED671A20EE010A9FED911AE0
:10D8700080EE010A8DED0F0A16989DF84410FFF70F
:10D88000D7FA8DED0E0A1699119AC2EB021001EB30
:10D89000800000F5D2709DED0F0A01EB8202D2EDFF
:10D8A0003E0AD1ED041A9FED821A8DED061AFEF79D
:10D8B00031FC9DED061A1698119900EB810080ED60
:10D8C0004C0A9DED0E0A8DED070A1699119BC3EBCC
:10D8D000031001EB800000F5437001F1E002D1F884
:10D8E00018C003EB830E0CEB4E0C9CF834C002EB1B
:10D8F0008C0C9CED0B0A02EB8302D2ED060AD1EDF3
:10D90000041AFEF707FCB0EE401A9DED070A20EE60
:10D91000010A1698119900EB810080ED520A1698C1
:10D92000119900EB810101F5987001F5A471FFF7E1
:10D9300049FA1698119900EB810090ED4C0A90ED90
:10D94000521A30EE010A80ED580A1699119A01EB2D
:10D95000421000F2AC5001EB820191ED580AFCF745
:10D9600047FF1698119900EB810080ED5E0A169929
:10D970008869119A02EB820300EB43002C3001EB23
:10D98000820191ED5E0AFDF795FEFFE711980130E7
:10D9900011904CE7169901F2744040F29452C2F291
:10D9A000000292ED000AD1ED041AD1ED490A9FED73
:10D9B000D41A8DED051AFEF7ADFB9DED051A1698EC
:10D9C00080ED640A169901F59660D1ED041AD1ED47
:10D9D0004B0A91ED640AFEF79DFB169880ED650AEF
:10D9E000169901F28C6091ED650AFCF701FF16981B
:10D9F00080ED660A16998869683091ED660AFDF730
:10DA000059FE15984078C00758B9FFE71698FFF7F8
:10DA10001FFD1698FFF7CCFD1699002081F8D00065
:10DA200037E041F25440C2F200000078C00778BBF2
:10DA3000FFE715988078C00750B3FFE716990220DA
:10DA400081F8D0001698007F01460491012808D083
:10DA5000FFE70498022809D0FFE7049803280BD0B9
:10DA600010E016990120A1F8200110E016998869AC
:10DA7000C069A1F820010AE0169941F60A20A1F830
:10DA8000200104E016990020A1F82001FFE7FFE73C
:10DA9000FFE70CE116981599FFF746FA00200D9064
:10DAA000FFE70D989DF85310884280F2B18003E0A3
:10DAB0000000000000C0DA45169880690D9901EB5E
:10DAC000810100EB410090F8340001388DF83300FB
:10DAD000169881699DF8332001EB820191ED020ACD
:10DAE00090ED671A20EE010A9FED861A80EE010A7A
:10DAF0008DED0B0A16989DF83410FFF799F98DED0E
:10DB00000A0A16990D9AC2EB021001EB800000F58B
:10DB1000D2709DED0B0A01EB8202D2ED3E0AD1EDEF
:10DB2000041A9FED771A8DED021AFEF7F3FA9DEDB8
:10DB3000021A16980D9900EB810080ED4C0A9DEDBC
:10DB40000A0A8DED030A16990D9BC3EB031001EB36
:10DB5000800000F5437001F1E002D1F818C003EB3A
:10DB6000830E0CEB4E0C9CF834C002EB8C0C9CED3D
:10DB70000B0A02EB8302D2ED060AD1ED041AFEF77E
:10DB8000C9FAB0EE401A9DED030A20EE010A16987C
:10DB90000D9900EB810080ED520A16980D9900EB6B
:10DBA000810101F5987001F5A471FFF70BF9169842
:10DBB0000D9900EB810090ED4C0A90ED521A30EE79
:10DBC000010A80ED580A16990D9A01EB421000F2F5
:10DBD000AC5001EB820191ED580AFCF709FE169852
:10DBE0000D9900EB810080ED5E0A169988690D9A07
:10DBF00002EB820300EB43002C3001EB820191ED3C
:10DC00005E0AFDF757FDFFE70D9801300D9048E7DC
:10DC1000169901F27440D1ED041AD1ED490A91ED43
:10DC2000680A9FED371A8DED011AFEF773FA9DED24
:10DC3000011A169880ED640A169901F59660D1EDE7
:10DC4000041AD1ED4B0A91ED640AFEF763FA1698B7
:10DC500080ED650A169901F28C6091ED650AFCF77A
:10DC6000C7FD169880ED660A16998869683091EDAF
:10DC7000660AFDF71FFD15988078C00788B9FFE791
:10DC80001699012081F8D0001698D0F8240140F2AE
:10DC90009451C2F20001086016990020A1F82001F9
:10DCA000FFE704E01699002081F8D000FFE7FFE7C6
:10DCB000169880692C30FDF7C3FA16988069406881
:10DCC000052806D3FFE7169880695430FDF7B8FAA7
:10DCD000FFE7169880696830FDF7B2FA15988078EA
:10DCE00000F0010041F25441C2F20001087000202E
:10DCF0008DF85F00FFE79DF95F0018B080BD00BFA1
:10DD00000000000000C0DA4583B001908DF80310D8
:10DD1000019820B9FFE7FF208DF80B0007E09DF880
:10DD200003000199087700208DF80B00FFE79DF9AB
:10DD30000B0003B07047000080B588B006900698CD
:10DD400020B9FFE7FF208DF81F0062E10698806987
:10DD500040688DF8170000200490FFE704989DF8B4
:10DD60001710884280F29680FFE706988069049930
:10DD700001EB810100EB41002C30FDF729FD0698F5
:10DD80008069049901EB810100EB41002C30FDF723
:10DD900091FB03900398A0B1FFE70698049900EB6C
:10DDA0000111DDF80CC0DCF82C00DCF83020DCF8C8
:10DDB0003430DCF838C0C1F82CC08B624A6208628B
:10DDC000FFE70699049A01EB421000F2EC4001EBE8
:10DDD000021191ED090AFCF70BFD0698049900EB7E
:10DDE000810080ED380A0698049900EB810090EDDF
:10DDF000380A9FED8C1A80EE010A80ED3E0A0698E3
:10DE0000049900EB810090ED3E0AB7EE001AB4EEE3
:10DE1000410AF1EE10FA09DDFFE70698049900EBDC
:10DE200081014FF07E50C1F8F800FFE70698049991
:10DE300000EB810090ED3E0ABFEE001AB4EE410AFD
:10DE4000F1EE10FA0ADAFFE70698049900EB810177
:10DE50000020CBF68070C1F8F800FFE7069901F1C9
:10DE6000E000049A00EB820393ED061A896902EB45
:10DE7000820201EB420191F8341000EB810090ED39
:10DE80000B0A30EE010A80ED0B0AFFE7049801301F
:10DE9000049063E701200290FFE70298012819DC53
:10DEA000FFE70698029900EB810090ED440A9DF887
:10DEB000171001EE101AB8EEC11A80EE010AB0EE8A
:10DEC000001A80EE010A80ED440AFFE70298013053
:10DED0000290E2E7069880696830FDF779FC0698C1
:10DEE00000F18001019180696830FDF7E3FA014695
:10DEF00001985022F2F7B5FA0698816991ED040A6B
:10DF000090ED321A20EE010A80ED490AFFE70698EB
:10DF100090ED490AB5EE400AF1EE10FA0ADAFFE791
:10DF2000069890ED490A9FED3D1A30EE010A80ED0A
:10DF3000490AECE7FFE7069890ED490A9FED371A8A
:10DF4000B4EE410AF1EE10FA0ADBFFE7069890ED15
:10DF5000490A9FED331A30EE010A80ED490AEAE7DB
:10DF6000069890F8A800C00750B1FFE7069890ED1A
:10DF7000491A9FED2A0A30EE410A80ED490AFFE76F
:10DF8000069901F26C6091ED230AFCF731FC0698CA
:10DF900080ED4A0A069890ED230A40F26C31C2F2F5
:10DFA000000191ED001A80EE010A80ED4B0A0698FF
:10DFB00090ED4B0AB7EE001AB4EE410AF1EE10FAFA
:10DFC00006DDFFE706994FF07E50C1F82C01FFE710
:10DFD000069890ED4B0ABFEE001AB4EE410AF1EE3E
:10DFE00010FA07DAFFE706990020CBF68070C1F837
:10DFF0002C01FFE7069890ED090A90ED0D1A30EE1E
:10E00000410A00F2AC6080ED000A00208DF81F008C
:10E01000FFE79DF91F0008B080BD00BFDB0FC940BE
:10E02000DB0FC9C000C0DA4580B582B0019002F0B4
:10E030006BFB02F01FFC02B080BD000080B582B017
:10E04000009000980138B0F1807F03D3FFE70120F2
:10E05000019019E0009801384EF21401CEF200014F
:10E0600008604FF0FF300F2101F018FC4EF218014C
:10E07000CEF20001002008604EF21002CEF2000243
:10E08000072111600190FFE7019802B080BD0000F8
:10E0900080B5F9F777FC05F08DFC012803D0FFE788
:10E0A00004F0A4FBFFE780BD80B594B008A8302140
:10E0B000F2F711FA00200790069005900490039063
:10E0C000FFE70020029043F64000C4F2020001681E
:10E0D00041F080510160006800F080500290029889
:10E0E000FFE7FFE70020019047F20000C4F20000C4
:10E0F000016841F480410160006800F480400190B3
:10E100000198FFE7012008904FF480300990022029
:10E110000E904FF480010F9106211091A8211191CA
:10E1200012900420139008A8F9F7C0FE18B1FFE779
:10E13000F7F770F9FFE70F2003900220049000200A
:10E1400005904FF4A05006904FF48050079003A81C
:10E150000521F9F7DBFC18B1FFE7F7F75BF9FFE7FB
:10E1600014B080BD4EF68851CEF20001086840F42C
:10E17000700008607047000083B00290019102981F
:10E180000068009002980021C4F20101884225D065
:10E19000FFE70298B0F1804F20D0FFE7029840F2ED
:10E1A0000041C4F20001884218D0FFE7029840F60F
:10E1B0000001C4F20001884210D0FFE7029840F647
:10E1C0000041C4F20001884208D0FFE7029840F203
:10E1D0000041C4F2010188420AD1FFE7009820F013
:10E1E0007000009001984168009808430090FFE794
:10E1F00002980021C4F20101884255D0FFE702983D
:10E20000B0F1804F50D0FFE7029840F20041C4F2D5
:10E210000001884248D0FFE7029840F60001C4F2AE
:10E220000001884240D0FFE7029840F60041C4F266
:10E230000001884238D0FFE7029840F20041C4F262
:10E240000101884230D0FFE7029844F20001C4F295
:10E250000101884228D0FFE7029844F20041C4F24D
:10E260000101884220D0FFE7029844F60001C4F281
:10E270000101884218D0FFE7029841F60001C4F27C
:10E280000001884210D0FFE7029841F60041C4F235
:10E290000001884208D0FFE7029842F20001C4F270
:10E2A000000188420AD1FFE7009820F440700090F6
:10E2B0000198C168009808430090FFE7009820F09B
:10E2C000800001994969084300900198806802998B
:10E2D000C862019800680299886202980021C4F21D
:10E2E0000101884208D0FFE7029840F20041C4F2E1
:10E2F0000101884205D1FFE701980069029908638E
:10E30000FFE70299086840F00400086002990120C4
:10E31000486100980299086003B0704784B0039088
:10E3200002910192029800F01F01012088400090A4
:10E33000009A0399086A904308620198029901F0D3
:10E340001F0100FA01F20399086A1043086204B041
:10E350007047000085B0049003910498006A019012
:10E360000499086A20F0010008620498406800904F
:10E37000049880690290029820F070000290029840
:10E3800020F003000290039801680298084302906D
:10E39000019820F0020001900398816801980843D9
:10E3A000019004980021C4F20101884208D0FFE7DF
:10E3B000049840F20041C4F2010188420ED1FFE707
:10E3C000019820F0080001900398C1680198084363
:10E3D0000190019820F004000190FFE704980021CB
:10E3E000C4F20101884208D0FFE7049840F20041DE
:10E3F000C4F20101884213D1FFE7009820F4807035
:10E400000090009820F400700090039841690098F3
:10E410000843009003988169009808430090FFE743
:10E4200000980499486002980499886103984068AC
:10E430000499486301980499086205B07047000088
:10E4400085B0049003910498006A01900499086AC9
:10E4500020F01000086204984068009004988069D9
:10E460000290029820F4E0400290029820F440705C
:10E47000029003980168029840EA012002900198F6
:10E4800020F02000019003988168019840EA011073
:10E49000019004980021C4F20101884208D0FFE7EE
:10E4A000049840F20041C4F2010188420FD1FFE715
:10E4B000019820F0800001900398C168019840EA1B
:10E4C00001100190019820F040000190FFE70498AE
:10E4D0000021C4F20101884208D0FFE7049840F20D
:10E4E0000041C4F20101884215D1FFE7009820F4F1
:10E4F00080600090009820F40060009003984169CB
:10E50000009840EA8100009003988169009840EAF1
:10E5100081000090FFE700980499486002980499F0
:10E520008861039840680499886301980499086297
:10E5300005B0704785B0049003910498006A01907B
:10E540000499086A20F4807008620498406800907A
:10E550000498C0690290029820F07000029002981E
:10E5600020F003000290039801680298084302908B
:10E57000019820F40070019003988168019840EAA6
:10E580000120019004980021C4F20101884208D0C2
:10E59000FFE7049840F20041C4F2010188420FD124
:10E5A000FFE7019820F4006001900398C16801988A
:10E5B00040EA01200190019820F480600190FFE77B
:10E5C00004980021C4F20101884208D0FFE70498B2
:10E5D00040F20041C4F20101884215D1FFE70098E2
:10E5E00020F480500090009820F400500090039890
:10E5F0004169009840EA01100090039881690098F1
:10E6000040EA01100090FFE70098049948600298E2
:10E610000499C861039840680499C86301980499F3
:10E62000086205B07047000085B00490039104981B
:10E63000006A01900499086A20F4805008620498E6
:10E64000406800900498C0690290029820F4E0406D
:10E650000290029820F4407002900398016802989A
:10E6600040EA01200290019820F4005001900398A4
:10E670008168019840EA0130019004980021C4F2B9
:10E680000101884208D0FFE7049840F20041C4F23B
:10E69000010188420BD1FFE7009820F480400090F0
:10E6A00003984169009840EA81100090FFE70098C4
:10E6B0000499486002980499C861039840680499D5
:10E6C000086401980499086205B0704780B586B067
:10E6D000059001F025FC4EF62900C0F6000047F633
:10E6E000F852C0F601020021029102F015F80299D9
:10E6F00042F2B402C2F20002049210604EF631609F
:10E70000C0F6000047F6AC62C0F6010202F004F861
:10E710000299049A50604EF6F120C0F6000047F6C8
:10E720001C62C0F6010201F0F7FF0299049A9060A2
:10E730004EF61940C0F6000047F64062C0F60102EE
:10E7400001F0EAFF0299049AD0604EF64150C0F6FB
:10E75000000047F66462C0F6010201F0DDFF029995
:10E76000049A10614EF60170C0F6000047F6D062C0
:10E77000C0F6010201F0D0FF029A0499486102201C
:10E7800003900A2101F0BAFC029A049B0146039807
:10E7900099612F2101F0B2FC029A049B0146039873
:10E7A000D961202101F0AAFC029A049B014603983A
:10E7B00019620C21019101F0A1FC0199029ADDF886
:10E7C00010C003460398CCF82C3001F097FC029A55
:10E7D000049B014603989962182101F08FFC029A6C
:10E7E000049B014603981963102101F087FC029AEB
:10E7F000049B014603985963042101F07FFC029AAF
:10E80000049B014603989963032101F077FC049966
:10E81000C86301F0DBFB01F077FF02F02BF806B0D4
:10E8200080BD00000000000080B58EB00D9001F0AA
:10E830004FFB08F0EFFB41EC100B9FEDA71B53ECD7
:10E84000112B51EC100B08F0DBF941EC100B51ECE3
:10E85000100B08F09BFB0C9000200A9001F0B4FA1A
:10E8600001F022FB0B9040F2F850C2F20000099038
:10E8700040F20801C2F20001F3F70CFA0998F3F72D
:10E88000E1F940F2E050C2F2000041F24441C2F22C
:10E890000001F1F741FF0A9941F20440C2F2000081
:10E8A00040F24C32C2F200029FED8D0AFDF7AAFD44
:10E8B0000A98F4F7F1FB0A9841F62131C0F60101FC
:10E8C000F4F7D2FA0A98F4F77FFAFFE70C990B985D
:10E8D00008440B90F3F7CEFBF3F79CF9F3F7AAF992
:10E8E000F3F7C2F9F3F7CEF901F01AFB40F2F85052
:10E8F000C2F200000890F3F791FA0898F3F708FBCA
:10E9000040F24060C2F200000078012865D1FFE7C4
:10E9100040F2F851C2F2000191ED071A40F6E070A2
:10E92000C2F2000090ED000A30EE010A80ED000A0C
:10E9300091ED081A90ED010A30EE010A80ED010A0E
:10E9400091ED091A90ED020A30EE010A80ED020AFB
:10E9500040F23E60C2F2000001880131018000886F
:10E9600041F28831884237DBFFE740F6E070C2F2BF
:10E97000000090ED000A9FED5B1A80EE010A40F264
:10E980000801C2F2000181ED000A90ED010A80EE5B
:10E99000010A81ED010A90ED020A80EE010A81ED83
:10E9A000020A40F24062C2F200020020107040F2FF
:10E9B000F850C2F200000790F3F76CF90798F3F7EC
:10E9C00041F940F2E050C2F2000041F24441C2F28B
:10E9D0000001F1F7A1FEFFE7FFE740F24060C2F25D
:10E9E0000000007801281BD0FFE740F2F850C2F287
:10E9F000000000F1100100F11C0240F2E050C2F2F0
:10EA00000000069041F24443C2F20003F1F7D0FF48
:10EA1000069941F2F830C2F20000F1F7CFFDFFE7AE
:10EA200001F0D4FA41F2F831C2F200010291086813
:10EA30004A688B6840F6C871C2F2000101914B61CF
:10EA40000A61C86040F2F852C2F2000252F81C0F8C
:10EA500004920860506892688A60486042F2B4008C
:10EA6000C2F200000390006B01F02AFC01990398A8
:10EA7000006B002305931A4601F0C0FB0398806ADF
:10EA800001F01EFC0499059B0398806A1A4601F068
:10EA9000B5FB0398C06A01F013FC0299059B03982B
:10EAA000C06A1A4601F0AAFB0498D0ED030A41F2AD
:10EAB0000440C2F200009FED0C0ADFED0C1AB0EE2C
:10EAC000611AFDF727FB0598F4F746FA0B9801F059
:10EAD00095F9FBE600BF00BF0000000000407F404A
:10EAE0000000FA4300409C45000020420000000066
:10EAF00080B590B00F9001F0EBF908F08BFA41EC83
:10EB0000100B9FED411B53EC112B51EC100B08F037
:10EB100077F841EC100B51EC100B08F037FA0E901F
:10EB2000002001F051F901F0BFF90D90F6F78EF9D0
:10EB3000014640F27060C2F200009FED350A00F01D
:10EB40000FFFFFE70E990D9808440D9042F2B400B4
:10EB5000C2F200000490C06A40F27061C2F200018B
:10EB6000029101F24441002303931A4601F066FA30
:10EB70000299039B0498806A01F22C411A4601F025
:10EB80005DFA0299039B0498806BFC311A4601F0F0
:10EB900055FA039B0498006A40F6B041C2F20001A6
:10EBA0001A4601F04BFA80B9FFE740F27060C2F2FA
:10EBB00000000190F6F70CF801980D9A40F6B0416C
:10EBC000C2F20001F4F778FE12E0002000900C90F1
:10EBD0000B900A90099008900790069005900D9A66
:10EBE00040F27060C2F2000005A9F4F765FEFFE78D
:10EBF00040F27060C2F20000F5F728F80D9801F0BD
:10EC0000FDF89FE700BF00BF0000000000407F400C
:10EC10000000FA430000000080B588B0079001F0C2
:10EC200057F908F0F7F941EC100B9FED431B53EC3B
:10EC3000112B51EC100B07F0E3FF41EC100B51ECE2
:10EC4000100B08F0A3F90690002001F0BDF801F0C8
:10EC50002BF9059040F69040C2F2000040F6485172
:10EC6000C2F20001F4F704FDFFE706990598084495
:10EC7000059001F055F942F2B400C2F20000C069FB
:10EC800041F6CC11C2F2000100231A4601F0D6F978
:10EC900078B9FFE740F69040C2F2000041F6CC118F
:10ECA000C2F2000140F64852C2F20002F4F7EEFC54
:10ECB000FFE740F69040C2F20000009041F6CC1110
:10ECC000C2F2000140F64852C2F20002019241F63F
:10ECD000FB13C2F200030293F4F72AFC01F076F969
:10ECE00042F2B400C2F200000490006A01F0E8FAB7
:10ECF00000990498006A002303931A4601F07EFAF3
:10ED00000498406B01F0DCFA0199039B0498406B76
:10ED10001A4601F073FA0498C06B01F0D1FA029917
:10ED2000039B0498C06B1A4601F068FA059801F03D
:10ED300065F89AE700BF00BF0000000000407F4078
:10ED400080B588B0079001F0C3F808F063F941EC92
:10ED5000100B9FED331B53EC112B51EC100B07F0F4
:10ED60004FFF41EC100B51EC100B08F00FF906901F
:10ED7000002001F029F801F097F80590F6F766F801
:10ED800000F1D00140F65850C2F200009FED260A73
:10ED9000F6F744FDFFE7069905980844059042F20E
:10EDA000B400C2F200000290006B40F6B071C2F2F3
:10EDB00000010091002301931A4601F03FF90099E8
:10EDC00040F65850C2F200000490F6F7C7FE019BCF
:10EDD0000298406B40F6D041C2F2000103911A46FE
:10EDE00001F02CF90498F6F753FE0298806B01F0BD
:10EDF00067FA019B04990298806B01F50A711A4623
:10EE000001F0FCF903990498F6F708FB0498F6F76B
:10EE10009DFD059800F0F2FFBDE700BF00BF00BFF9
:10EE20000000000000407F400000FA4300000000A6
:10EE300080B586B0059001F04BF808F0EBF841EC96
:10EE4000100B9FED2D1B53EC112B51EC100B07F009
:10EE5000D7FE41EC100B51EC100B08F097F8049022
:10EE6000002000F0B1FF01F01FF80390FDF702FC55
:10EE7000FFE70499039808440390FDF7B3FC1420BE
:10EE8000FDF7CAFC78B1FFE740F61450C2F200006B
:10EE900040F6E041C2F2000140F62852C2F2000200
:10EEA000FDF714FC12E040F61450C2F2000040F6E8
:10EEB000E041C2F200010291F6F7CAF8029940F669
:10EEC0002850C2F20000F6F7EDF8FFE742F2B40076
:10EED000C2F200000190C06901F0F2F90198C06926
:10EEE00040F6E041C2F2000100231A4601F086F923
:10EEF000039800F083FFBCE70000000000407F4063
:10EF000080B586B0059000F0E3FF08F083F841EC8F
:10EF1000100B9FED251B53EC112B51EC100B07F040
:10EF20006FFE41EC100B51EC100B08F02FF8049021
:10EF3000002000F049FF00F0B7FF0390F5F786FFCF
:10EF400000F5E47141F60020C2F200009FED180ABE
:10EF5000FEF7CAF8FFE7049903980844039042F2C9
:10EF6000B400C2F20000C06B42F2B001C2F2000174
:10EF7000019100231A4601F061F841F60020C2F227
:10EF800000000290FEF7D8FE019902980978FEF77A
:10EF9000BBFE01990298FEF75BF8039800F02EFF84
:10EFA000D9E700BF00BF00BF0000000000407F4065
:10EFB0000000FA4380B582B001900198806B009008
:10EFC00000990020C8850098FAF79EFE02B080BD27
:10EFD00080B584B00390002002900398806B01906C
:10EFE000019800684069C0B2C0090290019890F889
:10EFF000410021280AD1FFE7029838B1FFE70199C3
:10F000000020C884019800F013F9FFE70198006818
:10F010004069C0F380100290019890F842002228C5
:10F020000AD1FFE7029838B1FFE701990020C885AF
:10F03000019800F09FF8FFE70199486C40F010003C
:10F0400048640198FAF760FE04B080BD80B586B0D0
:10F0500005900598806B0490059800680068C005CD
:10F0600000285AD4FFE704990020C885FFE7FFE78E
:10F070000498006850E8030F20F480700390FFE7C5
:10F0800003990498026842E803100028F0D1FFE7D2
:10F09000FFE7FFE7FFE70498006850E8050F20F05E
:10F0A00001000290FFE702990498026842E8051007
:10F0B0000028F0D1FFE7FFE7FFE7FFE704980068CB
:10F0C00050E8050F20F040000190FFE701990498F7
:10F0D000026842E805100028F0D1FFE7FFE7049935
:10F0E000202081F842000498006B012814D1FFE72A
:10F0F000FFE7FFE70498006850E8030F20F01000D6
:10F100000090FFE700990498026842E80310002885
:10F11000F0D1FFE7FFE7FFE7FFE70499002048632E
:10F120000498006B012805D1FFE70498818DFAF758
:10F13000E5FD03E00498FBF777FAFFE706B080BD32
:10F1400080B582B001900198806B009000990120F9
:10F1500048630098006B012806D1FFE70098818D75
:10F160004908FAF7CBFD03E00098FBF787FAFFE7C1
:10F1700002B080BD84B00390FFE7FFE7039800680A
:10F1800050E8030F20F490700290FFE70299039873
:10F19000026842E803100028F0D1FFE7FFE7FFE72D
:10F1A000FFE70398006850E8050F20F00100019088
:10F1B000FFE701990398026842E805100028F0D1A2
:10F1C000FFE7FFE70398006B012814D1FFE7FFE793
:10F1D000FFE70398006850E8030F20F0100000904C
:10F1E000FFE700990398026842E803100028F0D175
:10F1F000FFE7FFE7FFE70399202081F8420003992A
:10F200000020086304B0704780B582B00190019877
:10F210000168C86820F04000C8600199202081F88A
:10F2200041000198FBF754FA002002B080BD0000B5
:10F2300082B00190FFE7FFE70198006850E8030FF4
:10F2400020F0C0000090FFE700990198026842E8B2
:10F2500003100028F0D1FFE7FFE70199202081F893
:10F26000410002B07047000082B000900098006832
:10F2700044F60001C4F20001884204D1FFE70020F7
:10F280008DF8070010E00098006841F20041C4F2D8
:10F290000101884204D1FFE701208DF8070003E057
:10F2A00003208DF80700FFE79DF8070002B07047C4
:10F2B00080B586B00490002003900290049890F8E6
:10F2C0004200222840F0A080FFE704988068B0F553
:10F2D000805F13D1FFE70498006978B9FFE70498CD
:10F2E000806A02900498006840686FF35F2002997A
:10F2F00008800499886A0230886223E00498806A52
:10F30000039004988068B0F5805F08D0FFE7049808
:10F31000806850B9FFE70498006930B9FFE70498A6
:10F32000006840680399087007E004980068406826
:10F3300000F07F0003990870FFE70499886A0130A4
:10F340008862FFE70499C88D0138C8850004002849
:10F3500056D1FFE704980168C86820F02000C86013
:10F3600004980168C86820F48070C8600498016837
:10F37000486920F0010048610499202081F842008A
:10F380000499002048630498006B012830D1FFE7FE
:10F39000049900200863FFE7FFE70498006850E83D
:10F3A000030F20F010000190FFE701990498026814
:10F3B00042E803100028F0D1FFE7FFE70498006857
:10F3C0000068C00600280ED5FFE7FFE70020009088
:10F3D00004980068006800900498006840680090F5
:10F3E0000098FFE7FFE70498818DFAF787FC03E0B8
:10F3F0000498FBF719F9FFE700208DF8170007E0E4
:10F4000000208DF8170003E002208DF81700FFE7B9
:10F410009DF8170006B080BD80B586B005900598B0
:10F420000068006920F44050059A1168D2681043C2
:10F430000861059988680B694A69C96918431043CE
:10F440000843049005980068C06849F20C6188433D
:10F450000499084305990968C860059800684069DF
:10F4600020F44070059A116892691043486105982C
:10F47000006841F20001C4F20101884209D0FFE7AF
:10F480000598006841F20041C4F20101884204D1AC
:10F49000FFE7F8F785FC039003E0F8F76FFC0390B3
:10F4A000FFE70598C069B0F5004F29D1FFE7039841
:10F4B0001921A0FB0101059A1368029353685A00B1
:10F4C000DB0FF0F7F3FE0299864648F21F53C5F2B0
:10F4D000EB13AEFB0320420910014FF0640C02FB5A
:10F4E0001CEC322202EBCC02A2FB0332F82303EA2B
:10F4F000521300EB4300C2F342121044886026E02E
:10F5000003981921A0FB0101059A13680193536820
:10F510009A009B0FF0F7CAFE0199844648F21F52E9
:10F52000C5F2EB12ACFB02304309642003FB10CCA4
:10F53000322000EB0C10A0FB0202F02000EA521077
:10F5400000EB0310C2F3431210448860FFE706B0DB
:10F5500080BD000080B58AB008900791ADF81A20F0
:10F56000079808998862BDF81A0008998885089953
:10F5700000204864089A222182F842100899CA6B38
:10F580004FF24D01C0F60001D1630899CA6B4FF2EA
:10F590004111C0F6000111640899CA6B4EF6D17191
:10F5A000C0F60001D1640899C96B086507A80590E9
:10F5B00008980168C06B0431059A1268BDF81A30CA
:10F5C000F7F7FAFE58B1FFE7089910204864089948
:10F5D000202081F8420001208DF827004EE0FFE74F
:10F5E000002004900898006800680490089800685B
:10F5F000406804900498FFE708980069A0B1FFE70D
:10F60000FFE7FFE70898006850E8030F40F48070B8
:10F610000390FFE703990898026842E80310002866
:10F62000F0D1FFE7FFE7FFE7FFE7FFE70898006893
:10F6300050E8050F40F001000290FFE7029908989A
:10F64000026842E805100028F0D1FFE7FFE7FFE776
:10F65000FFE70898006850E8050F40F0400001906F
:10F66000FFE701990898026842E805100028F0D1E8
:10F67000FFE7FFE700208DF82700FFE79DF8270050
:10F680000AB080BD83B00190019890F84100212814
:10F690003AD1FFE701988068B0F5805F13D1FFE7AA
:10F6A0000198006978B9FFE70198006A0090009816
:10F6B00000886FF35F200199096848600199086A22
:10F6C0000230086208E0019A106A411C1162007859
:10F6D000019909684860FFE70199C88C0138C8841E
:10F6E000000468B9FFE701980168C86820F080004D
:10F6F000C86001980168C86840F04000C860FFE732
:10F7000000208DF80B0003E002208DF80B00FFE7CE
:10F710009DF80B0003B0704780B541F21C30C2F277
:10F720000000FAF71BFB80BD80B582B041F2643067
:10F73000C2F200000190FAF711FB0198F3F742FEC4
:10F7400002B080BD80B582B041F2AC30C2F20000A0
:10F750000190FAF703FB0198F3F734FE02B080BD85
:10F76000FFE7FEE782B041EC100B8DED000B019836
:10F77000C0F30A5040F2FF71401A18BF012002B0D6
:10F780007047000082B041EC100B8DED000B01982A
:10F79000C0F30A5040F2FF71401A18BF012002B0B6
:10F7A0007047000081B000EE100A00900098C0F38E
:10F7B000C750FF3818BF012001B0704781B000EE7C
:10F7C000100A00900098C0F3C750FF3818BF0120FE
:10F7D00001B0704784B041EC100B8DED020B039A21
:10F7E00000200021CFF6E071B1EB420F019006D16D
:10F7F000FFE70298B0FA80F040090190FFE7019816
:10F8000000F0010004B0704781B000EE100A0090D3
:10F8100000994FF0807000EB4100B0FA80F0400991
:10F8200001B0704781B08DF803009DF903000028F6
:10F8300012D4FFE79DF9031001F01F020120904050
:10F840004A094EF28011CEF2000141F82200BFF3C6
:10F850004F8FBFF36F8FFFE701B0704781B08DF816
:10F8600003009DF9030000280ED4FFE79DF9031063
:10F8700001F01F02012090404A094EF20011CEF221
:10F88000000141F82200FFE701B070474EF60C502E
:10F89000CEF200000068C0F30220704782B08DF8FD
:10F8A000070000919DF9070000280AD4FFE700989F
:10F8B00000019DF907104EF20042CEF2000288547A
:10F8C0000BE0009800019DF8071001F00F014EF6C3
:10F8D0001452CEF200028854FFE702B070470000D5
:10F8E00082B08DF8070000919DF9070000280AD426
:10F8F000FFE7009800019DF907104EF20042CEF29A
:10F90000000288540BE0009800019DF8071001F0F8
:10F910000F014EF61452CEF200028854FFE702B0F7
:10F920007047000083B00290029800F0070000903A
:10F930004EF60C51CEF200010868019001984FF686
:10F94000FF02104001900198009A40EA0220002234
:10F95000C0F2FA52104301900198086003B070475A
:10F9600080B58EB00C900B918DED0A0A0C9858B1B1
:10F97000FFE70B9840B1FFE79DED0A0AB5EE400A9C
:10F98000F1EE10FA04DCFFE7FF208DF8370018E1F4
:10F990000B980C99C1F860040C99032008720C991B
:10F9A000D1F86004D0F8C800C1F818060C99D1F855
:10F9B0006004D0F8CC00C1F81C06F2F79DFD0020D1
:10F9C0000990FFE7099803280EDCFFE70C98D0F8B0
:10F9D0006004099900EBC1008030FBF7CFFDFFE721
:10F9E000099801300990EDE700200890FFE708989A
:10F9F00003280EDCFFE70C98D0F86004089900EBB0
:10FA0000C100A030FBF7BAFDFFE70898013008906D
:10FA1000EDE747F6F463C0F60103186859689A6881
:10FA2000DB6807930692059104900C990498059A57
:10FA3000069BDDF81CC0C1F85CC4C1F85834C1F89D
:10FA40005424C1F8500400200390FFE703980328D2
:10FA500016DCFFE70C990398C0EB001001EB800067
:10FA600000F538709DED0A0AD1F8601401F14002EA
:10FA70000021FCF7C7FCFFE7039801300390E5E79E
:10FA800000200290FFE70298032825DCFFE70C998D
:10FA90000298C0EB001001EB800000F5F8709DEDBE
:10FAA0000A0AD1F8602401210191FCF7ABFC01990D
:10FAB0000C9A0298C0EB001002EB800000F58070F9
:10FAC0009DED0A0AD2F860242032FCF79BFCFFE788
:10FAD000029801300290D6E70C9901F574709DED03
:10FAE0000A0AD1F8601401F160020121FCF78AFCD6
:10FAF0000C9800F284409DED0A0AF3EE040ACDED65
:10FB0000000AFAF7D1FEDDED000A0C9800F2A440DD
:10FB10009DED0A0AFAF7C8FEDDED000A0C9800F226
:10FB2000C4409DED0A0AFAF7BFFEDDED000A0C980D
:10FB300000F2E4409DED0A0AFAF7B6FEDDED000A98
:10FB40000C9800F204509DED0A0AFAF7ADFEDDEDC7
:10FB5000000A0C9800F224509DED0A0AFAF7A4FE60
:10FB6000DDED000A0C9800F244509DED0A0AFAF708
:10FB70009BFEDDED000A0C9800F264509DED0A0A30
:10FB8000FAF792FEDDED000A0C9800F284509DED2C
:10FB90000A0AFAF789FEDDED000A0C9800F2A4507B
:10FBA0009DED0A0AFAF780FEDDED000A0C9800F2DE
:10FBB000C4509DED0A0AFAF777FE00208DF8370051
:10FBC000FFE79DF937000EB080BD000082B08DEDDB
:10FBD000010ACDED000A01980099C90F61F3DF70A9
:10FBE00001909DED010A02B07047000080B588B019
:10FBF000069006980190019858B9FFE74FF0500021
:10FC000080F31188BFF36F8FBFF34F8F0790FFE72B
:10FC1000FEE7019841F24C51C2F2000109688842A6
:10FC200004D1FFE700208DF8170056E002F092F8AB
:10FC300001984069049041F25450C2F200000068FB
:10FC4000039041F25C50C2F200000068029002F0A2
:10FC5000ADF804980399884205D0FFE7049802990B
:10FC6000884204D1FFE702208DF8170034E00498A1
:10FC700043F21C11C2F20101884218D1FFE701983A
:10FC8000806A78B9FFE7019890F85800012804D1FC
:10FC9000FFE702208DF8170003E003208DF817001E
:10FCA000FFE703E002208DF81700FFE713E0049858
:10FCB00043F23011C2F20101884203D0FFE70498F9
:10FCC00020B9FFE704208DF8170003E001208DF82C
:10FCD0001700FFE7FFE7FFE7FFE79DF8170008B011
:10FCE00080BD000086B08DED050ACDED040A8DEDD6
:10FCF000031A02909DED030A9DED041A30EE410AAD
:10FD00008DED010A049800909DED050A9DED001A05
:10FD100030EE410A029901208840013801EE100AB4
:10FD2000B8EEC11A20EE010A9DED011A80EE010A1B
:10FD3000BDEEC00A10EE100A06B0704780B582B062
:10FD400000200190F7F72CFEFEF7AEF9FBF7D0FE8E
:10FD5000FBF750FEFBF7FEFDFBF724FEFBF7BCFFB5
:10FD6000FCF74AF8FCF76EF8FBF7DEFFFCF724F827
:10FD700000F0B2F8FBF79CFE00F0FEF8FFE7FEE7AC
:10FD800085B08DED040ACDED030A8DED021ACDED9F
:10FD9000011A8DED002A9DED040A9DED033A30EE27
:10FDA000430A9DED002A9DED011A32EE412A20EE14
:10FDB000020A9DED022A32EE432A80EE020A30EE5C
:10FDC000010A05B07047000080B584B00290EFF3DF
:10FDD00005800390039820B1FFE76FF005000190C4
:10FDE00009E000200190029820B1FFE7029802F09C
:10FDF0002BF9FFE7FFE7019804B080BD80B586B01E
:10FE00000490EFF305800590059820B1FFE76FF0AF
:10FE1000050001901BE00020019003F0E7FD039036
:10FE200004980399401A0290029858B1FFE702998A
:10FE30000020B0EBD17F05D1FFE7029903A802F0C3
:10FE40003BF903E06FF003000190FFE7FFE7019843
:10FE500006B080BD80B582B003F0ACFD01460091D4
:10FE600058B1FFE7009801280AD0FFE70098022860
:10FE700007D1FFE70220019012E0032001900FE07C
:10FE8000FFE740F27050C2F200000068012803D181
:10FE9000FFE70120019002E000200190FFE7FFE76B
:10FEA000019802B080BD000080B582B0EFF30580FC
:10FEB0000190019820B1FFE703F0A2FD009003E05C
:10FEC00003F094FD0090FFE7009802B080BD0000B1
:10FED0004FF47A707047000082B0EFF30580019014
:10FEE000019820B1FFE76FF00500009014E040F2A8
:10FEF0007050C2F20000006848B9FFE740F270514C
:10FF0000C2F20001012008600020009003E04FF0E1
:10FF1000FF300090FFE7FFE7009802B07047000055
:10FF200080B584B0EFF305800390039820B1FFE71C
:10FF30006FF0050002901BE003F03CFD01460191CB
:10FF400040B1FFE7019801280CD0FFE70198022893
:10FF500003D008E00120029009E002F02FFB00200E
:10FF6000029004E0FFE74FF0FF300290FFE7FFE769
:10FF7000029804B080BD000080B582B0EFF3058028
:10FF80000190019820B1FFE76FF00500009019E0A3
:10FF900040F27050C2F20000006801280DD1FFE766
:10FFA000FCF708FF40F27051C2F200010220086025
:10FFB00002F094FA0020009003E04FF0FF30009030
:10FFC000FFE7FFE7009802B080BD000080B584B075
:10FFD000EFF305800390039820B1FFE76FF0050071
:10FFE000029027E003F0E6FC0146019140B1FFE7F3
:10FFF0000198012818D0FFE70198022811D014E0D9
:020000040801F1
:100000000120029003F0C0FF012809D0FFE703F0B0
:10001000D1FC20B9FFE74FF0FF300290FFE7FFE788
:1000200007E00020029004E0FFE74FF0FF3002906D
:10003000FFE7FFE7029804B080BD000080B588B0FC
:100040000690059104920393069802900020019077
:10005000EFF305800790079868B3FFE7029830B187
:10006000FFE7059818B1FFE7039820B1FFE76FF0AD
:10007000030001901EE000200090029805996A4656
:1000800003F000F8012804D0FFE76FF002000190B0
:100090000FE0009860B1FFE74EF60451CEF2000188
:1000A0004FF080500860BFF34F8FBFF36F8FFFE7B3
:1000B000FFE7FFE71FE0029818B1FFE7059820B9B6
:1000C000FFE76FF00300019014E002980599039A8E
:1000D00002F0EAFE01280CD0FFE7039820B1FFE709
:1000E0006FF00100019003E06FF002000190FFE764
:1000F000FFE7FFE7FFE7019808B080BD80B588B053
:1001000006900591049200200390EFF3058007907C
:10011000079800286ED1FFE7069800286AD0FFE70D
:100120000598002866D0FFE74FF0FF300290049852
:1001300068B3FFE704988068A0B1FFE70498C0683F
:1001400050280FD3FFE70498006958B1FFE70498DF
:1001500040690699059A5143884203D3FFE701207D
:10016000029013E00498806878B9FFE70498C068AB
:1001700058B9FFE70498006938B9FFE70498406967
:1001800018B9FFE700200290FFE7FFE702E0002038
:100190000290FFE7029801280ED1FFE70698059923
:1001A000049A93681269EE464FF0000CCEF800C036
:1001B00002F0A2FB03900AE0029838B9FFE7069824
:1001C0000599002202F05EFB0390FFE7FFE703982A
:1001D00078B1FFE7049820B1FFE704980068019028
:1001E00002E000200190FFE70398019901F0D0FEA2
:1001F000FFE7FFE7039808B080BD000080B588B036
:10020000069005918DF81320039306980290002024
:100210000190EFF305800790079868B3FFE7029815
:1002200030B1FFE7059818B1FFE7039820B1FFE769
:100230006FF0030001901EE00023009302980599DF
:100240006A4602F055FD012804D0FFE76FF0020076
:1002500001900FE0009860B1FFE74EF60451CEF236
:1002600000014FF080500860BFF34F8FBFF36F8FD6
:10027000FFE7FFE7FFE720E0029818B1FFE70598E6
:1002800020B9FFE76FF00300019015E0029805998F
:10029000039A002302F016FC01280CD0FFE7039814
:1002A00020B1FFE76FF00100019003E06FF0020062
:1002B0000190FFE7FFE7FFE7FFE7019808B080BD87
:1002C00080B584B0029002980190EFF3058003900E
:1002D000039820B1FFE76FF0050000900DE0019852
:1002E00020B9FFE76FF00300009005E000210091C6
:1002F000019802F089FBFFE7FFE7009804B080BD9A
:1003000080B586B004900391049820F0010002901B
:10031000049800F00100009000200190EFF30580A8
:100320000590059820B1FFE76FF00500019033E0DC
:10033000029820B9FFE76FF0030001902BE00098CE
:10034000A0B1FFE70298039903F036F801280CD01A
:10035000FFE7039820B1FFE76FF00100019003E091
:100360006FF002000190FFE7FFE713E002980399A6
:1003700002F00CFF01280CD0FFE7039820B1FFE743
:100380006FF00100019003E06FF002000190FFE7C1
:10039000FFE7FFE7FFE7FFE7019806B080BD000039
:1003A00080B588B0069000200590EFF30580079097
:1003B0000798002840F08580FFE7069820B1FFE706
:1003C00006984068049002E000200490FFE79DF842
:1003D0001000C00718B1FFE70120039002E00020E1
:1003E0000390FFE7049800F00800082868D0FFE7B2
:1003F0004FF0FF3002900698C8B1FFE7069880687A
:1004000040B1FFE70698C068502803D3FFE70120FA
:1004100002900BE00698806838B9FFE70698C0683C
:1004200018B9FFE700200290FFE7FFE702E0002095
:100430000290FFE70298012812D1FFE7039838B134
:10044000FFE706988168042002F002FA059006E0B2
:1004500006988168012002F0FBF90590FFE711E0A2
:10046000029870B9FFE7039828B1FFE7042002F073
:10047000DBF9059004E0012002F0D6F90590FFE7D2
:10048000FFE7FFE7059878B1FFE7069820B1FFE79F
:1004900006980068019002E000200190FFE70598AF
:1004A000019901F075FDFFE7059840B1FFE703985A
:1004B00028B1FFE7059840F001000590FFE7FFE74E
:1004C000FFE7059808B080BD80B586B00490049819
:1004D00020F001000390049800F00100019000203A
:1004E0000290EFF305800590059820B1FFE76FF0CB
:1004F0000500029024E0039820B9FFE76FF00300A5
:1005000002901CE0019858B1FFE7039802F096FCB6
:10051000012804D0FFE76FF002000290FFE70DE032
:100520000398002319461A4602F0CCFA012804D099
:10053000FFE76FF002000290FFE7FFE7FFE7FFE74A
:10054000029806B080BD000080B58AB0089007917F
:1005500008980690069830B1FFE79DF81F00000646
:10056000002804D5FFE76FF0030005903BE04FF053
:10057000FF300590EFF305800990099820B3FFE75D
:1005800000230393049306980799EC4604AACCF839
:100590000020012203F022F9039A069869460A60B6
:1005A00005AB114603F01AF9049860B1FFE74EF667
:1005B0000451CEF200014FF080500860BFF34F8F1E
:1005C000BFF36F8FFFE70DE0069807990122002324
:1005D000029303F047F8029A069805AB114603F020
:1005E00041F8FFE7FFE705980AB080BD80B58CB001
:1005F0000A9009910892EFF305800B900B9820B1B7
:10060000FFE76FF0050007907AE09DF82B000006E9
:10061000002804D5FFE76FF0030007906FE09DF816
:1006200024008007002803D5FFE70020059002E0A2
:100630000A980590FFE7002007900898029003F0C1
:10064000D5F90490FFE70599029B002006AA03F064
:10065000C9FA0190019801283FD1FFE70A9907984C
:100660000840079006990798084307909DF82400D2
:10067000C00780B1FFE70A9907980840884201D176
:10068000FFE73BE0089820B9FFE76FF00200079012
:1006900034E0FFE70EE00A980799084201D0FFE72F
:1006A0002CE0089820B9FFE76FF00200079025E0E2
:1006B000FFE7FFE703F09AF90499401A03900398C3
:1006C0000299884203D9FFE70020029004E00399D1
:1006D0000298401A0290FFE70BE0089820B9FFE764
:1006E0006FF00200079003E06FF001000790FFE752
:1006F000FFE7FFE701980028A5D1FFE7FFE7FFE745
:1007000007980CB080BD000080B582B003F048F9B6
:100710000190019802B080BDB0B58EB00B900A91E7
:10072000099200200690EFF305800D900D980028A7
:1007300040F09980FFE70B98002800F09480FFE7D5
:100740008020079018200590002008904FF0FF307F
:100750000490099800284DD0FFE70998006820B15F
:10076000FFE7099800680890FFE70998806920B1C1
:10077000FFE7099880690590FFE7059848B1FFE712
:100780000598382805D8FFE709980079C00718B1FF
:10079000FFE700200C9069E00998406928B1FFE765
:1007A0000998406980080790FFE70998806880B140
:1007B000FFE70998C0685C280BD3FFE70998006938
:1007C00038B1FFE70998406918B1FFE701200490AC
:1007D0000FE00998806858B9FFE70998C06838B9F0
:1007E000FFE70998006918B9FFE700200490FFE7C8
:1007F000FFE702E000200490FFE70498012817D1EA
:10080000FFE70B980899079A0A9BDDF814C0DDF8FA
:1008100024E0DEF80850DEF81040EE46CEF808502E
:10082000CEF80440CEF800C002F0B4FE069019E005
:100830000498B0B9FFE70B980899BDF81C200A9BF3
:10084000DDF814C0EE4606ACCEF80440CEF800C089
:1008500002F050FE012803D0FFE700200690FFE7DA
:10086000FFE7FFE7FFE706980C90FFE70C980EB054
:10087000B0BD000080B586B0049004980390EFF3FB
:1008800005800590059820B1FFE76FF00500029004
:100890001CE0039820B9FFE76FF00300029014E01A
:1008A0000398FFF7A3F98DF807009DF807000428C7
:1008B00006D0FFE700200290039801F087FC03E0D8
:1008C0006FF002000290FFE7FFE7FFE7029806B033
:1008D00080BD00000000000080B586B08DED040BE7
:1008E0009DED040B9FED261B04F0CAFA51EC100B92
:1008F0009FED250B53EC102B06F018FC41EC100B70
:100900008DED000B9DED040B9FED211B04F0B8FA5B
:1009100051EC100B9FED200B53EC102B06F006FC56
:100920009DED001B41EC100B51EC110B53EC102B07
:1009300006F0AAF841EC100B8DED020B0498059916
:100940009FED170B53EC102B06F0F0FB9DED021BF7
:1009500041EC100B51EC110B53EC102B06F094F8FA
:1009600041EC100B51EC100B9FED0F0B53EC102BC7
:1009700006F08AF841EC100B06B080BD00BF00BF46
:1009800000000000000008405F09A4C4AEEDDA3F9B
:100990000000000000000040412B3064752B02C0B5
:1009A0004CFDBCA948851040BC5CC47762D6FFBF33
:1009B00080B584B00390029143F24410C2F201006A
:1009C0000068009041F24C50C2F200000068043010
:1009D00001F0F2F808B9FFE700E0FFE70398013003
:1009E00080B9FFE7029868B1FFE741F24C50C2F2CC
:1009F00000000068011D43F21C10C2F2010001F06A
:100A000081F93DE00098039908440190019841F272
:100A10004C51C2F20001096848600198009988426F
:100A20000ED2FFE741F25C50C2F20000006841F2D2
:100A30004C51C2F200010968043101F02DF91EE0A9
:100A400041F25450C2F20000006841F24C51C2F22F
:100A500000010968043101F01FF9019843F2A8016F
:100A6000C2F201010968884207D2FFE7019843F208
:100A7000A801C2F20101086000E0FFE7FFE7FFE71D
:100A800004B080BD80B582B0019001F063F942F6F8
:100A90007C11C2F2010108680130086041F24C503B
:100AA000C2F20000006898B9FFE7019841F24C518A
:100AB000C2F20001086042F67C10C2F20100006838
:100AC000012803D1FFE700F021FB00E0FFE71CE075
:100AD00043F21010C2F201000068A0B9FFE741F232
:100AE0004C50C2F200000068C06A0199C96A88428D
:100AF00007D8FFE7019841F24C51C2F200010860AB
:100B000000E0FFE700E0FFE7FFE742F68810C2F2EF
:100B10000100016801310160006801994864019891
:100B2000C06A42F68C11C2F201010968884208D9F4
:100B3000FFE70198C06A42F68C11C2F20101086019
:100B4000FFE70199C86A00EB800241F26450C2F2EB
:100B5000000000EB8200043101F0D4F801F026F926
:100B600043F21010C2F201000068C8B1FFE741F281
:100B70004C50C2F200000068C06A0199C96A8842FC
:100B80000CD2FFE74EF60451CEF200014FF0805038
:100B90000860BFF34F8FBFF36F8F00E0FFE700E007
:100BA000FFE702B080BD000080B584B001F0D2F84C
:100BB00043F24810C2F201000068002840D1FFE76C
:100BC00043F24800C2F20100029001F045F843F2FE
:100BD0005C00C2F20100039001F03EF80299039814
:100BE00041F25052C2F20002116041F26051C2F271
:100BF0000001086069460020086041F25542C2F2D7
:100C0000000241F2F843C2F200030A20102101F071
:100C100073FE014643F24810C2F201000160006811
:100C200060B1FFE743F24810C2F20100006847F6E6
:100C30003971C0F6010101F0ABF900E0FFE700E017
:100C4000FFE701F0B3F804B080BD000080B582B0CA
:100C5000FFE742F68010C2F20100006808B3FFE728
:100C600001F078F843F23010C2F20100C068C068A9
:100C700001900198043000F09FFF42F67C11C2F20F
:100C8000010108680138086042F68011C2F20101D2
:100C900008680138086001F089F8019800F08CF8C4
:100CA000D7E702B080BD000080B582B0019000910E
:100CB0000198006CB8B1FFE70199C8680A6C10444C
:100CC000C86001988168C068884204D3FFE7019931
:100CD0000868C86000E0FFE70098019AD168126CCC
:100CE000EFF77AFBFFE702B080BD000080B586B069
:100CF000059004910392002002900598806B01906A
:100D00000598006C78B9FFE70598006848B9FFE7D7
:100D10000598806802F0D2FF029005990020886053
:100D200000E0FFE741E00398B8B9FFE7059A0499AE
:100D30005068126CEFF750FB059948680A6C104434
:100D40004860059948688968884204D3FFE7059997
:100D50000868486000E0FFE726E0059A0499D0683B
:100D6000126CEFF739FB0599C8680A6C801AC860E5
:100D700005980168C068884206D2FFE7059988682F
:100D80000A6C801AC86000E0FFE70398022809D1C6
:100D9000FFE7019820B1FFE701980138019000E0DA
:100DA000FFE700E0FFE7FFE7FFE701980130059963
:100DB0008863029806B080BD80B582B0009000982C
:100DC00090F8590040B9FFE70098006B01F014F863
:100DD000009801F011F81CE0009890F859000128E3
:100DE00004D1FFE7009801F007F811E0009890F8AF
:100DF000590002280BD0FFE74FF0500080F3118814
:100E0000BFF36F8FBFF34F8F0190FFE7FEE7FFE760
:100E1000FFE702B080BD000082B001900198406AF7
:100E200038B1FFE70198006B0068C0F1380000900E
:100E300002E000200090FFE7009802B07047000039
:100E400082B0019041F25050C2F200000068006888
:100E5000B0FA80F04009019908600198006848B92B
:100E6000FFE741F25050C2F200000068C06800681D
:100E7000009002E000200090FFE7009802B0704769
:100E800084B04FF48030009042F67010C2F200003F
:100E900001909DF80400400788B1FFE701980730F2
:100EA0000190019820F007000190019A42F670111C
:100EB000C2F200010098891A08440090FFE70198E7
:100EC0000290029943F21410C2F201000160002165
:100ED00041600298009A10440190019808380190EE
:100EE000019820F007000190019A41F25850C2F297
:100EF000000002600268516002681160029903916B
:100F00000199039A891A516000680399086003984F
:100F1000406843F2A401C2F20101086003984068EE
:100F200043F29C01C2F20101086043F27001C2F277
:100F300001014FF00040086004B0704780B582B0F6
:100F40000190FFE7FFF782FE41F26450C2F2000019
:100F5000006802280CD3FFE74EF60451CEF20001E0
:100F60004FF080500860BFF34F8FBFF36F8F00E0EA
:100F7000FFE7E7E780B582B00190019868B1FFE72D
:100F8000019800238360019803600198C360019871
:100F900019461A4601F096FD00E0FFE702B080BD59
:100FA00080B584B0DDF818C00390029101928DF8ED
:100FB0000330029818B9FFE70698006003E0019833
:100FC00006990860FFE703980699C8630298069996
:100FD00008640698012101F017FD9DF803000699A9
:100FE00081F84C0004B080BD80B588B0DDF834C015
:100FF000DDF830C0DDF82CC0DDF828C00690059182
:10100000049203930C98006B04998900A522EFF7D2
:101010005AFA0C98006B049900EB81000438029096
:10102000029820F0070002909DF80800400758B190
:10103000FFE74FF0500080F31188BFF36F8FBFF3CD
:101040004F8F0790FFE7FEE70598F8B1FFE7002014
:101050000190FFE701980F2813D8FFE70598019A40
:10106000805C0C99114481F8340005980199405C2A
:1010700008B9FFE705E0FFE7FFE7019801300190BD
:10108000E8E70C99002081F8430004E00C99002067
:1010900081F83400FFE70A98382803D3FFE73720A8
:1010A0000A9000E0FFE70A980C99C8620A980C9928
:1010B000C8640C990020009008650C98043000F07A
:1010C000E3FD0C98183000F0DFFD00980C990961E1
:1010D0000A99C1F138010C9A91610C9949620C99F5
:1010E00048650C9981F8580002980699039A00F017
:1010F000E7FC0C9908600B9820B1FFE70C980B995E
:10110000086000E0FFE708B080BD000080B584B053
:1011100000200390FFE70398372810D8FFE70398D3
:1011200000EB800141F26450C2F2000000EB81004C
:1011300000F092FDFFE7039801300390EBE743F2E4
:101140007400C2F20100019000F086FD43F28800B5
:10115000C2F20100029000F07FFD43F2BC00C2F237
:10116000010000F079FD43F23010C2F2010000F0FE
:1011700073FD43F21C10C2F2010000F06DFD0199F5
:10118000029841F25452C2F20002116041F25C51E5
:10119000C2F20001086004B080BD000083B002907C
:1011A00043F21410C2F201000190FFE701980068B9
:1011B0000299884205D2FFE7FFE701980068019095
:1011C000F4E7019800900098019949680844029951
:1011D000884209D1FFE702984268019948681044A3
:1011E00048600198029000E0FFE7029800900098A4
:1011F00002994968084401990968884220D1FFE7AB
:101200000198006841F25851C2F200010968884211
:101210000DD0FFE7019800684268029948681044C1
:1012200048600198006800680299086007E041F290
:101230005850C2F20000006802990860FFE704E01D
:101240000198006802990860FFE7019802998842B6
:1012500004D0FFE702980199086000E0FFE703B0BF
:101260007047000080B586B0059004910392029308
:101270000020019004980599486005980061049841
:101280000399884216D8FFE703980299401A0599F6
:101290008969884203D3FFE70120019009E041F208
:1012A0006050C2F2000000680599043100F0F4FCBF
:1012B000FFE717E003980299884208D2FFE70498F5
:1012C0000299884203D3FFE70120019009E041F22F
:1012D0005050C2F2000000680599043100F0DCFCB7
:1012E000FFE7FFE7019806B080BD000080B582B03F
:1012F000019000F02FFD0198806B18B9FFE70120E5
:10130000009002E000200090FFE700F04FFD009801
:1013100002B080BD80B582B0019000F01BFD019845
:10132000806B0199C96B884203D1FFE701200090CF
:1013300002E000200090FFE700F038FD009802B0C6
:1013400080BD000008480068006880F308884FF0FE
:10135000000080F3148862B661B6BFF34F8FBFF30D
:101360006F8F00DF00BF00BF08ED00E080B586B0E2
:101370000490039141F25050C2F200000068C0682E
:10138000C06801900198043000F016FC019890F8B4
:1013900028004007002823D5FFE70198049B8169B6
:1013A0001944039AFFF75EFFC0B1FFE70198049A62
:1013B000694600230B60194602F0F4FE0290029881
:1013C00058B9FFE74FF0500080F31188BFF36F8FDB
:1013D000BFF34F8F0590FFE7FEE700E0FFE707E070
:1013E000019991F8280000F0FE0081F82800FFE73D
:1013F0000198016A884706B080BD000080B58EB0B4
:10140000FFE743F24810C2F20100006807A900227A
:1014100001F04AFD002800F0B880FFE70798B0F11E
:10142000FF3F17DCFFE707A804300290029858B985
:10143000FFE74FF0500080F31188BFF36F8FBFF3C9
:101440004F8F0B90FFE7FEE702990A6848688968AA
:10145000904700E0FFE70798002800F19580FFE73C
:10146000099806900698406928B1FFE7069804306D
:1014700000F0A2FB00E0FFE705A800F0FBF80390F6
:1014800007980190092800F27D800199DFE801F0BA
:101490000505053D456605053D45069991F8280079
:1014A00040F0010081F828000698089B81691944E2
:1014B000039AFFF7D7FE30B3FFE70698016A884723
:1014C000069890F82800400700281AD5FFE70698EC
:1014D000089982690A44694600230B60194602F0A4
:1014E00061FE0490049858B9FFE74FF0500080F374
:1014F0001188BFF36F8FBFF34F8F0C90FFE7FEE7AC
:1015000000E0FFE700E0FFE73DE0069991F82800E2
:1015100000F0FE0081F8280035E0069991F82800D7
:1015200040F0010081F82800089806998861069823
:10153000806958B9FFE74FF0500080F31188BFF37E
:101540006F8FBFF34F8F0D90FFE7FEE70698039B69
:10155000816919441A46FFF785FE14E0069890F851
:1015600028008007002804D4FFE7069800F044FC18
:1015700007E0069991F8280000F0FE0081F82800A5
:10158000FFE700E0FFE7FFE73BE70EB080BD0000AC
:1015900080B584B00390029101F010F8684600F025
:1015A00069F801900098D8BBFFE7029860B9FFE79F
:1015B00003980199884207D8FFE702F0E5FC0398F9
:1015C0000199FFF7D3FE2AE0029858B1FFE741F2F4
:1015D0006050C2F2000000680068B0FA80F0400974
:1015E0000290FFE743F24810C2F20100006803993D
:1015F000019A891A029A00F0F5FC02F0C5FC60B964
:10160000FFE74EF60451CEF200014FF08050086023
:10161000BFF34F8FBFF36F8F00E0FFE7FFE702E0FC
:1016200002F0B2FCFFE704B080BD000081B041F2DF
:101630005450C2F200000068006840B9FFE743F26E
:10164000A801C2F201014FF0FF3008600FE041F243
:101650005450C2F200000068C068C0680090009852
:10166000406843F2A801C2F201010860FFE701B03F
:101670007047000080B582B0019002F0B7F9009089
:10168000009841F24851C2F200010968884206D22E
:10169000FFE700F011F801990120086003E00199CB
:1016A00000200860FFE7009841F24851C2F20001B3
:1016B0000860009802B080BD80B588B0FFE741F2B5
:1016C0005050C2F200000068006800284ED0FFE7CA
:1016D00041F25050C2F200000168C96809680691E1
:1016E0000068C068C06803900398043000F064FA92
:1016F0000398016A8847039890F82800400700285B
:1017000032D5FFE706980399896908440590059842
:10171000069988420FD9FFE7059803994860039816
:10172000006141F25050C2F2000000680399043198
:1017300000F0B2FA17E00398069A694600230B609E
:10174000194602F02FFD0290029858B9FFE74FF0BA
:10175000500080F31188BFF36F8FBFF34F8F079056
:10176000FFE7FEE7FFE700E0FFE7A8E741F250529E
:10177000C2F200021068049041F26051C2F200010E
:10178000086810600498086008B080BD83B000202D
:10179000009040F27830C2F200000068013058B189
:1017A000FFE74FF0500080F31188BFF36F8FBFF356
:1017B0004F8F0190FFE7FEE74FF0500080F3118854
:1017C000BFF36F8FBFF34F8F0290FFE7009808B908
:1017D000FFE7FBE703B0704780B584B00390FFE7F5
:1017E00001A8FFF72DFB029002980199FFF7D0FEA8
:1017F000FFF704FEF4E7000080B582B0019000F02E
:10180000A9FA019890F845008DF80300FFE79DF9CB
:101810000300012816DBFFE70198406A58B1FFE793
:101820000198243002F048FB18B1FFE700F068FD92
:1018300000E0FFE700E005E09DF8030001388DF8C7
:101840000300E4E70199FF2081F8450000F0AEFABB
:1018500000F080FA019890F844008DF80200FFE74C
:101860009DF90200012816DBFFE70198006980B1AD
:10187000FFE70198103002F01FFB18B1FFE700F0FE
:101880003FFD00E0FFE79DF8020001388DF80200FF
:1018900000E000E0E4E70199FF2081F8440000F057
:1018A00085FA02B080BD000080B58AB006900020A5
:1018B000029000F083FE41F25850C2F2000000682E
:1018C00018B9FFE7FFF7DCFA00E0FFE7069843F2FC
:1018D0007001C2F201010968084240F0C580FFE7CB
:1018E000069800B3FFE70698083006909DF81800A8
:1018F0004007B0B1FFE7069820F0070008300690D7
:101900009DF81800400758B1FFE74FF0500080F3F2
:101910001188BFF36F8FBFF34F8F0790FFE7FEE78C
:1019200000E0FFE700E0FFE70698002800F09A805B
:10193000FFE7069843F29C01C2F201010968884260
:1019400000F29080FFE743F21410C2F2010004900D
:1019500000680590FFE705984168069A00209142CB
:10196000019007D2FFE705980068002818BF012002
:101970000190FFE70198C00730B1FFE70598049098
:10198000059800680590E6E7059841F25851C2F2C3
:1019900000010968884263D0FFE7049800680830B6
:1019A00002900598006804990860059840680699B7
:1019B000401A112821D3FFE705980699084403909F
:1019C0009DF80C00400758B1FFE74FF0500080F33E
:1019D0001188BFF36F8FBFF34F8F0890FFE7FEE7CB
:1019E000059840680699401A039948600698059939
:1019F00048600398FFF7D2FB00E0FFE705984268D4
:101A000043F29C00C2F201000168891A016000687B
:101A100043F2A401C2F20101096888420BD2FFE738
:101A200043F29C00C2F20100006843F2A401C2F23A
:101A30000101086000E0FFE743F27000C2F201001C
:101A400002680599486810434860059900200860BD
:101A500043F2B001C2F2010108680130086000E001
:101A6000FFE700E0FFE700E0FFE702F08DFA9DF8F6
:101A70000800400758B1FFE74FF0500080F311888D
:101A8000BFF36F8FBFF34F8F0990FFE7FEE7029818
:101A90000AB080BD41F24C50C2F20000006848B16B
:101AA000FFE741F24C50C2F200000168086D0130BE
:101AB0000865FFE741F24C50C2F200000068704731
:101AC00083B002900191009202980438029002992A
:101AD0004FF080700860029804380290019820F05E
:101AE000010002990860029804380290029941F2BC
:101AF0008D70C0F6010008600298143802900098BA
:101B00000299086002980438029002996FF002006E
:101B10000860029820380290029803B070470000D5
:101B200080B540F24060C2F200000078C0B9FFE723
:101B30004FF47A70F1F788FB40F24061C2F2000185
:101B40000120087040F23E61C2F2000100200880CE
:101B500040F6E071C2F20001086048608860FFE76B
:101B600080BD000086B005908DED040ACDED030A1E
:101B700002919DED030A9DED041A30EE410A8DEDB0
:101B8000010A049800909DED050AB8EEC00A9DED8B
:101B9000011A20EE010A029901208840013801EE65
:101BA000100AB8EEC11A80EE010A9DED001A30EE5F
:101BB000010A06B07047000082B0019001980069E8
:101BC0000090019841688068886001994868896838
:101BD0004860009840680199884205D1FFE7019864
:101BE00080680099486000E0FFE7019900200861E3
:101BF00000990868013808600098006802B07047D2
